:020000040800F2
:100000000000011015BB0308DD4503086DE1000881
:1000100019BC030819BC030819BC03080000000040
:10002000000000000000000000000000294C030850
:10003000254C030800000000214C03085DD900088E
:1000400019BC030819BC030819BC030819BC030830
:1000500019BC030819BC0308F1E100081DE30008FE
:10006000E1E20008A5E2000869E20008E5A800084E
:10007000D5A80008C5A80008B5A80008A5A80008CC
:1000800091A800087DA8000819BC030819BC030842
:1000900019BC030819BC030819BC03082DE20008A9
:1000A00019BC030819BC030819BC030819BC0308D0
:1000B000C1D20008B1D2000819BC0308D5BD0008A0
:1000C000DDBD0008C5BD0008CDBD000819BC030892
:1000D00019BC0308D1DA000819BC030831DA00089A
:1000E000B5E1000819BC03082D4C030819BC03082E
:1000F00019BC0308A1D2000819BC030869A80008AC
:1001000019BC030819BC030819BC030819BC03086F
:1001100019BC030819BC03087DDC010861DC010877
:1001200055A8000841A800082DA8000819A8000833
:1001300005A8000819BC030819BC030819BC03086A
:1001400019BC030819BC030819BC0308E1450308DE
:10015000F1A70008DDA70008C9A7000891D9000889
:10016000B5BD0008BDBD000819BC030819BC0308D3
:1001700019BC030819BC030819BC030819BC0308FF
:0801800019BC030819BC0308B7
:08018800ACB603000100000009
:1001900002020300241F0020201F00200000000096
:1001A000000000000E020200181F0020281F00207F
:1001B00000000000DC0500082700040040250020A6
:1001C000B425002000000000DE050008160008002D
:1001D000C8250020DC25002000000000E205000802
:1001E0000A020A008026002090260020000000005D
:1001F000EA05000801200800802D0020A02D002025
:1002000000000000F40500081A000800682D002016
:10021000A82D002000000000FC05000822000C00B2
:10022000CC3D0020603E00200000000004060008D5
:100230001B00F400B82D00206C3E002000000000E0
:10024000A927020826000E00703F0020603F002012
:1002500000000000FD1A020803123300374200209C
:1002600004420020000000001006000825005A008B
:1002700050410020AA4100200000000000000000C2
:10028000F6110C004441002038410020000000001D
:10029000440600081500700058400020C8400020A7
:1002A00000000000000000002A006000983F0020CD
:1002B000F83F002000000000DDF301080002050007
:1002C000D44200201845002000000000000000007B
:1002D0001E000400DC420020204500200000000039
:1002E0005006000814000200D84900202C4A0020C3
:1002F000000000005406000803010A006C4A0020B8
:10030000784A002000000000560600082C0010006B
:10031000B04D0020A04D00200000000065970208AD
:100320002B002400E44D0020C04D00200000000000
:100330003597020829005000D44C0020084E0020B8
:10034000000000000000000001010400984E0020A1
:10035000A85D0020000000000000000006020C0064
:10036000485D0020AC5D002000000000B9C000081E
:10037000070202007C5D0020B85D00200000000044
:100380006006000802000C00545D0020BC5D0020E7
:100390000000000000000000F7010600D45C00200F
:1003A000C85D00200000000062060008FE01090090
:1003B000AC5F0020C05F002000000000DDBE000830
:1003C0000510060004610020CC6100200000000040
:1003D000680600080E20EA00E45F0020D4610020D7
:1003E0000000000049F401081300040088610020A7
:1003F000C062002000000000700600080201030037
:10040000CF5F0020C46200200000000089AE020817
:100410000B2010001C650020646600200000000016
:1004200074060008F9010400206B0020686B0020AE
:1004300000000000A1C00008FD011E00006B0020AC
:100440006C6B00200000000031C0000806001600A0
:10045000886700208C6B00200000000069F4010810
:10046000FB010100C4660020A46B00200000000016
:10047000D5BE0008FC010900CC7A0020B87B002022
:1004800000000000A1BE00080A101200C072002087
:10049000C47B002000000000840600083400100027
:1004A000F0710020D87B00200000000005F4010856
:1004B00018102C009C710020E87B00200000000038
:1004C0003D9D02080D002400C8710020147C00200E
:1004D00000000000759A03081F000E008C7D0020AC
:1004E000C87D0020000000009606000805020100FB
:1004F000747D0020D87D002000000000A4060008C4
:1005000004008000DC900020DC910020000000004E
:1005100000000000100003009C950020A095002022
:1005200000000000A6060008280010008C9500209E
:10053000A4950020000000001D62020823001000A6
:100540007C950020B495002000000000396202086C
:100550001900050074950020C495002000000000DB
:10056000AA060008F811010070950020CC95002023
:1005700000000000B0060008000104006C95002097
:10058000D095002000000000B20600082F001100E6
:1005900058950020D495002000000000B606000801
:1005A000030001009C970020A49700200000000099
:1005B0000000000012200C00059800205898002030
:1005C00000000000C80600080C002400129800205B
:0C05D000649800200000000061AE0208EA
:1005DC00000020030000C4090000190128280000B5
:1005EC004A01B400D6010000E8036400040A0001CB
:1005FC007E05EA05B4053200C800141E0100640033
:10060C002C01280000000000000000000000000089
:10061C0000000000000000000000000000000000CE
:10062C0000000000000000000000000000000000BE
:10063C0000000000000001000000000000000000AD
:10064C0000000000000001000300040101006C1612
:10065C0000000000013C3C000100000020000301F0
:10066C0000000000010000002B21231E640101008A
:10067C00000001000A01290000300400005A0000AB
:10068C00000090012C01C800640000000000000074
:10069C000100000000050000000000010500000042
:1006AC002801000002009001000000000000000082
:1006BC00000000000000000000000000000000012D
:0806CC00000543464251000005
:1006D40050010000070000000200000000000000BC
:1006E400000000000102030406070809FF000000DF
:1006F4000101000078010408A02A04080000000099
:1007040000000000880104089001040800000000B3
:1007140001200000940104089C010408000000006A
:1007240001400000A001040898190408000000001A
:1007340001200000AC010408B80104080000000016
:1007440004000000BC010408C80104080000000003
:1007540004000000CC01040818290408000000006B
:1007640001000000020100000000803F0000803F03
:100774000000803F000000000000000000000000B6
:100784000000803F000000000000000000000000A6
:100794000000803F00000000000000000000000096
:1007A4000000000000000000000000000000000045
:1007B40000000000000000000000803F0000000076
:1007C400000000000000000000000101FFFF000025
:1007D400FFFFFFFF0001010101000000FF00000016
:1007E40000000000010203040102030406070809D3
:1007F4000101D6015D910208000000000000000024
:1008040014EE0308050804000000000048FE030875
:1008140038F2030834FE03080000000040EE030829
:1008240005080A000000000048FE030838F2030827
:10083400F8EF03080000000000600240106002406E
:1008440000000000000B0000000020000000000079
:100854000000000000600240286002400000000028
:10086400060C000000002000000000000000000052
:10087400006002404060024000000000100D0000D3
:1008840000002000000000000000000000600240A2
:100894005860024000000000160E00000000200016
:1008A4000000000000000000006002407060024090
:1008B40000000000200F00000000200000000000E5
:1008C4000000000000600240886002400000000058
:1008D40026100000000020000000000000000000BE
:1008E40000600240A06002400000000030110000DF
:1008F4000000200000000000000000000060024032
:10090400B860024000000000362F00000000200004
:100914000000000000000000006402401064024077
:10092400000000000038000000004000000000004B
:10093400000000000064024028640240000000003F
:100944000639000000004000000000000000000024
:10095400006402404064024000000000103A0000BD
:10096400000040000000000000000000006402409D
:100974005864024000000000163B000000004000E4
:1009840000000000000000000064024070640240A7
:1009940000000000203C00000000400000000000B7
:1009A400000000000064024088640240000000006F
:1009B4002644000000004000000000000000000089
:1009C40000640240A06402400000000030450000C2
:1009D400000040000000000000000000006402402D
:1009E400B8640240000000003646000000004000E9
:1009F400000000000000000020700020702D720034
:100A04000000000000000000C4100020FFFFFFFFF2
:100A1400FA0000000100000001000000DC2A0408C4
:100A240000000000000000000000000000000000C2
:100A3400C92A0408040000009F8A0308000000007B
:100A440000000000E42A0408010000000000000087
:100A54000000000000000000000000000D00000085
:100A64000000000000000000000000008E91002043
:100A74000100C409000000008C9100200100C40999
:100A8400000000008A9100200100C4090000000059
:100A9400889100200100C409000000008491002016
:100AA4000100C40900000000869100200100C4096F
:100AB40000000000829100200100C4090000000031
:100AC400809100200100C409000000000000000023
:100AD400000000004C030020307D00209CFF2C010E
:100AE40000000000001700200A000000F8EF0308CF
:100AF400A8970020E0150C17000000000217002042
:100B04000800000038F20308011700200500000067
:100B140048FE0308AA9700200200000010F0030812
:100B24000A6100200100FF7F010000000361002032
:100B3400020000001CF00308D85F0020030000003E
:100B44002CF00308D75F0020030000002CF00308FA
:100B5400D66000200000F40101000000D4600020F1
:100B64000000F40101000000D26000200000F40144
:100B740001000000D06000200000F401010000002A
:100B8400CE60002000FF0100EE600020E803D007E3
:100B94000A000000EC600020006401000A0000006C
:100BA400E860002000640100E760002000640100A8
:100BB400ED600020006401000A000000E6600020EF
:100BC400006401000A000000EB60002000640100E2
:100BD4000A000000EA600020006401000A0000002E
:100BE400E9600020006401000A000000E5600020C4
:100BF40000FF01000A000000E460002000FF010083
:100C04000A000000E05F00200000F4010100000081
:100C1400DE5F00200000F40101000000DC5F002022
:100C24000000F40101000000DA5F00200000F4017C
:100C340001000000E06000201400E803010000004F
:100C4400DE600020E803307501000000DD60002054
:100C540000C80100DC60002000C80100DB60002047
:100C640000C80100DA600020006401000A000000EE
:100C7400D960002000FF01000A000000F960002094
:100C840000C80100F860002000C80100F7600020DF
:100C940000C80100F660002000C80100F5600020D3
:100CA40000C80100F460002000C80100F3600020C7
:100CB40000C80100F260002000C80100F1600020BB
:100CC40000C80100182B0408000000000000000008
:100CD4000000000000000000282B040809000000A8
:100CE40000000000F003002004000000302B040882
:100CF4000900000000000000E403002004000000DC
:100D04000C2F04080900000000000000D803002094
:100D140004000000382B0408090000000000000053
:100D2400CC030020040000003C2B04080900000050
:100D340000000000C003002004000000442B04084D
:100D44000900000000000000B403002004000000BB
:100D54004C2B04080900000000000000A803002038
:100D640004000000542B04080900000000000000E7
:100D74009C03002004000000E42A04080100000091
:100D8400000000000000000000000000000000005F
:100D94000D00000000000000000000000000000042
:100DA400682C04080000000000000000000000009F
:100DB40000000000782C040805000000000000007A
:100DC400D65F002000000000E42A040801000000AF
:100DD400000000000000000000000000000000000F
:100DE4000D000000000000000000000000000000F2
:100DF400802C040800000000000000000000000037
:100E040000000000A02A0408000000000000000008
:100E140037160020040000008C2C04080C0000008D
:100E2400018B030844040020000000006837040814
:100E34000C00000019890308380400200000000099
:100E4400902C04080C000000FD8803082C040020EA
:100E540000000000982C04080800000000000000B6
:100E64002004002004000000A02C04080C00000052
:100E74004B8803081404002000000000A82C040878
:100E84000900000000000000080400200400000025
:100E9400B02C04080300000001DA0208FC0300205F
:100EA40000000000E42A0408010000000000000023
:100EB4000000000000000000000000000D00000021
:100EC400000000000000000000000000B42C040832
:100ED400000000000000000000000000000000000E
:100EE400C42C04080C000000000000005C04002076
:100EF40000000000CC2C04080A00000000000000E0
:100F04007061002000000000D82C04080A000000D2
:100F1400000000007861002000000000E02C0408BC
:100F24000A000000000000008061002000000000B2
:100F3400E82C040808000000000000005004002011
:100F440000000000E42A0408010000000000000082
:100F54000000000000000000000000000D00000080
:100F6400000000000000000000000000F02C040855
:100F7400000000000000000000000000000000006D
:100F8400042D04080C00000000000000740400207C
:100F940000000000142D04080400000021DC0208F5
:100FA40000000000000000001C2D04080C000000DC
:100FB400000000006804002000000000302D040838
:100FC4000400000001DC0208000000000000000032
:100FD400E42A0408010000000000000000000000F2
:100FE40000000000000000000D00000000000000F0
:100FF4000000000000000000382D0408000000007C
:101004000000000000000000000000004C2D040857
:101014000700000000000000B004002000000000F1
:10102400582D04080800000000000000A40400205B
:1010340000000000642D0408080000000000000007
:101044009804002000000000702D0408080000002F
:10105400000000008C040020000000007C2D040827
:1010640008000000000000008004002000000000D0
:10107400E42A040801000000000000000000000051
:1010840000000000000000000D000000000000004F
:101094000000000000000000882D0408000000008B
:1010A400000000002B03002000000000942D040821
:1010B4000B000000000000002805002000000000D4
:1010C4009C2D04080B000000000000001C050020FB
:1010D40000000000A82D04080B0000000000000020
:1010E4001005002000000000B42D04080B000000CF
:1010F400000000000405002000000000C02D0408CA
:101104000B00000000000000F804002000000000B4
:10111400CC2D04080B00000000000000EC040020AB
:1011240000000000D42D04080B00000000000000A3
:10113400E004002000000000E02D04080700000087
:1011440000000000D804002000000000E82D04087E
:101154000700000000000000D00400200000000090
:10116400F42D04080B00000000000000C40400205B
:1011740000000000002E0408080000000000000029
:10118400B804002000000000E42A04080100000064
:10119400000000000000000000000000000000004B
:1011A4000D0000000000000000000000000000002E
:1011B4000C2E0408000000000000000000000000E5
:1011C40000000000202E04080800000000000000B9
:1011D40058050020000000002C2E04080800000020
:1011E400000000004C05002000000000382E040818
:1011F400080000000000000040050020000000007E
:10120400442E0408080000000000000034050020FB
:1012140000000000E42A04080100000000000000AF
:101224000000000000000000000000000D000000AD
:101234000000000000000000000000004C2E040824
:10124400000000000000000028030020000000004F
:101254005C2E04080B00000000000000A005002024
:1012640000000000682E04080B00000000000000CD
:101274009405002000000000742E040807000000FC
:10128400000000008C05002000000000802E0408EF
:10129400070000000000000084050020000000009A
:1012A4008C2E040807000000000000007C050020CC
:1012B40000000000982E0408080000000000000050
:1012C4007005002000000000A02E040808000000A3
:1012D400000000006405002000000000E42A040867
:1012E40001000000000000000000000000000000F9
:1012F400000000000D0000000000000000000000DD
:1013040000000000A82E04080000000000000000F7
:101314002803002000000000B42E04080700000089
:1013240000000000EC05002000000000BC2E0408B2
:101334000700000000000000E40500200000000099
:10134400C42E04080700000000000000DC05002093
:1013540000000000CC2E040807000000000000007C
:10136400D405002000000000D42E0408070000006B
:1013740000000000CC05002000000000DC2E040862
:101384000700000000000000C40500200000000069
:10139400E42E04080700000000000000BC05002043
:1013A40000000000EC2E040807000000000000000C
:1013B400B405002000000000F42E0408070000001B
:1013C40000000000AC05002000000000E42A04082E
:1013D4000100000000000000000000000000000008
:1013E400000000000D0000000000000000000000EC
:1013F400000000000000000061D60208F40500208F
:10140400D45F00201B0000003CF00308D35F0020E1
:101414000A320100D25F002001FA0100CE5F0020F1
:1014240000C80100CC5F0020E803D00701000000E1
:101434004352415A59464C4945324251000000003A
:1014440077D60208D5DB0208D00600208588030879
:10145400000000002007002081DB0208BDD802083C
:10146400FC07002099D60208000000009C08002018
:1014740021D70208F1D6020828090020A9D70208BA
:10148400EDD70208C8090020E26000200103010032
:10149400CDD60208A9D60208E00A002051D70208D6
:1014A40041DC02086C0B00201DD8020899DC0208FC
:1014B400340C0020D860002001030100FC2E040835
:1014C4000000000000000000000000000000000018
:1014D400082F04080800000000000000540D00203C
:1014E40000000000102F04080700000000000000A6
:1014F4004C0D002000000000202F0408070000000D
:1015040000000000440D0020000000002C2F0408FF
:1015140007000000000000003C0D00200000000057
:10152400382F04080C00000000000000300D0020DB
:1015340000000000442F04080300000001DA020840
:10154400240D002000000000E42A0408010000002B
:101554000000000000000000000000000000000087
:101564000D0000000000000000000000000000006A
:101574004C2F0408000000000000000000000000E0
:10158400000000005C2F04080A00000000000000B6
:101594000C03040800000000642F04080A00000083
:1015A4000000000058010408000000006C2F04082B
:1015B4000A00000000000000FA60002000000000A3
:1015C400742F04080A00000000000000600D0020D1
:1015D40000000000E42A04080100000000000000EC
:1015E4000000000000000000000000000D000000EA
:1015F4000000000000000000000000007C2F040830
:1016040000000000000000000000000000000000D6
:10161400902F04080300000001DA0208880D00205E
:10162400000000009C2F04080300000001DA0208F7
:101634000417002000000000A42F04080300000089
:1016440001DA02087C0D002000000000AC2F040821
:101654000300000001DA0208700D00200000000001
:10166400E42A04080100000000000000000000005B
:1016740000000000000000000D0000000000000059
:101684000000000000000000B82F04080000000063
:10169400000000000000000000000000C42F040847
:1016A40007000000E5DC0208E40D00200000000053
:1016B400103304080300000001DA0208D80D0020EA
:1016C40000000000D02F04080300000001DA020823
:1016D400CC0D002000000000D82F040803000000F7
:1016E40001DA0208C00D002000000000E02F040809
:1016F40007000000C9DC0208B80D0020000000004B
:10170400843704080300000001DA0208AC0D00204D
:1017140000000000EC2F04080300000001DA0208B6
:10172400A00D002000000000F82F040803000000B2
:1017340001DA0208940D002000000000E42A0408E5
:101744000100000000000000000000000000000094
:10175400000000000D000000000000000000000078
:101764000000000029D60208F1D50208EC0D002083
:1017740089D8020800000000A00E0020000000002C
:10178400000000002C0F002061D8020801DD0208CF
:10179400B80F00200430040800000000000000001E
:1017A40000000000000000001030040803000000E6
:1017B40001DA0208B8100020000000001830040804
:1017C4000300000001DA0208AC1000200000000051
:1017D400243004080300000001DA0208A0100020ED
:1017E40000000000303004080300000001DA0208A1
:1017F40094100020000000003830040802000000AB
:1018040081DD0208000000000000000040300408F0
:101814000200000081DD0208010000000000000059
:101824004C3004080200000081DD020802000000C0
:1018340000000000000000000D0000000000000097
:101844000000000000000000542004080000000014
:10185400000000009DAE0208A08601000400000004
:101864000000000000000000000000000000000074
:101874000000000000000000000000001033040815
:10188400A81F040800000000B14501087D00000005
:10189400060000000000000000000000000000003E
:1018A4000000000000000000000000000000000034
:1018B400583004080000000000000000A1130108D3
:1018C400E803000003000000000000000000000026
:1018D4000000000000000000000000000000000004
:1018E4000000000060300408000000000000000058
:1018F4009DF501081027000003000000000000000F
:1019040000000000000000000000000000000000D3
:1019140000000000000000006C300408000000001B
:101924000D960208E1E90008204E000005000000C1
:1019340000000000000000000000000000000000A3
:10194400000000000000000000000000E021040886
:10195400000000000000000091E4000810270000CF
:101964000100000000000000000000000000000072
:101974000000000000000000000000000000000063
:101984007030040800000000000000006DBE000874
:10199400E803000005000000000000000000000053
:1019A4000000000000000000000000000000000033
:1019B400000000007C30040800000000000000006B
:1019C400C5B00208204E0000030000000000000023
:1019D4000000000000000000000000000000000003
:1019E40000000000000000008C300408000000002B
:1019F40000000000CDAE0208204E000003000000ED
:101A040000000000000000000000000000000000D2
:101A14000000000000000000000000009C300408EA
:101A240000000000000000000D180108400D030034
:101A3400030000000000000000000000000000009F
:101A44000000000000000000000000000000000092
:101A540018210408000000000000000075A003081D
:101A6400102700000100000000000000000000003A
:101A74000000000000000000000000000000000062
:101A840000000000C41F0408000000000000000063
:101A9400355B02081027000003000000000000006E
:101AA4000000000000000000000000000000000032
:101AB4000000000000000000AC300408000000003A
:101AC4000000000005AC0308A0860100010000002E
:101AD4000000000000000000000000000000000002
:101AE400000000000000000000000000B430040802
:101AF4000000000000000000B9980308A08601005F
:101B040001000000000000000000000000000000D0
:101B140000000000000000000000000000000000C1
:101B2400E821040800000000000000007D1A0108FC
:101B3400A00F0000010000000000000000000000F1
:101B44000000000000000000000000000000000091
:101B540000000000C0300408000000000000000085
:101B6400B921020810270000010000000000000055
:101B74000000000000000000000000000000000061
:101B840000000000000000004C22040800000000D7
:101B9400000000008D2B0308102700000100000046
:101BA4000000000000000000000000000000000031
:101BB400000000000000000000000000901F040866
:101BC400000000000000000021DF02081A410000AC
:101BD4000100000000000000000000000000000000
:101BE40000000000000000000000000000000000F1
:101BF400CC3004080000000000000000C9A4030861
:101C0400400D030000000000000000000000000080
:101C140000000000000000000000000000000000C0
:101C240000000000D43004080000000000000000A0
:101C340085A40308400D030000000000000000001C
:101C44000000000000000000000000000000000090
:101C54000000000000000000DC3004080000000068
:101C640000000000755F0208A08601000300000068
:101C74000000000000000000000000000000000060
:101C8400000000000000000000000000010000004F
:101C94000000803FD5800208257D020825800208C7
:101CA40000000000617A02080D4003089540030813
:101CB4006D3F03080000000000000000493E0308D7
:101CC400C93D0308C53D0308C13D0308B53D0308EC
:101CD400B13D0308BD3D0308B93D03083D3E03087B
:101CE400313E0308093E03081D3E0308F53D030881
:101CF400E13D0308CD3D030800FFFF0000000000A4
:101D0400AA5505010000012D202D2D202D2D2D2D4E
:101D1400202D2D2D2D0000000000000000000000EB
:101D2400000000000000AA550B010000AA5507019D
:101D34000000AA5509020000000000000100000094
:101D4400C012AA5503009F000403090412010002F3
:101D54000202004083044057000201020301000014
:101D640009024300020100C032090400000102021A
:101D740001000524001001052401000104240202CD
:101D84000524060001070582030800FF0904010079
:101D9400020A000000070501024000000705810255
:101DA40040000000F98102082587020875820208B4
:101DB400BD7A0208C97D0208CD7A0208E97A0208D0
:101DC400957A0208857A02080000000000000000ED
:101DD4000101010035890308000000007818002083
:101DE400BC370408000000000000000000000000F0
:101DF40000000000A02A0408000000000000000009
:101E0400B81C002004000000683704080C0000001F
:101E140059DB0208A01C002000000000902C0408DC
:101E24000C00000031DB0208941C002000000000BC
:101E3400982C04080800000000000000881C002002
:101E440004000000A02C04080C000000CDD50208FA
:101E54007C1C002000000000B02C040803000000DB
:101E640001DA0208701C002000000000CC370408CE
:101E74000300000001DA0208641C002000000000D6
:101E8400E42A040801000000000000000000000033
:101E940000000000000000000D0000000000000031
:101EA4000000000000000000BC370408000000002F
:101EB400000000000000000000000000A02A040848
:101EC4000000000000000000B81C00200400000016
:101ED4001037040803000000DD890308581C0020A3
:101EE40008000000A02C04080C000000CDD5020856
:101EF4007C1C002000000000B02C0408030000003B
:101F040001DA0208701C002000000000CC3704082D
:101F14000300000001DA0208641C00200000000035
:101F2400E42A040801000000000000000000000092
:101F340000000000000000000D0000000000000090
:101F44000000000000000000D43704080000000076
:101F5400000000000000000000000000A02A0408A7
:101F64000000000000000000B81C00200400000075
:101F7400183704080300000001DA0208AC1C002032
:101F840000000000E42A0408010000000000000032
:101F94000000000000000000000000000D00000030
:101FA400000000000000000000000000AE970020C8
:101FB40088136F1701000000B097002088136F1773
:101FC400000000006C36040800000000000000005F
:101FD40000000000000000007C3604080800000037
:101FE40000000000E81800200400000088360408FF
:101FF4000800000000000000DC18002000000000C1
:10200400B02C040804000000258B03080000000025
:1020140000000000E42A04080100000000000000A1
:102024000000000000000000000000000D0000009F
:10203400000000000000000000000000AC97002039
:1020440088136F17010000006C7D002088136F1740
:10205400000000009589030800000000F418002027
:10206400D29700200100000008FE03086E7D0020C6
:102074000100000014FE0308647D0020020000003B
:102084001CFE0308D69100200000000000000000A0
:10209400D49100200000000000000000D291002034
:1020A4000000000000000000D091002000000000AB
:1020B40000000000CE91002000000000000000009D
:1020C400CC910020000000000000000070160020E9
:1020D4000000000000000000AB9700200200000098
:1020E40028FE0308C83604080000000000000000B1
:1020F40000000000000000007C3604080800000016
:10210400000000007819002004000000883604084C
:1021140008000000000000006C190020000000000E
:10212400B02C0408040000006989030800000000C2
:1021340000000000E42A0408010000000000000080
:102144000000000000000000000000000D0000007E
:10215400000000000000000000000000D836040861
:10216400000000000000000000000000000000006B
:10217400E83604080C000000D9DA0208A819002087
:1021840004000000F43604080C00000081DA0208A0
:102194009C19002004000000003704080C00000013
:1021A400A5DA020890190020000000000C3704088A
:1021B40003000000FD8903088419002008000000C2
:1021C400183704080300000001DA0208AC1C0020E0
:1021D40000000000E42A04080100000000000000E0
:1021E4000000000000000000000000000D000000DE
:1021F400000000000000000000000000DC2A0408C9
:1022040000000000000000000000000000000000CA
:102214002037040804000000418B0308000000007C
:1022240000000000E42A040801000000000000008F
:102234000000000000000000000000000D0000008D
:1022440000000000000000000000000070370408D7
:10225400000000000000000000000000000000007A
:10226400E02204080C00000000000000081A00200E
:10227400040000008037040808000000000000008B
:10228400FC190020040000008C370408080000003A
:1022940000000000F0190020040000009437040836
:1022A4000800000000000000E41900200400000001
:1022B4009C3704080800000000000000D819002022
:1022C40004000000A4370408080000000000000017
:1022D400CC19002004000000AC37040808000000FA
:1022E40000000000C019002004000000B4370408F6
:1022F4000800000000000000B419002004000000E1
:10230400E42A0408010000000000000000000000AE
:1023140000000000000000000D00000000000000AC
:102324000000000000000000818903080000000094
:10233400141A002000000000000000008C1A002085
:1023440000000000000000002C1B00206A7D00201B
:102354000400000034FE0308687D0020E0150C171B
:1023640000000000677D00200800000038F2030828
:10237400667D00200500000048FE03080000000000
:10238400000000007C1B00202D202D2D202D2D2D44
:102394002D202D2D2D000000000000000000000065
:1023A4000000000000000001DC1C00200000000010
:1023B4000000000000000000000000000000000019
:1023C4000000000000000000000000000000000009
:1023D40000000000000000000000000000000000F9
:1023E40000000000000000000000000000000000E9
:1023F40000000000000000000000000000000000D9
:102404000000000000000000000000004300000085
:1024140000000000000000000000000000000000B8
:102424000000000000000000000000004300000065
:102434000000000000000000000000000000000098
:102444000000000000000000000000004300000045
:102454000000000000000000000000000000000078
:102464000000000000000000000000004300000025
:102474000000000000000000000000000000000058
:102484000000000000000000000000004300000005
:102494000000000000000000000000000000000038
:1024A40000000000000000000000000043000000E5
:1024B4000000000000000000000000000000000018
:1024C40000000000000000000000000043000000C5
:1024D40000000000000000000000000000000000F8
:1024E4000000000000000000000000005BBE0308C4
:1024F40037BE0308000000008F390408C52A040809
:102504005031040850310408503104085031040893
:102514005031040850310408503104085031040883
:1025240050310408FFFFFFFFFFFFFFFFFFFFFFFF26
:10253400FFFF00000100415343494900000000002F
:102544000000000000000000000000000000000087
:10255400000000000000415343494900000000000E
:102564000000000000000000000000000000000067
:0C2574000000000000000000010000005A
:10800000002870B51EDB0928044620DD012303EBA0
:1080100083035B00B0FBF3F2092AF8D87BB10E4E64
:10802000B4FBF3F00928CCBF57223022A6FB03E5AE
:10803000024403FB1044EB0801F8012BF0D10023AC
:108040000B7070BD2D230B7040420131DBE73030E7
:1080500001F8010BF3E700BFCDCCCCCC884230B4A3
:108060004FF001042ED301FB04F4B0FBF4F58D4274
:10807000F9D284B1AAB901E0B0FBF4F5092DCCBF67
:10808000572230222A4404FB150003F8012BB4FBCD
:10809000F1F4002CF0D100221A7030BC7047B0FB14
:1080A000F4F5092DCCBF372230222A4404FB1500F9
:1080B00003F8012BB4FBF1F4002CF0D100221A706C
:1080C00030BC70470546002AEBD1D7E72DE9F047D1
:1080D00014461D46064600234FF47A722046294670
:1080E00033F044FBDFF840814B4A4C4F88FB0031B2
:1080F0000144C31782FB002EC3EB611188FB0128EA
:1081000087FB00278644464AC3EBEE2EC1EB011CD9
:1081100082FB0E29A0EB8C0C0744424A86F806C06D
:10812000C3EB27474FEAEE7C08EB010ACCEBA90C26
:1081300082FB07824FEAE1780CEB4C0CC8EB6A1823
:10814000AEEBCC0EC8EB0818DFF8E0C086F804E010
:10815000A1EB880171718CFB0010F917C1EBE212E1
:1081600040F2B55101FB1272C3EBE050B2F5896FDA
:108170004FEA80073CDA40F2DA239A4242DCB2F559
:10818000B77FB4BF4FF0000C4FF0010C4FEA4C0921
:10819000DFF89C8009EB0C0308EBC3031FFA8CFE8D
:1081A000D88A09EB0C0108EBC10116310B2301E061
:1081B00031F8020D824218DA013BF9D1CC44012397
:1081C00038F83C00B37007F2B2770132121ABE449D
:1081D000F270A6F800E0204629464FF47A72002398
:1081E00033F0C4FA3281BDE8F0870133DBB2E9E74E
:1081F0004FF0030EF44640F29650DFF834804FF013
:108200000609CEE74FF0020EDFF82480F44640F274
:1082100029404FF00409C4E7C5B3A29107452EC217
:10822000ABAAAA2A73B06D1689888888792D0311A4
:1082300068CF030803685A1C02601970704700BFBA
:108240002DE9F047089C2578002B804689460CBF15
:108250004FF0200A4FF0300A661C35B3002A29DDA2
:10826000334601E0024698B113F8011B501E002965
:10827000F8D1971E60B13D46013D51464046C84782
:108280006B1C002BF8DC257827EAE770013055B12C
:10829000041B29464046C847301916F8015B002DDB
:1082A000F7D1BDE8F087BDE8F087002A04DC284656
:1082B000BDE8F0870020EBE7571EDCE783684268E3
:1082C000D0ED037A00EB83010133934281ED040A80
:1082D000836004BF0023836000EB830393ED047A83
:1082E000036870EE277A9A42C0ED037A77EEC77A78
:1082F000C0ED037A0CDA013307EE103AF8EEC76AE4
:10830000B7EE007A87EEA60A036030EE070A7047E0
:1083100007EE102AB8EEC77A87EE870A704700BFCB
:1083200090ED057A90ED004AD0ED066AD0ED014A55
:10833000D0ED047A90ED035AD0ED025AA4EE007A03
:10834000B0EE406AB0EE470AB0EE667AA6EE247A46
:1083500067EEC07AA0EE457AE6EE257A80ED057AE2
:10836000C0ED067A704700BFD0ED057A90ED013A76
:10837000D0ED003AD0ED064A90ED024A90ED077A32
:1083800090ED035A90ED086AD0ED045AC0ED067ADC
:10839000F0EE406A27EE830AC0ED056AA3EEA60A56
:1083A00080ED087AA4EE240AA5EE470AA5EEC60AD7
:1083B00080ED070A704700BFD0ED007A90ED017A9A
:1083C00030EE670AE7EE007AB0EE670AC0ED007A99
:1083D000704700BF704700BF0A44914214D030B4C8
:1083E0000139551E41F2210211F8014F082380EA9C
:1083F000042004044CBF82EA40004000013B80B2EC
:10840000F7D18D42F0D130BC704700BF03788B426A
:1084100086BF034B53F82100002080B2704700BF95
:10842000B01E0020044B93F8380018B1002283F8E6
:1084300038200120704700BFB01E002070B4784B78
:1084400093F8392093F83A10013285B083F8392037
:1084500006290CD8DFE801F00E18212E486504002B
:1084600093F83D20824264D0002283F83A2005B080
:1084700070BC7047A0F1BC00B0FA80F0400983F8EE
:108480003A0005B070BC7047CF280CBF0222002212
:1084900083F83A2005B070BC7047C0B2032283F85D
:1084A0003C0083F83D0083F8400083F83A2005B093
:1084B00070BC70472028D7D893F83C2093F83D1023
:1084C000C4B222440028D2B2114414BF04250525A9
:1084D000002083F8414083F83C2083F83D1083F866
:1084E0003A5083F86200C2E793F8622093F83C1098
:1084F00093F83D4093F84150C0B29E1801440132B8
:10850000C9B2D2B20C44954286F8420083F8622088
:1085100083F83C1083F83D40A9D1052283F83A2026
:10852000A5E793F83C2082429ED1062283F83A20A8
:108530009DE793F84020002A96D193F8421009094C
:10854000032909D007298FD193F8431003294AD072
:10855000012283F8382087E7D3F84320D3F8474037
:10856000DFED307AD3F84B00B3F84F502E4905EECB
:10857000902AB2EE047A05EE104AF0EE676AE5EE54
:10858000876A4FF47A7202FB05F2F0EE675AE5EE65
:10859000475A81FB02411144B7EE046AB0EE657A96
:1085A00005EE900AE5EE867AD217C2EBE132FCEED8
:1085B000E66ABCEEC77AFCEEE77ACDED016A8DED96
:1085C000027ACDED037ABDF80440BDF80800BDF88D
:1085D0000C10986002F57A72012583E81400D960C6
:1085E00083F8385040E793F84440B3F84B60B3F851
:1085F0004550B3F84700B3F849101E6014F00F045B
:108600005D609860D960A3D0111D03EB4100013279
:10861000D2B2B0F8450043F82100A242F4DB97E75C
:10862000B01E00200080BB440180008043780078A9
:1086300040EA032010FB01F04FF4807190FBF1F051
:1086400000F30F0000B27047012380F845307047F7
:108650004FF4006383827047BFF34F8F0549064B89
:10866000CA6802F4E0621343CB60BFF34F8F00BFD0
:10867000FDE700BF00ED00E00400FA0570B4037BE5
:1086800004681F2B08D9203B2021626801FA03F3FC
:108690001A421CD170BC70472021226801FA03F3F2
:1086A0001A42F7D0426914495C2000FB021251685B
:1086B0005689CD680868296821F0010129608289FE
:1086C00092B222EA06028281A36070BC70474269BE
:1086D00009495C2000FB021251685689CD68086880
:1086E000296821F001012960828992B222EA0602FA
:1086F0008281E36070BC7047B06700202B4B197813
:10870000002951D02A4B30B41C689888002262623C
:10871000A5899A80284380B20129A08143D09C6812
:1087200098896262A589284380B20229A0819A8132
:1087300039D01C69988A6262A589284380B20329CE
:10874000A0819A822FD09C69988B6262A589284368
:1087500080B20429A0819A8325D01C6A988C626219
:10876000A589284380B20529A0819A841BD09C6AE0
:10877000988D6262A589284380B20629A0819A85D6
:1087800011D01C6B988E6262A589284380B207299C
:10879000A0819A8607D0986B998F42628489214381
:1087A00089B281819A8730BC704700BF906A0020EF
:1087B000946A002010B4037B01681F2B09D9203B69
:1087C00020224C6802FA03F31C4214D15DF8044BDA
:1087D000704720220C6802FA03F31C42F6D00C4AC0
:1087E00040680024147002685DF8044B22F0010216
:1087F00002608B607047064A40680024147002686B
:108800005DF8044B22F001020260CB60704700BFAC
:108810006A2F0020F0B5C40022189200B8498B5886
:108820005B689D8AADB2EEB2F7070A445FD4B70722
:1088300034D5BFF35F8F167EF6B2012E00F0D480E0
:10884000B04D1A8BBFF35F8F221801EB8202167EA8
:10885000022E00F0E480221801EB8202167E032E25
:1088600000F093809A8895F9636092B242F4806236
:108870009A80221801EB8202127E0132964261D167
:1088800095F86520002685F86460002A40F0A080F5
:10889000204401EB800000234375F0BD770752D4DC
:1088A00016F0400600F0D880964D1E8A95F963E0D8
:1088B000176AF6B207F80E605FFA8EFE0EF1010C31
:1088C0004FFA8CFC177E85F863C00CF103029742C7
:1088D000664600F02F81221801EB8202127E944539
:1088E000C7D10EF1020676B285F86360C1E71E8833
:1088F000844D26F400663604360C1E801E88B6B2FF
:1089000046F480661E80967E002785F86370002EF0
:1089100050D095F86460002E49D0221801EB8202F5
:108920000126127E85F86460022A00F0C5802218B4
:1089300001EB8202927D42F001021A82204401EB97
:108940008000037EF0BD6F4D967E012785F865702F
:10895000002E7CD095F86460002E40F084802218B0
:1089600001EB8202527E002A00F0AC801A8895F852
:10897000636092B2013642F4007276B21A8085F8D2
:1089800063601A88D205FCD473E7927E002A3FF414
:1089900069AF95F86420002A3FF464AF9A8895F98E
:1089A000636022F480621204120C9A8061E7D27D27
:1089B000FF2AB2D0221801EB8202967D06F0FE0655
:1089C0001E82D37DFF2BB9D0FF2385F86330B5E736
:1089D0009A8822F4407212042044120C01EB8000A9
:1089E0009A8000234375F0BD927E464D002A3FF4E5
:1089F00028AF95F86420002A3FF423AF1A8822F4A8
:108A000080621204120C1A80BFF35F8F1A8B1A88CF
:108A100085F8656092B242F400721A8022E7927E75
:108A2000002A3FF418AF95F86420002A3FF413AFF2
:108A30001A8895F9636022F480621204120C1A807D
:108A40009A8822F480621204120C9A8011E795F839
:108A50006420002A83D089E715F0800F294D3CD18E
:108A600095F9636005E7167ED2F820E01F88022E94
:108A700095F9636048D927F480673F043F0C1F8055
:108A80001F8AFFB20EF806701F88D2F820E0BFB22E
:108A900047F400771F80F2B21F8A561C76B2FFB2ED
:108AA0000EF806709F88961CBAB276B242F48062C5
:108AB00085F863609A8064E71A8892B242F4006293
:108AC0001A8034E71A8895F9636092B242F4807292
:108AD00001271A8085F8647053E795F96370B7F140
:108AE000FF3F2ED0D669F65D1E8292F818E001375E
:108AF0007AB29645164685F863207FF4BAAE9FE7B2
:108B0000DC5C0020B01E0020BFB247F400771F805D
:108B10001F8AFFB20EF80670F6B21F8AD2F820E064
:108B2000721C52B20336FFB276B20EF8027085F8AC
:108B3000636026E79A8822F480621204120C9A80FD
:108B4000C9E6D77D1F8285F86360957E1DB9127EC8
:108B5000002A7FF4F3AE9A8822F480621204120C89
:108B60009A80EBE6F8B50468C4F30D0405460E469A
:108B700004B32F6820F000F8092840F08880454CA5
:108B8000236923F440732361236943F40073236151
:108B9000236943F0010323613E601FF0EDFF236969
:108BA000092823F00103236171D12B6804332B6062
:108BB0000020F8BD384B394A93422BD902F5804248
:108BC000934226D902F5804293422AD902F5804287
:108BD000934228D902F58032934226D902F5003219
:108BE000934224D902F50032934222D902F5003291
:108BF000934220D902F5003293421ED902F5802219
:108C000093421CD9B3F1016F1BD3052003F094FBF1
:108C1000FBE708241FF0B0FF092814D04FF0FF3005
:108C2000F8BD1024F6E71824F4E72024F2E72824FE
:108C3000F0E73024EEE73824ECE74024EAE7482464
:108C4000E8E75824E6E7134F3B6923F440733B61A0
:108C50003B6943F400733B613B6923F0F8033B61DC
:108C60003B6943F002031C433C613B6943F480339E
:108C70003B611FF081FF3B6923F002033B613B69CD
:108C8000092823F0F8033B613FF473AFC6E76FF0A8
:108C90000100F8BD003C024000400008FF3F000812
:108CA000F8B504460D468E180027B54201D120695B
:108CB000F8BDE368591CE160234415F8012B1A72D2
:108CC0000429F2D1206918B9A1682046FFF74AFFAC
:108CD0002061E760E9E700BF014B186804F0BCBF02
:108CE000741F0020F8B5057B466903681F2D29D93C
:108CF000A5F120045F682021A1400F422A4613D02D
:108D00001022A240D960DA605A68E240D10703D548
:108D1000012202FA04F4DC600446304604F028FF25
:108D2000227B23681F2A20D9A2F1200008215A683B
:108D30008140114200D0D9600422596882400A4221
:108D400021D1F8BD20211C68A9400C422A460CD034
:108D50001022AA4099609A601A68EA40D207DBD5CF
:108D6000012202FA05F59D60D6E7082118689140B6
:108D7000014200D099600421186801FA02F202420F
:108D800003D09A60F8BDDA60F8BDF8BD427A02B946
:108D9000704710B504460368406804F10A0198471B
:108DA0000023637210BD00BF437A5A1C0344D2B241
:108DB00042729972037A934200D802B9704710B593
:108DC00004460368406804F10A019847002363726F
:108DD00010BD00BF50B30123302803FA01F122D0A7
:108DE000312820D032281ED033281CD034281ED061
:108DF00035281CD020281AD0212818D0102812D0AD
:108E0000112810D012280ED013280CD014280ED000
:108E100015280CD0162801D0172806D111F0030010
:108E200018BF012070474A0703D1002070478B0705
:108E3000FBD00120704700BF302829D0312829D02D
:108E4000322829D0332829D0342829D0352829D0D0
:108E5000202829D0212829D0102829D0112829D02C
:108E6000122829D0132829D0142829D0152829D030
:108E7000162805D0172808BF0F2302D000207047FE
:108E80000E23114A03EB4303134493F86200704727
:108E90000023F6E70123F4E70223F2E70323F0E7D8
:108EA0000423EEE70523ECE70623EAE70723E8E7D8
:108EB0000823E6E70923E4E70A23E2E70B23E0E7D8
:108EC0000C23DEE70D23DCE768CF030870B5448888
:108ED00006460D46C4F30B0422460021284633F013
:108EE000D4FF3369094A934209D3094A934206D20F
:108EF000224628461946BDE8704032F0CBBE23B169
:108F000021462846BDE87040184770BDDC050008C2
:108F1000D4060008064B07498B4202D300231846AB
:108F200070471A88C2F30B029042F8D01433F3E76B
:108F300090010008DC050008024A136823EA0000DB
:108F40001060704788610020F8B5174D2B78A52B6D
:108F500028D16B78BE2B25D1022229464FF6FF700F
:108F6000FFF73AFA114FAC1C22884AB1A618BE424C
:108F700018D2052A16D92146FFF72EFA3446F3E710
:108F800021460222FFF728FA0222A118FFF724FA4D
:108F90000634074B641B1C8041F60F53C31A58421A
:108FA0005841F8BD0020F8BD0040000800800008CE
:108FB000923F00202DE9F04FDFF84C914D4F8BB0E0
:108FC0000326A7EB09071822002104A833F05DFF50
:108FD000494BCDF8109005971A69002A04DA474AE0
:108FE0005A6002F188325A6001228DF82420F3225F
:108FF000DA60434B434C1B88ADF8003002226946CF
:1090000004A8FFF74DFE022269464FF6FF70FFF7F6
:10901000E3F9DFF8F8A080464FF0000B544539D350
:109020000AAC002524F8245D0222214604A8FFF79B
:1090300037FE022221464046FFF7CEF940BAC04330
:10904000ADF80800022202A904A8FFF729FE07983C
:1090500078B106ABC0F104022946184433F015FF7D
:10906000089818B9069904A8FFF77CFD002308901A
:1090700007939DF82430089A23B11F490B6943F0E8
:1090800000430B61013E2DD0002A9CD1FFF75CFF0D
:1090900050B32CE065888DF80DB0C5F30B05AB1D02
:1090A000ADF808302388C3F30B02ADF80A201B0B80
:1090B000062202A904A88DF80C30FFF7F1FD062264
:1090C00002A94046FFF788F9616880462A4604A84D
:1090D000FFF7E6FD616840462A46FFF77DF9143444
:1090E00080469BE7002AD1D0052003F025F90BB07C
:1090F000BDE8F08F00800008003C02402301674576
:10910000F8CF03089001000800400008DC050008C3
:109110000378202B024600F10100F9D0092BF7D08B
:109120002D2B2CD02B2B03BF5378B7EE000A024611
:10913000B7EE000AA3F13001C8B209289FED467AC4
:1091400010D8F2EE046A07EE901AF8EEE77A12F8F9
:10915000013FE7EE267AA3F13001C8B20928B0EE4C
:10916000677AF0D92E2B4CD003F0DF03452B0BD0C0
:10917000F7EE007A67EE276A20EE260A70475378EA
:10918000BFEE000A0246D5E710B451782D2959D018
:109190002B290ABF9178501C901C0024A1F13003A8
:1091A000092B53D8002303EB830301EB430310F88F
:1091B000011FA1F13002092AA3F13003F3D9B3F55D
:1091C0009A7F28BF4FF49A73072B42D9DFED236AA9
:1091D0001A46F7EE007A083A072A67EEA67AFAD816
:1091E00003F007032BB1F2EE046A013B67EEA67AA7
:1091F000FBD124B3C7EE276A5DF8044B20EE260AA4
:1092000070475378A3F13001C8B2092802F1010276
:10921000AAD8F2EE046AF0EE665A07EE901AF8EE5B
:10922000E77A12F8013F87EEA66AA3F13001C8B2CF
:10923000092866EEA56A37EE067AEED994E767EE5E
:10924000276AD9E7901C91780124A7E7F7EE007A06
:10925000CFE7F7EE007AC5E70000000020BCBE4C67
:10926000B5EEC00ADFED317AF1EE10FACCBF30EE88
:10927000270A30EE670ADFED2E7A20EE270A30B596
:10928000FDEEC07A87B017EE904A054684EAE47096
:10929000002303A9A0EBE47001930093029327F04D
:1092A000E5FB002CACBF20232D2303A88DF8003054
:1092B00031F0B2FD012803A924D002282DD00328C3
:1092C00005BF3023684668468DF8013033F0E5FD70
:1092D000684631F0A1FD0338C4B2224669462846EB
:1092E00033F012FE00232B55284631F095FD2E2237
:1092F000431C2A540DEB0401E81833F0EBFD28461B
:1093000007B030BD302368468DF801308DF802304B
:109310008DF8033033F0C1FDDAE7302368468DF86D
:1093200001308DF8023033F0B8FDD1E76F12033A07
:1093300000007A442DE9F041064615460846B6FB82
:10934000F2F43CB905FB1464124B1B5D00F8013BC1
:10935000BDE8F081B4FBF2F767B90E4B05FB174788
:1093600005FB1464DA5D00F8012B1B5D00F8013B7E
:10937000BDE8F081B7FBF2F8B8F1000F02D040462B
:10938000FFF7D8FF05FB1878024B13F8082000F808
:10939000012BE3E770000408104B2DE93048D3E9B6
:1093A000004554EA05020BD1034601220020187142
:1093B000587198719A70DA7018801881BDE83088F9
:1093C000074B1A6814EB020B45F1000C5A46634632
:1093D000FEF77CFE0120BDE8308800BFD0250020CC
:1093E000D45D0020F0B402888578154FC3780479E5
:1093F0004179A2F2B27202F0030606EB4606013D85
:1094000005EB8605013B37F815608579008940F248
:10941000B557920807FB0232931903EB430304EBA1
:10942000C303C3EB031301EB8303C3EB031305EB8C
:10943000830300214FF47A72C2FB0301F0BC704732
:1094400068CF0308FAB170B48E18044603E0101A0E
:1094500014D1B14214D014F8012BA2F14103192BFD
:1094600011F8013BA3F1410598BF2032192D03F1FA
:109470002000ECD9D01A01D1002BEAD170BC704782
:10948000002070BC70471046704700BF4FF0FF329D
:10949000FFF7D8BFA0F16103192B98BF20387047A0
:1094A000A0F14103192B98BF20307047202805D028
:1094B000093804288CBF0020012070470120704724
:1094C000613819288CBF00200120704741381928C5
:1094D0008CBF002001207047303809288CBF002045
:1094E00001207047A0F13003092B07D920F020009C
:1094F000413819288CBF0020012070470120704797
:1095000030B402681146531C036011F8024B01602D
:10951000D31C517803609378151D05601B0443EA42
:109520000123D078234343EA006030BC704700BF7A
:109530000368591C1A46016012F8021B0260587831
:1095400041EA0020704700BF03685A1C0260187887
:10955000704700BF38B504460068154632F09AFBE4
:1095600022682A44226038BD036810B40A0E5C1CCD
:1095700004601A7003680A0C5C1C04601A700368AB
:109580000A0A5C1C04601A7003685A1C0260197095
:109590005DF8044B704700BF036810B40A0A5C1CF6
:1095A00004601A7003685A1C026019705DF8044B5D
:1095B000704700BF03685A1C026010B4197003683A
:1095C0000A0A5C1C04601A7003680A0C5C1C0460C4
:1095D0001A700368090E5A1C026019705DF8044B7A
:1095E000704700BF03685A1C026019700368090ABB
:1095F0005A1C0260197070472DE9F047002488B0AA
:1096000080460F461E46A14605AD531C03931178B4
:1096100039B3252933D1931CCDF81090039350789A
:1096200030284ED04FF0000AA0F13003DBB2092BF6
:1096300042D96C2819D0642800F0938024D82528BA
:109640001CD063D9582876D063281BD13178404686
:10965000B847039A531C0393117804360134002948
:10966000D7D1204608B0BDE8F087039B5A1C03926F
:109670001B78642B7CD02AD8252B54D12521404639
:109680000134B847039AC0E7732833D044D975280A
:109690004FD106F1040E30682B4600220A2176468F
:1096A000FEF7DCFC049A0095534639464046FEF727
:1096B000C7FD039A0444A8E704AA03A927F0B2F956
:1096C000B7E7D31C039390784FF0010AACE7732BF4
:1096D00010D05BD9752B3AD0782B96D1A3F15802D4
:1096E000B2FA82F2306852092B4610210436FEF796
:1096F000B5FCD7E73368049A009339460023404607
:10970000FEF79EFD04360444039A7EE70028B9D193
:10971000204608B0BDE8F0876E28B3D1039A3368BD
:1097200004361C6071E72AD9582BD7D0632B8DD013
:109730006BE77828A6D1A0F15802B2FA82F230681D
:1097400052092B461021FEF789FC0436AAE706F1E0
:10975000040E30682B4600220A217646FEF77EFC76
:10976000A0E7331D306829461E46FEF749FC99E7FD
:10977000331D306829461E46FEF742FC92E7002B57
:109780007FF443AF204608B0BDE8F0876E2BC6D00B
:109790003BE700BF0EB400B584B005AB019053F8B1
:1097A000042B0649039301A8FFF726FF019B002223
:1097B0001A7004B05DF804EB03B0704735820008FE
:1097C0002DE9F047484BB3F968708CB00646002F7E
:1097D00056D13D463C460A8840F2B1739A4203D9BD
:1097E0008B78581E0B282FD9002301201946ADF87D
:1097F00024308DF828308DF829308DF82A30ADF8D6
:109800002C309C469A4699461A46984686468DF8CC
:1098100026008DF827000346002CACBF2B242D24F6
:10982000049107950697CDF80CC0CDF808A0CDF8A7
:109830000490CDF800E0304605942C49FFF7AAFFCC
:1098400040460CB0BDE8F08791F803E00EF1FF3020
:109850001E28C9D891F80490B9F1170FC4D891F80F
:1098600005A0BAF13B0FBFD891F806C0BCF13B0F81
:10987000BAD80989B1F57A7FB6D24FF00108CBE7A3
:109880001B4C84FB0734E319FC17C4EB6314C4EBD3
:109890000415A7EB85052DB2002D0846B8BF6D4213
:1098A000FFF7A0FD4FF47A7200238046894631F01D
:1098B0005DFF3C2307FB03074FF47A720023404609
:1098C000494631F053FF24B24FF47A7192B200232B
:1098D000C1FB072309A884EAE477FEF7F7FBA7EBAF
:1098E000E47709A977E700BFB01E002098000408BC
:1098F000898888880FB430B583B006AB0A490B4815
:1099000053F8042B096800680193FFF775FE084CB3
:109910000546206804F08CF90028FAD0284603B0E8
:10992000BDE8304004B07047B05C0020B45C00205B
:10993000741F0020DFED2B7AB4EEE70AF1EE10FA87
:109940004ADDDFED296A9FED297A01E0B0EE670A72
:10995000B4EEC70AF1EE10FA70EE667AF6DC9FED0F
:10996000247AF4EEC77AF1EE10FA38D5DFED1E6AEC
:109970009FED207A01E0F0EE407AF4EEC77AF1EE46
:1099800010FA37EEA60AF6D4DFED1B7AB4EEE70A3A
:10999000F1EE10FA14DDDFED137A37EEC00A60EE57
:1099A000006A9FED166A9FED167ADFED167AA6EE35
:1099B000867A20EE266AE6EE877AA6EE270A7047B8
:1099C000DFED117AB4EEE70AF1EE10FA44BFDFEDF5
:1099D000087A37EEC00AE2E7F0EE407ABFE7B0EE71
:1099E000670AD1E7DB0F4940DB0FC940E4CB1641E2
:1099F000DB0F49C0E4CB16C1DB0FC93F92E741B989
:109A00009730083C15A82ABEDB0FC9BF09B909E089
:109A1000194690FBF1F301FB13030846002BF7D125
:109A2000084670470146FBE7F0EEC07AB0EEE07AF8
:109A3000B4EEE77AF1EE10FAB4BFB0EE676AB0EEBA
:109A4000476AB5EE406AF1EE10FA46D0B4EEE77A16
:109A5000F1EE10FA8CBFF0EE675AF0EE475AC5EE01
:109A6000866A9FED1F3A9FED1F6A9FED1F4A9FED8B
:109A70001F5ADFED1F3ADFED1F4ADFED1F5AA6EE3A
:109A8000C36AE6EEA34AA6EE864AB7EE006AA6EEE1
:109A9000845AA6EEA46AE6EE855AC5EE866AB4EE4E
:109AA000E77AF1EE10FA48BFDFED147AF5EEC00A5E
:109AB00048BF77EEE66AF1EE10FA48BFDFED107AA4
:109AC000B5EEC00A48BF77EEE66AF1EE10FA48BF7D
:109AD000F1EE666AB0EE660A7047DFED076ADEE710
:109AE00039094E3DE3B59E3E88FA163E45FE7F3F5E
:109AF00099FB243F69A2163EA7DFA834DB0FC93FBC
:109B0000DB0F4940DFED317A30EE277AFDEEC76A90
:109B100016EE903A2033402B02D99FED2D0A704764
:109B2000B4EEE70AF1EE10FA4DDD9FED2A6ADFEDA3
:109B30002A6A01E0B0EE677AB4EEE67AF1EE10FA46
:109B400077EE467AF6DC9FED257AF4EEC77AF1EEF1
:109B500010FA35D5DFED1F6A9FED217A01E0F0EEB6
:109B6000407AF4EEC77AF1EE10FA37EEA60AF6D490
:109B7000DFED167AB4EEE70AF1EE10FA1BDCDFED4A
:109B8000197AB4EEE70AF1EE10FA44BFDFED137A6A
:109B900037EEC00A60EE006A9FED136A9FED137AFC
:109BA000DFED137AA6EE867A20EE266AE6EE877A55
:109BB000A6EE270A7047DFED0F7A37EEC00AE9E715
:109BC000B0EE670AD4E7F0EE477ABCE7DB0FC93F97
:109BD00000000000DB0FC940E4CB1641DB0F49C099
:109BE000E4CB16C1DB0FC9BF92E741B99730083CFF
:109BF00015A82ABEDB0F4940FDEEC07A17EE903A59
:109C00002033402B51D8DFED2D7AB4EEE70AF1EE88
:109C100010FA50DDDFED2A6A9FED2A7A01E0B0EEFE
:109C2000670AB4EEC70AF1EE10FA70EE667AF6DC57
:109C30009FED257AF4EEC77AF1EE10FA38D5DFED14
:109C4000206A9FED227A01E0F0EE407AF4EEC77AC6
:109C5000F1EE10FA37EEA60AF6D4DFED1D7AB4EE77
:109C6000E70AF1EE10FA1BDCDFED1A7AB4EEE70A30
:109C7000F1EE10FA44BFDFED147A37EEC00A60EE61
:109C8000006A9FED156A9FED157ADFED157AA6EE55
:109C9000867A20EE266AE6EE877AA6EE270A7047D5
:109CA000DFED067A37EEC00AE9E79FED0E0A70474E
:109CB000B0EE670AD1E7F0EE407AB9E7DB0F494032
:109CC000DB0FC940E4CB1641DB0F49C0E4CB16C122
:109CD000DB0FC93FDB0FC9BF92E741B99730083CA2
:109CE00015A82ABE0000000007EE901AF8EE677A69
:109CF0009FED837A27EE800A20EE070AFDEEC07AF8
:109D000017EE903A2033402B00F28C80DFED7D7A05
:109D1000B4EEE70AF1EE10FA40F3E880B0EE407AD4
:109D20009FED796ADFED796A01E0B0EE677AB4EE13
:109D3000E67AF1EE10FA77EE467AF6DC9FED747A69
:109D4000F4EEC77AF1EE10FA40F1CD809FED6E6A25
:109D5000DFED706A01E0F0EE477AF4EEE67AF1EEBC
:109D600010FA37EE867AF6D4DFED6B7AB4EEE77A46
:109D7000F1EE10FA51DCDFED697AB4EEE77AF1EE3C
:109D800010FA44BFDFED627A37EEC77A27EE076A32
:109D9000DFED635ADFED637ADFED636A9FED635AAF
:109DA000E6EE257A67EE065AE6EE276AF7EE007AC7
:109DB000A5EEA67AF0EE675AE7EE055AE7EE457A89
:109DC00087EEA55ADFED547A30EE277AFDEEC76AAA
:109DD00016EE903A2033402B29D99FED557AF6EEB6
:109DE000006AB7EE006AF7EE004AC4EEA57A0023D7
:109DF000836143610362C36180ED045A67EEA66A22
:109E000027EE866A27EE877AC0ED006AC0ED026A07
:109E100080ED016A80ED037A7047DFED3A7A37EE24
:109E2000C77AB3E7B7EE005AF0EE455ACAE7B4EE88
:109E3000E70AF1EE10FA5FDD9FED336ADFED336A7A
:109E400001E0B0EE677AB4EEE67AF1EE10FA77EE62
:109E5000467AF6DC9FED2E7AF4EEC77AF1EE10FA30
:109E600047D59FED296ADFED2B6A01E0F0EE477AD6
:109E7000F4EEE67AF1EE10FA37EE867AF6D4DFEDFC
:109E8000267AB4EEE77AF1EE10FA27DCDFED237ADA
:109E9000B4EEE77AF1EE10FA44BFDFED1D7A37EE4B
:109EA000C77A27EE076ADFED1E4ADFED1E6ADFED97
:109EB0001E7AE6EE246A67EE064AE6EE267AB7EEEA
:109EC000006AA4EEA77AF6EE006A36EE476AF8EE6C
:109ED000007A27EE277A66EE266A84E7DFED097AB4
:109EE00037EEC77ADDE7B0EE677A3DE7F0EE407A0D
:109EF00024E7B0EE677AC2E7F0EE477AAAE700BF40
:109F000027D4D236DB0F4940DB0FC940E4CB1641E2
:109F1000DB0F49C0E4CB16C1DB0FC93FDB0FC9BF64
:109F200092E741B99730083C15A82ABEF304353FA3
:109F30000000008070B406688E4217D90139751E82
:109F4000002311F8014F0822634013F0800F4FEAFD
:109F5000430318BF83F0D503013ADBB2F5D18D423C
:109F6000EFD1721C0260337070BC70470023F8E7B9
:109F700010B44C09012250F8243001F01F0102FAFC
:109F800001F10B4340F824305DF8044B704700BFEB
:109F90004B0901F01F0150F82320012303FA01F1BE
:109FA000114214BF18460020704700BF0C4B984266
:109FB00013D0A3F5806398420FD003F580439842F5
:109FC0000BD003F58063984207D003F58063984275
:109FD00003D0044B186840087047024B186870475C
:109FE00000040140C47A0020F0B5774B774A87B06F
:109FF0001968914200AF00F0DB800023744A3B6097
:10A000007B60136843F48033136003E03B68B3F56F
:10A01000A04F09D0136803F400337B603B68013321
:10A020003B607B68002BF1D0694B1B6813F4003355
:10A0300018BF01237B607B68012B7BD0654D644B8F
:10A04000654AEA606549586F654A0860AA605E6BB8
:10A05000644C654A654826F080065E635E6F46F094
:10A0600080765E67196B0C431C63596B5963996B5F
:10A070009963196C41F05B5141F47B1141F41F610C
:10A0800041F00F011964596C07F118040A4348F2B2
:10A09000FF715A6444F8101D002621460123FB730A
:10A0A0003E737E73BE731EF07BFD21464FF6FF7339
:10A0B0004F48BB601EF074FD4FF6FF7321464D48BC
:10A0C000BB601EF06DFD21464B481EF069FD214628
:10A0D0004A481EF065FD214649481EF061FD2146B3
:10A0E00048481EF05DFD214647481EF059FD2146B7
:10A0F00046481EF055FD20461EF0BCFB444B454C27
:10A100001B68BA6844484549A4FB03439B09A0FB6C
:10A110000202013B920CB3F1807F0A6007D2404AF1
:10A12000F0200721536085F82300966011601C37EA
:10A13000BD46F0BD264B3B4D1A6C3B4842F0805269
:10A140001A642C684268816844F440442C609C681E
:10A150009C609C6844F400449C609C6844F4A05457
:10A160009C600068120642EA801242F480024908AC
:10A1700042F00802013942EA01425A601A6842F08C
:10A1800080721A601A689201FCD52849104A40F280
:10A1900005700860996821F003019960996841F0A1
:10A1A00002019960936803F00C03082BFAD145E78C
:10A1B00000221A6062B61E4B1B6883F308881D4B91
:10A1C0001B689847FEE700BFFCFF0120EFBEADDE35
:10A1D0000038024000ED00E00005FA05FC6A0020AE
:10A1E00000000008FF916700335F07000000024095
:10A1F0000004024000080240000C0240001002402F
:10A200000014024000180240001C024000200240DE
:10A21000C47A0020D34D621083DE1B43D85D00203A
:10A2200010E000E00070004000000020003C024010
:10A230000000FF1F0400FF1F08B5054B1B6803B19A
:10A240009847044B044A1A6072B6FEF705FA00BF3D
:10A25000B0450020FCFF0120EFBEADDE08B5034B8A
:10A260001B6803B1984772B6FEF7F6F9B0450020B7
:10A270002DE9F04F7A4C54F8204083B0002C00F0C8
:10A28000EA80D4F86090B9F1000F00F0E680D9F8C8
:10A290001050D9F80470734EA16004F16601266075
:10A2A000616104F266264FF40071A661E1602161EC
:10A2B000A765A0464DB3DFF8B4C14FF0000E61466C
:10A2C0004E68B54201F11C0106D00EF1010EBEF13F
:10A2D000100FF5D14FF0000ECEEBCE0E0CEB8E0131
:10A2E000DFF884C10E69DCF830E04FF00C0A4EEA6A
:10A2F000060E461CCCF830E081F818A04E76D9F84E
:10A300000810E1630437676565630546D9F80C00FA
:10A310001F46164600283CD0DFF850C10021634696
:10A320005A68904203F11C0303D001311029F7D180
:10A330000021C1EBC1010CEB81014B4B0A69186B89
:10A34000DFF82CE1104318630B200876681C487670
:10A35000186B024399F81F001A63830991F80DC026
:10A360008DF80530002201234C61C1F808E001A8F6
:10A370008DF806208DF807308DF804C01EF042FAE3
:10A38000A36DD9F80810D9F80C20A2630433216416
:10A39000236594F8650002F05DFF824694F864003E
:10A3A00002F058FF834699F81C00002850D1380766
:10A3B00039D4B2070ED5BAF1000F0BD00B226B1CAB
:10A3C0008AF806208AF80730504699F81D20222185
:10A3D00002F0A8FDF30716D4E36B83B999F81E20A9
:10A3E0008DF8042099F820208DF8063001A89309F3
:10A3F00001228DF805308DF807201EF003FA404643
:10A4000003B0BDE8F08FBBF1000FE5D001350C23A0
:10A410008BF807508BF80630584699F81D202221FA
:10A4200002F080FDD8E70135EDB2BAF1000F04D09B
:10A430000B238AF807508AF8063017F0100F5046A1
:10A440000CBF1221022199F81D2002F06BFDC3E719
:10A4500022F012FCABE7A046D1E7C846CFE700BF29
:10A46000BC5C0020FCCF03080038024068010020DB
:10A47000E58C000800B97047F0B595B0064622F0AB
:10A4800093FDB24DC36802682A600446002B00F0B9
:10A490003881304602F0DEFEAD4BD86618B1292275
:10A4A00000238271C371227A2A2102F03BFD2868C1
:10A4B00002F08AFF22F0E0FB2A68138823F00103F0
:10A4C0001B041B0C13801046FFF770FDA14B984234
:10A4D00000F219810026DFF8B4E29F4F13889F49EC
:10A4E00006F1010CB0FBFCF04FF0030CB0FBF1F0F7
:10A4F00081B2B1FBFCF1AEF80010490039809849F7
:10A500008A429BB200F0098101F580618A4200F025
:10A510000481B2F1804F00F00081A1F580318A42C0
:10A5200000F0FB8001F580618A4200F0F68001F5C1
:10A5300080618A4200F0F1808A498A4200F00281FB
:10A5400001F580618A4200F0FD8023F44071844B64
:10A5500089B29A421180D062168500F0F080824B59
:10A560009A4200F0EC8001219182E2796020002380
:10A57000ADF800009007ADF80230ADF8043002935A
:10A58000ADF80C30ADF80E30ADF81030ADF812303B
:10A5900040F1C78012F0010F0CBF1A4608220423B5
:10A5A000ADF80E20ADF804300023286861790293DD
:10A5B0006A4602F073FA60792B680C2816D8DFE837
:10A5C00010F0F9001500150015000D00150015001C
:10A5D0001500F000150015001500E7001A8B22F495
:10A5E00000621204120C42F400621A83B3F8442091
:10A5F0005E4E5F4F6FEA42426FEA524292B2A3F858
:10A6000044201A8892B242F080021A80E279198CB2
:10A6100092074CBF04220122824092B289B221EA01
:10A6200002011984198C89B20A431A841A88514983
:10A6300092B242F001021A80237D086B1C2202FBB9
:10A6400003634FF0290E1A6900261043086383F84C
:10A6500018E05E76086B02430A635A7B9F605E6176
:10A6600005A801238DF814208DF815308DF81730CA
:10A670008DF816601EF0C6F8E3683F4F18463B6041
:10A680001EF0E2F93868036823F0010303601EF04E
:10A69000DBF905A81EF09AF92B68627938680A96EA
:10A6A00034331344069340F22A3309934FF4806302
:10A6B00022690B93314B0592079340224FF480534C
:10A6C00005A908920C934FF480424FF440330D9249
:10A6D0000F930E961EF08CF9637928683968284C20
:10A6E0000C2B9CBF274A32F81330828988BF33462F
:10A6F00092B2134383810B68012243F010030B6075
:10A70000227015B0F0BD00F1B77303F558531E4920
:10A71000B3FBF1F3013B9EB2DDE623F070039BB285
:10A720000AE712F0010F0CBF002202224FF48073DF
:10A73000ADF80210ADF80C20ADF8103034E700236E
:10A74000138610E71380D06216850CE7E897002087
:10A75000B01E0020FF6BDC02DE97002000350C00ED
:10A76000000001400010004000040140680100208A
:10A77000B587000800380240E49700206C300020C4
:10A78000E097002028F10308006CDC02DC97002031
:10A790009A8B22F400621204120C42F400629A8333
:10A7A00024E79A8B22F008021204120C42F00802ED
:10A7B0009A831BE71A8B22F008021204120C42F053
:10A7C00008021A8312E700BF0348D0F8AC3113B176
:10A7D00000F5D27018477047680100200348D0F890
:10A7E000903113B100F5C47018477047680100201C
:10A7F0000348D0F8743113B100F5B67018477047AC
:10A80000680100200348D0F8583113B100F5A87052
:10A8100018477047680100200348D0F83C3113B155
:10A8200000F59A7018477047680100200348D0F877
:10A83000203113B100F58C70184770476801002073
:10A840000348D0F804310BB1FC301847704700BF03
:10A85000680100200348D0F8E8300BB1E030184719
:10A86000704700BF680100200348D0F8CC300BB11E
:10A87000C4301847704700BF680100200348D0F873
:10A88000B0300BB1A8301847704700BF68010020F6
:10A890000348D0F894300BB18C301847704700BF94
:10A8A000680100200248836F0BB170301847704771
:10A8B000680100200248C36D0BB15430184770473F
:10A8C000680100200248036C0BB13830184770470C
:10A8D000680100200248436A0BB11C3018477047DA
:10A8E000680100200248836803B11847704700BF21
:10A8F00068010020431C00F00E812DE9F04F4FEA63
:10A90000C00808EB00039B00DFF8E8A25AF803B088
:10A9100087B00AEB0304BBF1000F00F0F980143399
:10A920000AEB03010022DBF804704AF803204A60B6
:10A930008A60CA600346A56801900133D4F80C9080
:10A94000DBB2002D00F0E8801522EB71AA71B9F19D
:10A95000000F00F0FA80162289F8062089F80730E7
:10A960009BF80E0022F088F9BB8823F440731B0487
:10A970001B0CBB80284603F0A7FB484603F0A4FB52
:10A980001121284603F08CF91121484603F088F97B
:10A990000826642403E03CB121F02AFD013C28464E
:10A9A00003F0FEFB0028F6D0284603F087FB21F0D9
:10A9B0001FFD284603F088FB21F01AFD013EEED171
:10A9C000484603F07BFB21F013FD284603F076FB9D
:10A9D00021F00EFD284603F077FB21F009FD4846E3
:10A9E00003F072FB019B08EB03040AEB8404284686
:10A9F000637C002B0CBF12213221042202F092FA58
:10AA0000637C002B0CBF122132214846042202F045
:10AA100089FA714B9F4200F0B880704B9F4200F062
:10AA2000BF806F4B9F4200F0A580BB8801996D4AA3
:10AA30006D4C23F440731B041B0CBB803B88884483
:10AA40000AEB880A9BB243F001039AF810103B808E
:10AA5000BD8802A8002918BF14461DF00BFF049AF8
:10AA60006248B2FBF4F325F03F05A0FB02122D046F
:10AA7000900C2D0C0543BD805D4C39884FF49672C7
:10AA800002FB00F284FB02409BB2D217002BC2EB08
:10AA9000A01221F0010108BF01230904013243F48F
:10AAA0000043090C92B239803A84BB833B889BB245
:10AAB00043F001033B803B8823F4816323F00203CE
:10AAC0001B041B0C43F480634FF480423B803A81AB
:10AAD0003B8823F080031B041B0C3B809BF8103049
:10AAE0008DF808300024012302A88DF80B308DF872
:10AAF00009408DF80A401DF085FE9BF80F308DF857
:10AB0000083002A88DF809408DF80A401DF0A0FE1B
:10AB100007B0BDE8F08F7047B9F1000F4BD0162297
:10AB200089F8073089F806209BF80E0022F0A4F877
:10AB3000BB8823F440731B041B0C2846BB8003F026
:10AB4000C3FA484603F0C0FA1EE79BF80E0022F055
:10AB500093F8BB8823F440731B041B0CBB8028466E
:10AB600003F0B2FA484603F0AFFA1121284603F089
:10AB700097F80DE703F5EE331A6A42F400021A6201
:10AB80001A6A22F400021A624FE703F5F2331A6AD6
:10AB900042F400121A621A6A22F400121A6244E79E
:10ABA00003F5F0331A6A42F480021A621A6A22F438
:10ABB00080021A6239E79BF80E0022F05DF8BB882C
:10ABC00023F440731B041B0C4846BB8003F07CFA43
:10ABD000484603F079FADBE6005400400058004094
:10ABE000005C0040009F2400804F120083DE1B4366
:10ABF000D34D6210DC5C0020F0B5C60033189B001A
:10AC0000254DEA585468A28A83B092B20192019A03
:10AC10002B4412F4706F1CBF01221A75019B13F4B0
:10AC2000E06F07460CD1A38A3E4423F4706305EB22
:10AC300086051B041B0C0022A3826A7503B0F0BDBD
:10AC4000238BA38823F480631B041B0CA380019B2C
:10AC50009B05E8D423889805E5D42388D9050ED52B
:10AC60002388DA05FCD423889BB243F40073238045
:10AC700023889B05FCD43846FFF73CFED3E72388A6
:10AC80009BB243F400732380A38823F440731B0416
:10AC90001B0CA380C7E700BFDC5C0020037C012BFA
:10ACA00001D00020704790F914104A1CF9D00329F4
:10ACB000F7DCF0B5CE00384D721805EB820283B098
:10ACC000D2F804E0BEF1000F58D0447D6400E4B235
:10ACD0009475002706244FF0430C82F817C057766E
:10ACE0009376147653751775BEF80430C2F820D0E9
:10ACF0009C05C2F81CD01AD4BEF80030DA050FD477
:10AD00004FF4805401E0013C3BD0BEF800309B057D
:10AD1000F9D4BEF800309BB243F48073AEF8003033
:10AD2000BEF804309BB243F44073AEF804300E44D6
:10AD300005EB86024FF4805401E0013C21D0537DA5
:10AD4000002BFAD105EB86052B7DBBB99DF8006081
:10AD50009DF801109DF802509DF803209DF80440D5
:10AD60009DF8053041EA062142EA052243EA042320
:10AD7000018742878387012003B0F0BD002003B024
:10AD8000F0BD064A1388013308469BB21380FFF7D3
:10AD9000B1FD2046F0E700BFDC5C0020903F0020C2
:10ADA000037A012B01D00020704790F90C104A1C47
:10ADB000F9D00329F7DCF0B5CE00384D721805EB59
:10ADC000820283B0D2F804E0BEF1000F58D0447B79
:10ADD0006400E4B29475002706244FF03B0C82F81F
:10ADE00017C057769376147653751775BEF80430EE
:10ADF000C2F820D09C05C2F81CD01AD4BEF800308E
:10AE0000DA050FD44FF4805401E0013C3BD0BEF88A
:10AE100000309B05F9D4BEF800309BB243F4807338
:10AE2000AEF80030BEF804309BB243F44073AEF885
:10AE300004300E4405EB86024FF4805401E0013CDF
:10AE400021D0537D002BFAD105EB86052B7DBBB9B4
:10AE50009DF800609DF801109DF802509DF80320B8
:10AE60009DF804409DF8053041EA062142EA05229A
:10AE700043EA0423C18202834383012003B0F0BD6F
:10AE8000002003B0F0BD064A1388013308469BB288
:10AE90001380FFF72FFD2046F0E700BFDC5C0020A9
:10AEA000903F0020F0B583B0441C8DF8073001D0EE
:10AEB000032802DD002003B0F0BDC700244E3B187C
:10AEC00006EB83035D68002DF4D04900C9B2997583
:10AED00001240021DA755C7699761C765C7519750B
:10AEE000A9880DF107028905DA611A6214D42B884A
:10AEF000DA050CD44FF4805401E0013C1ED02B88BD
:10AF00009B05FAD42B889BB243F480732B80AB88CB
:10AF10009BB243F44073AB80074406EB87024FF4C7
:10AF2000805401E0013C09D0537D002BFAD106EB9F
:10AF300087073C7D84F0010003B0F0BD054A13880B
:10AF400001339BB21380FFF7D5FC2046B3E700BF67
:10AF5000DC5C0020903F002010B40478012C03D06A
:10AF600000205DF8044B704713465DF8044B0A4619
:10AF7000417990F9040095E72DE9FF41037B013BFE
:10AF8000012B04460E4600F10C0713D801230DF1E6
:10AF900007020221384603F019FA58B19DF807302C
:10AFA000DB0707D5072302AA0321384603F00EFA70
:10AFB000054620B90025284604B0BDE8F0819DF87B
:10AFC0000E8011220A213846FFF7C6FF18F0080F3D
:10AFD000F0D1B4F91A1002A8FDF728FB40423080E6
:10AFE000B4F91C100DF10A00FDF720FB40427080FF
:10AFF000B4F91E1003A8FDF719FB4042B080DAE750
:10B0000037B500F10C04054600220A212046FFF75F
:10B01000A3FF0F220A212046FFF79EFF01AA032368
:10B020001021204603F0D2F99DF8043080336B8361
:10B030009DF805308033AB839DF806308033EB8379
:10B0400000220A212046FFF787FF0DF103020123AA
:10B050000221204603F0BAF901230DF10302092170
:10B06000204603F0B3F911220A212046FFF774FFAE
:10B07000012003B030BD00BF2DE9F04F85B090F83E
:10B0800055300190002B40F0B085019B1B7C012BBB
:10B0900007D101988023417D90F914006B22FFF7BE
:10B0A00001FFBB4CBB4DDFF8F492BB48DFF8F0E288
:10B0B0004FF0640A4FF0100C4FF47A76D9F8043050
:10B0C000C3F30803002B40F08C84EFF31183002BB3
:10B0D00040F087842168826800BF23689942F9D1D3
:10B0E0002F6806FB07F39B1AB3FBF7F306FB01314E
:10B0F00001270091D9F80430C3F30803002B40F076
:10B100003584EFF31183002B40F03084236881688D
:10B1100000BF22689342F9D1D5F800B006FB0BF2CC
:10B12000521AB2FBFBF206FB0323009A9B1AB3F5FB
:10B130007A7FDFD3BAF1010AC0D1019B1B7C012BBE
:10B1400007D101980723417D90F914006822FFF789
:10B15000A9FEDFF84892904EDFF844C24FF0640A2F
:10B160004FF010084FF47A77D9F80430C3F308038E
:10B17000002B40F01984EFF31183002B40F014846E
:10B180002168B26800BF23689942F9D1286807FB9B
:10B1900000F39B1AB3FBF0F307FB01310120009190
:10B1A000D9F80430C3F30803002B40F0C283EFF357
:10B1B0001183002B40F0BD832368B16800BF226873
:10B1C0009342F9D1D5F800B007FB0BF2521AB2FB4B
:10B1D000FBF207FB0323009A9B1AB3F57A7FDFD3B8
:10B1E000BAF1010AC0D1019B1B7C012B07D1019848
:10B1F0005346417D90F914006B22FFF753FEDFF8B0
:10B200009C916548DFF898E14FF0640A4FF0100C0C
:10B210004FF47A76D9F80430C3F30803002B40F0DA
:10B220008E84EFF31183002B40F0898421688268BB
:10B2300000BF23689942F9D12F6806FB07F39B1AD8
:10B24000B3FBF7F306FB013101270091D9F8043075
:10B25000C3F30803002B40F04F83EFF31183002B5F
:10B2600040F04A832368816800BF22689342F9D185
:10B27000D5F800B006FB0BF2521AB2FBFBF206FB4C
:10B280000323009A9B1AB3F57A7FDFD3BAF1010A40
:10B29000C0D1019B1B7C012B06D101986B22417D03
:10B2A00090F91400FFF7FEFDDFF8F0903A48DFF860
:10B2B000F0E04FF00F0A4FF0100C4FF47A76D9F807
:10B2C0000430C3F30803002B40F01C84EFF3118318
:10B2D000002B40F017842168826800BF23689942E0
:10B2E000F9D12F6806FB07F39B1AB3FBF7F306FBB4
:10B2F000013101270091D9F80430C3F30803002B72
:10B3000040F0DD82EFF31183002B40F0D8822368F8
:10B31000816800BF22689342F9D1D5F800B006FBDE
:10B320000BF2521AB2FBFBF206FB0323009A9B1AA4
:10B33000B3F57A7FDFD3BAF1010AC0D1019A92F84E
:10B340004F30127C042B34BF18231A23012A06D154
:10B3500001981B22417D90F91400FFF7A3FDDFF84F
:10B360003C900D48DFF838E04FF00F0A4FF0100C1A
:10B370004FF47A76D9F80430C3F30803002B40F079
:10B380001784EFF31183002B40F012840AE000BF12
:10B39000D45D0020D85D002010E000E000ED00E06A
:10B3A000D05D00202168826800BF23689942F9D1EE
:10B3B0002F6806FB07F39B1AB3FBF7F306FB01317B
:10B3C00001270091D9F80430C3F30803002B40F0A3
:10B3D0005982EFF31183002B40F054822368816877
:10B3E00000BF22689342F9D1D5F800B006FB0BF2FA
:10B3F000521AB2FBFBF206FB0323009A9B1AB3F529
:10B400007A7FDFD3BAF1010AB4D1019B1B7C012BF7
:10B4100007D101981823417D90F914001C22FFF7F1
:10B4200041FDDFF8D492B248DFF8C8E24FF00F0ACE
:10B430004FF0100C4FF47A76D9F80430C3F30803B8
:10B44000002B40F09983EFF31183002B40F094839D
:10B450002168826800BF23689942F9D12F6806FBF2
:10B4600007F39B1AB3FBF7F306FB013101270091A9
:10B47000D9F80430C3F30803002B40F0E681EFF362
:10B480001183002B40F0E1812368816800BF2268AE
:10B490009342F9D1D5F800B006FB0BF2521AB2FB79
:10B4A000FBF206FB0323009A9B1AB3F57A7FDFD3E6
:10B4B000BAF1010AC0D1019B1B7C012B08D1019874
:10B4C0001A2290F84E30417D90F91400FFF7EAFC03
:10B4D000DFF824928648DFF81CE24FF00F0A4FF0A5
:10B4E000100C4FF47A76D9F80430C3F30803002B1C
:10B4F00040F0B082EFF31183002B40F0AB82216863
:10B50000826800BF23689942F9D12F6806FB07F3D0
:10B510009B1AB3FBF7F306FB013101270091D9F821
:10B520000430C3F30803002B40F07281EFF3118362
:10B53000002B40F06D812368816800BF2268934230
:10B54000F9D1D5F800B006FB0BF2521AB2FBFBF2B0
:10B5500006FB0323009A9B1AB3F57A7FDFD3BAF177
:10B56000010AC0D1019B1B7C012B08D10198192233
:10B5700090F85030417D90F91400FFF793FCDFF80C
:10B5800078915B48DFF86CE14FF0640A4FF0100CE3
:10B590004FF47A76D9F80430C3F30803002B40F057
:10B5A0003D82EFF31183002B40F0388221688268DE
:10B5B00000BF23689942F9D12F6806FB07F39B1A55
:10B5C000B3FBF7F306FB013101270091D9F80430F2
:10B5D000C3F30803002B40F0FE80EFF31183002B30
:10B5E00040F0F9802368816800BF22689342F9D156
:10B5F000D5F800B006FB0BF2521AB2FBFBF206FBC9
:10B600000323009A9B1AB3F57A7FDFD3BAF1010ABC
:10B61000C0D1019B1B7C012B07D101981223417DD6
:10B6200090F914003722FFF73DFCDFF8CC80304959
:10B63000304F4FF00F094FF0100E4FF47A70D8F8DA
:10B640000430C3F30803002B40F03E82EFF3118374
:10B65000002B40F0398222688E6800BF23689A422E
:10B66000F9D1D5F800C000FB0CF39B1BB3FBFCF336
:10B6700000FB023300930126D8F80430C3F308031B
:10B68000002B40F08C80EFF31183002B40F087807B
:10B690002368D1F808A000BF22689342F8D1D5F8FA
:10B6A00000B000FB0BFCACEB0A0CBCFBFBFC00FB92
:10B6B00003C3009A9B1AB3F57A7FDDD3B9F1010970
:10B6C000BDD1DFF834800A490A4F4FF00F094FF01F
:10B6D000100E4FF47A70D8F80430C3F30803002B2F
:10B6E00040F0D481EFF31183002B40F0CF8105E0CF
:10B6F00010E000E0D05D002000ED00E022688E68E0
:10B7000000BF23689A42F9D1D5F800C000FB0CF3C2
:10B710009B1BB3FBFCF300FB023300930126D8F81C
:10B720000430C3F30803F3B9EFF31183DBB92368E3
:10B73000D1F808A000BF22689342F8D1D5F800B034
:10B7400000FB0BFCACEB0A0CBCFBFBFC00FB03C3DB
:10B75000009A9B1AB3F57A7FE1D3B9F10109BAD106
:10B7600005B0BDE8F08FEFF3118A8EF312888A6876
:10B770000B68DB0344BF3E608A682368D7F800C0CB
:10B780005FFA8AFA8AF31188D5F800A09C4400FB7E
:10B790000AF39B1AB3FBFAF300FB0C33D8E7EFF381
:10B7A000118A8EF312888A680B68DB0344BF3E60FF
:10B7B0008A682368D7F800C05FFA8AFA8AF311888A
:10B7C000D5F800A09C4400FB0AF39B1AB3FBFAF3E4
:10B7D00000FB0C336DE7EFF311888CF3128881685E
:10B7E0000368DB0344BFCEF8007081682368DEF88D
:10B7F00000205FFA88F888F31188D5F800801A4491
:10B8000006FB08F35B1AB3FBF8F306FB0233F8E61A
:10B81000EFF311888CF3128881680368DB0344BF5F
:10B82000CEF8007081682368DEF800205FFA88F89F
:10B8300088F31188D5F800801A4406FB08F35B1AD8
:10B84000B3FBF8F306FB023384E6EFF311888CF3C5
:10B85000128881680368DB0344BFCEF800708168FA
:10B860002368DEF800205FFA88F888F31188D5F89D
:10B8700000801A4406FB08F35B1AB3FBF8F306FBDF
:10B88000023310E6EFF311888CF3128881680368A5
:10B89000DB0344BFCEF8007081682368DEF8002027
:10B8A0005FFA88F888F31188D5F800801A4406FBFF
:10B8B00008F35B1AB3FBF8F306FB02339DE5EFF3E5
:10B8C00011888CF3128881680368DB0344BFCEF8CB
:10B8D000007081682368DEF800205FFA88F888F33A
:10B8E0001188D5F800801A4406FB08F35B1AB3FBF5
:10B8F000F8F306FB023319E5EFF311888CF3128895
:10B9000081680368DB0344BFCEF800708168236858
:10B91000DEF800205FFA88F888F31188D5F80080F7
:10B920001A4406FB08F35B1AB3FBF8F306FB023379
:10B93000A7E4EFF3118E88F31288B1683368DB0354
:10B9400044BFCCF80000B1682368DCF800205FFA3F
:10B950008EFE8EF31188D5F800E01A4407FB0EF333
:10B960005B1AB3FBFEF307FB023334E4EFF31188F9
:10B970008CF3128881680368DB0344BFCEF8007043
:10B9800081682368DEF800205FFA88F888F3118860
:10B99000D5F800801A4406FB08F35B1AB3FBF8F3F2
:10B9A00006FB0233FFF7C1BBEFF3118288F3128865
:10B9B000B0683368D90303D50123CCF80030B068F0
:10B9C0002368DCF80010D2B282F311882A68194487
:10B9D00007FB02F31B1AB3FBF2F307FB0131FFF77E
:10B9E000DDBBEFF311828CF3128887680368D903FB
:10B9F00003D50123CEF8003087682368DEF80010F5
:10BA0000D2B282F311882A68194406FB02F3DB1BC9
:10BA1000B3FBF2F306FB0131FFF76ABBEFF31182D0
:10BA20008CF3128887680368D90303D50123CEF805
:10BA3000003087682368DEF80010D2B282F31188E4
:10BA40002A68194406FB02F3DB1BB3FBF2F306FB87
:10BA50000131B9E5EFF311828CF31288876803682E
:10BA6000D90303D50123CEF8003087682368DEF8B8
:10BA70000010D2B282F311882A68194406FB02F33F
:10BA8000DB1BB3FBF2F306FB013146E5EFF3118656
:10BA90008EF31288D1F808C00B68DA0303D50123AE
:10BAA0003B60D1F808C023683A68F6B286F3118883
:10BAB0002E681A4400FB06F3A3EB0C03B3FBF6F36A
:10BAC00000FB0233009329E6EFF311868EF3128810
:10BAD000D1F808C00B68DA0303D501233B60D1F825
:10BAE00008C023683A68F6B286F311882E681A44B3
:10BAF00000FB06F3A3EB0C03B3FBF6F300FB0233EE
:10BB00000093B8E5EFF311828CF31288876803681D
:10BB1000D90303D50123CEF8003087682368DEF807
:10BB20000010D2B282F311882A68194406FB02F38E
:10BB3000DB1BB3FBF2F306FB0131FFF7DABBEFF3DC
:10BB400011828CF3128887680368D90303D5012317
:10BB5000CEF8003087682368DEF80010D2B282F396
:10BB600011882A68194406FB02F3DB1BB3FBF2F3CE
:10BB700006FB0131FFF768BBEFF311828CF31288EB
:10BB800087680368D90303D50123CEF8003087689E
:10BB90002368DEF80010D2B282F311882A681944B3
:10BBA00006FB02F3DB1BB3FBF2F306FB01315DE4A2
:10BBB000EFF311828CF3128887680368D90303D5E9
:10BBC0000123CEF8003087682368DEF80010D2B277
:10BBD00082F311882A68194406FB02F3DB1BB3FBCE
:10BBE000F2F306FB0131FFF7EBBB1C09013C032C10
:10BBF00003F00F0300F2B980634A32F8140040FAF0
:10BC000003F2D20740F1B180012505FA03F3013BAD
:10BC100018402FF0FBFD5D4B5D4F1E5D064417EB9A
:10BC2000C60400F0A28020220023A271E37157F81D
:10BC30003600584A00F13F4303F57E039B0AD25C6D
:10BC400002F01F035209032A05FA03F300F097805C
:10BC5000042A00F08F80022A00F08280A3880293D9
:10BC600002A9002503951CF09BFFA088019A4A4B6E
:10BC7000D360B0FA80F0C0F11F00431C53D0C3B2B0
:10BC800003F0FC0E0EF1804E0EF59C3E03F0030215
:10BC9000910057F83630DEF80860404FDFF80CC1ED
:10BCA0000F228A4026EA0202019E03F13F430C362E
:10BCB00047F8206003F57E03CEF80820C3F38722FF
:10BCC000DEF80830364F8A4001261A4306FA00F3A0
:10BCD000CEF808207B613968DFF8D4E0DA43114000
:10BCE0003960796811407960396819433960B968F9
:10BCF0001140B960F9680A402A49FA60DCF800701E
:10BD000008441F4390F8BC20CCF800701EF80200D5
:10BD1000F0280BDC002B3FF4B8A921490A68134333
:10BD20000B60FFF7B2B901238340F3E7114402A887
:10BD300091F8CC308DF80830F02103238DF80930CC
:10BD40008DF80A508DF80B600EF802101CF05AFDA9
:10BD5000A388B3FA83F3C3F11F0306FA03F3D9E709
:10BD6000114A516C0B43536478E7019A0A4BD36034
:10BD7000FFF78BB90C4A116B0B4313636EE70A4A4A
:10BD8000116C0B43136469E7F0EF0308ECEF030851
:10BD9000105E002048F10308498600082C1F00208F
:10BDA000003C014068CF030800380240083C0140D5
:10BDB0006C1F00200220FCF72DBD00BF0220FEF703
:10BDC0001BBF00BF0120FCF725BD00BF0120FEF70F
:10BDD00013BF00BF0020FCF71DBD00BF0020FEF711
:10BDE0000BBF00BF1549164B16480A6810B48C6883
:10BDF0001549B2FBF4F203FB02F30360D1F888208B
:10BE0000124B134C42F47002C1F888201A680020CB
:10BE100042F001021A6098601A6822F0847222F4DB
:10BE200080321A605C601A684FF0006422F480224D
:10BE30001A60D8608C605DF8044B704700000020E9
:10BE400040420F00C47A002000ED00E000380240BC
:10BE500010300024044B4FF4F0700A21022283E8D2
:10BE60000700FFF7BFBF00BF0000002038B50B4C34
:10BE700023688BB15A68821A002A054604DA0CE05E
:10BE80005A68AA1A002A07DB9A68226018461A68BC
:10BE900090472368002BF3D138BD38BD704C00208B
:10BEA0000B4B002210B4027203F59C74012102E0D6
:10BEB000072A09DC9979890702D519798154013259
:10BEC0009C4203F11803F3D15DF8044B704700BFA7
:10BED0009CEE030817230370704700BF012316214F
:10BEE000152241704271037203700371704700BFE5
:10BEF000436A8269D154436A0169826B01338B4280
:10BF000028BF00234362002A2FD0EFF31182502371
:10BF100083F31288836B1968C9072CD470B45E68E8
:10BF20006EB9456A816A8D4217D084690C44DC6021
:10BF30000ED9691A59608562002180F85C10196871
:10BF400041F00101D2B2196082F3118870BC7047D0
:10BF50000469611A59608662EEE7012380F85C305B
:10BF6000D2B282F3118870BC7047826DD36843F0FF
:10BF70008003D3607047D2B282F31188704700BF4C
:10BF8000426B10B462B1C36CC2684469D11A013B00
:10BF9000615C5DF8044B08BF1346C364C8B27047C8
:10BFA000016A4369C4685B5C0131A14228BF114644
:10BFB00001625DF8044BD8B2704700BF836B13B1C8
:10BFC00090F85C007047836A406A181AB0FA80F0F3
:10BFD00040097047416A836A99420AD3CB1A816B40
:10BFE000026961B14968501E0B4483420AD2C01AEB
:10BFF000704702691144CB1A816B0029F2D1501E9F
:10C00000C01A704700207047436B43B1C26C5B6835
:10C0100093422FBF981AC0689B1AC0187047C26914
:10C02000036A9A422FBFD01AC0688018C01A70479E
:10C030000A4B30B503F10C0493F900205D78072A10
:10C04000C8BF143A811804338D7213F8025C85540A
:10C0500013F8012C0A75A342EED130BD3CD0030881
:10C0600003682DE9F041DF691FB13B46BDE8F041AF
:10C070001847002A164611DD04460D460E4400E01E
:10C0800023689B68204698470028F9D0236815F854
:10C09000011B1B6820469847AE42F1D1BDE8F081F4
:10C0A00010B4302142243322002304704170827086
:10C0B000C3705DF8044B7047002318220360827040
:10C0C000392243604271012283600272C372704759
:10C0D000038A2DE9F0478589ADB21D4029D00F466E
:10C0E00006464FF000484FF00009B5FA85F328FAEC
:10C0F00003F2D24391B21B3B15403182042B16D878
:10C10000DFE803F03129211903007B6A002B32D0CC
:10C1100003F1FF3A1FFA8AFAC7F824903C6A34B157
:10C1200023682046514698476468002CF8D1002DBA
:10C13000DBD1BDE8F0873868716B036889B2984736
:10C14000002DD2D1F5E77868B16B036889B29847C2
:10C15000002DCAD1EDE7B868F16B036889B2984742
:10C16000002DC2D1E5E7F868316C036889B29847C1
:10C17000002DBAD1DDE7F36A1FFA83FACEE700BFDC
:10C1800030B50446806D61718389A26823F4005341
:10C190001B041B0C838185B0A379009213F0040269
:10C1A0002ED04FF4805213F00203ADF804203CD19E
:10C1B000ADF806304FF480630022ADF8083011F07E
:10C1C0000103ADF80C2026D1ADF80A3008238A0708
:10C1D000694648BFADF80A301CF096FBA379A26D02
:10C1E00013F0080F938A1BD123F008031B041B0CC8
:10C1F000938293899BB243F40053938105B030BD81
:10C2000013F00203ADF8042012D04FF4005513468A
:10C21000ADF80650D0E70423ADF80A300C23D6E77A
:10C220009BB243F008039382E3E74FF40053BFE768
:10C23000ADF80630C0E700BF10B50446806DA160C0
:10C24000838923F400531B041B0C8381A37984B0DE
:10C2500013F00402009133D04FF4805213F0020324
:10C26000ADF804203CD1ADF806304FF4806362791C
:10C27000ADF80830D1074FF00003ADF80A30ADF843
:10C280000C3045BF0423ADF80A3008230C2369465F
:10C29000920748BFADF80A301CF036FBA379A26DB7
:10C2A00013F0080F938A16D123F008031B041B0C0C
:10C2B000938293899BB243F40053938104B010BDE1
:10C2C00013F00203ADF804200DD04FF400511346D3
:10C2D000ADF80610CBE79BB243F008039382E8E782
:10C2E0004FF40053BFE7ADF80630C0E7022828BF7F
:10C2F000022010B4084C094B207000EB8002C0EB08
:10C30000C20207495DF8044B013003EB4203C0B29F
:10C310000B602DF08FBF00BF05980020E45F002068
:10C320008465002008B51DF081FDFCF743FEBDE8E3
:10C3300008401DF063BD00BF2DE98048013085B085
:10C34000C3B203938B4D8C4F8C4C8D4E0A230293BA
:10C350003220DFF8309220F011FA4FF4FA7A4FF0E1
:10C36000100C4FF47A70D9F80430C3F30803002B93
:10C3700040F0C180EFF31183002B40F0BC802968AE
:10C38000A26800BF2B689942F9D1D7F800E000FB02
:10C390000EF39B1AB3FBFEF300FB01314FF0010ECD
:10C3A0000191D9F80430C3F30803002B40F08780D3
:10C3B000EFF31183002B40F082802B68A16800BF4F
:10C3C0002A689342F9D1D7F800B000FB0BF2521A59
:10C3D000B2FBFBF200FB0323019A9B1AB3F57A7FB1
:10C3E000DFD3BAF1010ABED1039B002B40F0BD8020
:10C3F0004FF47A7ADFF88C9150464FF0100CD9F850
:10C400000430C3F30803002B40F09280EFF3118354
:10C41000002B40F08D802968A26800BF2B689942EC
:10C42000F9D1D7F800E000FB0EF39B1AB3FBFEF343
:10C4300000FB01314FF0010E0191D9F80430C3F334
:10C44000080303BBEFF31183EBB92B68A16800BFAE
:10C450002A689342F9D1D7F800B000FB0BF2521AC8
:10C46000B2FBFBF200FB0323019A9B1AB3F57A7F20
:10C47000E3D3BAF1010AC2D1029B013B02937FF4DC
:10C4800067AFFDF7D9FEEFF311888CF31288A1682E
:10C490002368DB0344BFC6F800E0A1682B6832685C
:10C4A0005FFA88F888F31188D7F800801A4400FBF7
:10C4B00008F35B1AB3FBF8F300FB0233D4E7EFF3A6
:10C4C00011888CF31288A1682368DB0344BFC6F887
:10C4D00000E0A1682B6832685FFA88F888F3118859
:10C4E000D7F800801A4400FB08F35B1AB3FBF8F39B
:10C4F00000FB023370E7EFF311828CF31288D4F85B
:10C5000008E02368D90303D501233360D4F808E099
:10C510002B683168D2B282F311883A68194400FB63
:10C5200002F3A3EB0E03B3FBF2F300FB013135E79B
:10C53000EFF311828CF31288D4F808E02368D90352
:10C5400003D501233360D4F808E02B683168D2B2F8
:10C5500082F311883A68194400FB02F3A3EB0E033F
:10C56000B3FBF2F300FB013164E718461FF08EFFC6
:10C570003EE700BFD45D0020D85D002010E000E061
:10C58000D05D002000ED00E038B5484B5A8999890C
:10C59000914224BF00225A81198ADA89914224BF2C
:10C5A0000022DA81DA78CAB1072A41496AD091F8C3
:10C5B0005300404D012400210A282C709C70D97131
:10C5C0005DD00C2807D0002A6CD0DFED3B7A072A1B
:10C5D0000ED00A2862D0DFED397A09E0344A92F8A9
:10C5E00053000A2856D00C285BD1D979DFED347A74
:10C5F000344C9FED350AA278002918BFF0EE407A3E
:10C60000062A04D8314901EB820191ED030A217910
:10C6100079B1013A032A0BD8F7EE007A87EE800A47
:10C620002FF078FC2388984228BF1846208038BD18
:10C6300038BD9B781F4A07EE103A1178B8EEC77ADA
:10C6400067EE277A07EE101AB8EEC77A27EE277A38
:10C65000B4EEC70AF1EE10FAEADD80EE277AFDEEBD
:10C66000C77A17EE903A102BA8BF1023012BB8BF42
:10C670000123DBB28B4238BF0B46137038BDDFEDB0
:10C68000147AA4E791F853000A2803D00C28ACD000
:10C69000D9799AE7D979DFED0E7AA9E7DFED0D7A3E
:10C6A000A6E7D979DFED047AA2E700BFC0720020C7
:10C6B000D4720020709500206F1203396F12833AF4
:10C6C0000AD7A339886700206F1203383CD00308CB
:10C6D0005304E9380F506E3A2DE9F047AC4FAD4E98
:10C6E0001DF0A4FBBE421ED2DFF82483DFF82493A2
:10C6F0004446258862197DB14A450DD2052D0BD9D6
:10C7000033886188C3F30B03994200F0E380144639
:10C7100025886219002DEFD1716830461436FCF778
:10C72000D5FBBE42E4D39C4A1378A3F1170102293A
:10C730000FD99A4911F83300002840F0FA80D80048
:10C740000144497829B1964911F833300BB91823BF
:10C750001370944B5A78022A00F2DC809249934875
:10C7600002EB420201EB82011A780160022A00F218
:10C77000DA8002EB82018E4BC2EBC10203EB420373
:10C78000998C5A8C8B4C9142236001D300225A849D
:10C79000894B9A78042A00F0ED8032B91A88B2F5F4
:10C7A000F07F84BF4FF4F0721A80844DFFF7ECFEE7
:10C7B0002B68834A1A40002A00F0E580D80700F170
:10C7C000D480590400F1CC801A0700F1BB809B048F
:10C7D00000F1BF8024F018FF10B97A482DF04AF913
:10C7E0004020FCF7A9FB4FF40070FCF7A5FB4FF4C9
:10C7F0008020FCF7A1FB4FF40010FCF79DFB4FF0ED
:10C800000070FCF799FB4FF08060FCF795FB14F08B
:10C8100085FF002130226C4830F037FB206813F090
:10C82000EDFE6A4B256803F1500102E004339942A2
:10C830007DD01A78002AF9D19C78D8788442F5D234
:10C840006349644B0A7028461D602CF061FA624A05
:10C8500062491079624A634B1160C822642111FB5E
:10C860000021002259609A60DA601A615A619A6167
:10C87000DA6183F8202083F821201AF0B3FF5A4BA5
:10C880009FED5A5A1B885A4A9FED5A6A50795A4965
:10C8900006EE903AF8EEE66A1388C5EE265A07EEE1
:10C8A000103A53881279C1ED005A07EE903AB8EE6B
:10C8B000C77A524BF8EEE77A18725A7227EE067A68
:10C8C00067EE867ABDE8F04783ED017AC3ED007A22
:10C8D0001DF094BA63799B077FF419AF716894F8DF
:10C8E00004A03046FCF7F2FA3388BAEB133F04D0C9
:10C8F0001436BE42FFF4FCAE15E773887068AA1FB9
:10C90000C3F30B039A4204F10601A8BF1A462FF0A5
:10C91000C1F9EDE700225A701A78244822490160D3
:10C92000022A7FF626AF00221A70214B28E7012247
:10C9300086E7D8000C186468002C7FF401AF172438
:10C940001470FDE62E48FCF7F7FA2B689B047FF580
:10C9500041AF2C48FCF7F0FA4020FCF7EDFA39E73C
:10C960002948FCF7E9FA2B682EE72848FCF7E4FA97
:10C970002B6826E79A8AB2F57A7FBFF416AF4FF498
:10C980007A729A8211E743F001032B6016E700BF29
:10C99000DC05000890010008D849002060F2030877
:10C9A000C4F803080598002012980020886500202C
:10C9B000E45F0020846500208867002088610020F3
:10C9C00009600002C871002060200020D44C0020C3
:10C9D000D71C002094200020802D0020829500206C
:10C9E000A8200020442F002040250020C0C9FB487B
:10C9F000C825002017B7D13844250020EC27002097
:10CA000001600002094000020920000208600002E3
:10CA1000024000080080000808B51DF007FAFCF786
:10CA2000C9FA1DF0EBF9FFF757FE0120BDE80840F9
:10CA30002DF000BC38B50C4C0C4DAC4206D26168F0
:10CA400020461434FCF742FAAC42F8D3084A094BAA
:10CA5000094C1460002209491A705A70084808608D
:10CA6000BDE8384016F09AB890010008DC050008CF
:10CA70008465002005980020E45F00208865002080
:10CA80001298002008B5FFF7D5FF1DF0CFF9FCF78D
:10CA900091FABDE808401DF0B1B900BFF0B50C290E
:10CAA00034D8DFE801F0893333335E333333343342
:10CAB00033330700048C9689B2F802E01788734D6F
:10CAC00024F480542404240C0484038C8488818BF3
:10CAD00023F4005321F4E6411B0409041B0C46EA2D
:10CAE0000E06090C43EA063341EA0721A8429BB22D
:10CAF000A4B289B200F09E8005F58065A84200F0DE
:10CB0000998092688480818302640384F0BD048CE0
:10CB10009589B2F802C0B2F800E05C4F24F480744A
:10CB20002404240C0484038C8688818B23F40073F2
:10CB30001B0421F073011B0C45EA0C04090443EAB1
:10CB40000423090CB8429BB2B6B241EA0E015CD094
:10CB50004F4CA04259D0926886808183C26303847F
:10CB6000F0BD048C9589B2F802C0B2F800E0474EDF
:10CB700024F010042404240C0484038C8788018B83
:10CB800023F0200321F4E6411B0409041B0C45EAB1
:10CB90000C04090C43EA041341EA0E21B0429BB293
:10CBA000BFB289B25DD03A4CA0425AD09268878019
:10CBB000018382630384F0BD048C9789B2F802E09C
:10CBC0001688324D24F001042404240C0484038CC0
:10CBD0008488018B23F002031B0421F073011B0CDA
:10CBE00047EA0E0709043B43090CA8429BB2A4B2D2
:10CBF00041EA060125D005F58065A84221D092685A
:10CC00008480018342630384F0BDD589148A578AE6
:10CC100023F4006343EA05254FF6FF332B40958844
:10CC200026F440563C4343EA052346EA04169BB2E9
:10CC3000B6B290E7158A24F4804444EA8514A4B27D
:10CC40005FE7D689158A578A23F00803334324F413
:10CC5000407496883D4323F004032C433343A4B22D
:10CC6000CDE7D489158A568A23F0800343EA04135A
:10CC70004FF6BF741C40938827F44067354344EA5D
:10CC8000031347EA85079BB2BFB28FE7000001405C
:10CC9000000401402DE9F84F782200219148924C80
:10CCA000DFF86892914D924E924FDFF8648230F037
:10CCB000ECF891489149DFF85CE2DFF85CC20022B1
:10CCC0001359834200F0E980B3F1804F00F0E78010
:10CCD000AB4200F0F280B34200F0F180BB4200F0C2
:10CCE000F080734500F0EF80634500F0EE8043452F
:10CCF00000F0ED80DFF824A2534500F0EA800AF549
:10CD0000806A534500F0E7800AF5806A534500F0D9
:10CD1000E480AAF5983A534500F0E1800AF5806A6C
:10CD2000534500F097800AF5806A534508BF0D23EC
:10CD300000F091801832B2F5A87FC1D16A4EDFF8B9
:10CD4000E0A106F5A8774FF003094FF0020803E0D1
:10CD50001836B74200F09F80B379002BF8D03379B2
:10CD60001C09013C032C03F00F03F1D8644A32F88C
:10CD7000140040FA03F2D207EAD5012505FA03F3BD
:10CD8000013B18402EF042FD5E4B1B5D18441AEB30
:10CD9000C002DDD05AF830305B4C317A03F13F40AD
:10CDA00000F57E00800A205C00F01F044009032883
:10CDB00005FA04F57BD0042873D0022804D14F482B
:10CDC000406C05434D484564B2F804E0BEFA8EF26B
:10CDD000C2F11F0292B2D00803EB800002F00702FA
:10CDE000046A92000F25954024EA05040462046A4F
:10CDF00001FA02F22243002502624FF0010C2A469A
:10CE000003E0102A05F10205A2D00CFA02F030EA84
:10CE10000E0102F10102F4D11C6809FA05F1C943BF
:10CE20000C401C60D3F800B008FA05F444EA0B0487
:10CE30001C609C680C409C609C689C605C6824EA58
:10CE40000000586058685860D8680140D960D968B7
:10CE5000D960D6E70C2309EBC3034FF0010A1B7915
:10CE600003F01F0B5B09032B0AFA0BFA09D0042B02
:10CE70000CD0022B7FF45EAF4B6C4AEA03034B6489
:10CE800058E70B6C4AEA03030B6453E70B6B4AEA5F
:10CE900003030B634EE7BDE8F88F0023DBE70123B4
:10CEA000D9E71648006B0543144805638CE713481F
:10CEB000006C05431148056486E70223CBE7032392
:10CEC000C9E70423C7E70523C5E70623C3E707230C
:10CED000C1E70823BFE70923BDE70A23BBE70B230C
:10CEE000B9E700BFEC2500209CEE030800040040D9
:10CEF00000080040000C00400000014000380240E3
:10CF0000F0EF0308ECEF030848F1030850F10308C1
:10CF100000040140001000400014004000400140A7
:10CF2000105E002000286AD003682DE9F04F03F15D
:10CF30003F4404F57E045F4EA40A0125345D04F0ED
:10CF40001F066409032C05FA06F559D0042C00F0DD
:10CF5000AC80022C59D08588B5FA85F0C0F11F004D
:10CF600080B2C40803EB840400F00700266A800046
:10CF70000F27874026EA07062662276A01F0030684
:10CF80008240701E3A430128C1F3810CC1F300189E
:10CF90002262C1F341113DD90024224601274FF0FE
:10CFA000030E03E0102A04F1020426D007FA02F06F
:10CFB000A84302F10102F5D1D3F800C00EFA04F043
:10CFC000C04300EA0C0CC3F800C0D3F8008006FA96
:10CFD00004FC4CEA080CC3F800C0D3F80CC000EA0B
:10CFE0000C00D860D3F80CC001FA04F040EA0C0041
:10CFF000102AD86004F10204D8D1BDE8F08F704740
:10D000002D4C266C35432564A5E72B4C666C3543C7
:10D010006564A0E7002002464FF0010E4FF00309BF
:10D0200004E00132102A00F102003CD00EFA02F7AF
:10D0300037EA0504F5D1D3F800A009FA00F4E44377
:10D040000AEA040AC3F800A0D3F800B006FA00FA0E
:10D050004AEA0B0AC3F800A0D3F808A004EA0A0AB7
:10D06000C3F808A0D3F808B00CFA00FA4AEA0B0A91
:10D07000C3F808A0D3F804A02AEA07075F60D3F832
:10D0800004A008FA02F747EA0A075F60DF683C403D
:10D09000DC60DF6801FA00F401323C43102ADC60F6
:10D0A00000F10200C2D1BDE8F08F034C266B35437E
:10D0B000256350E748F103080038024003682DE972
:10D0C000F04F03F13F4404F57E04604EA40A0125AD
:10D0D000345D04F01F066409032C05FA06F500F020
:10D0E000AF80042C00F0A780022C54D08588B5FABC
:10D0F00085F0C0F11F0080B2C40803EB840400F087
:10D100000700266A80000F27874026EA0706266266
:10D11000276A01F0030602FA00F0721E3843012A62
:10D12000C1F3810CC1F300182062C1F3411137D95A
:10D130000024224601274FF0030E03E0102A04F1D9
:10D14000020426D007FA02F0A84302F10102F5D149
:10D15000D3F800C00EFA04F0C04300EA0C0CC3F888
:10D1600000C0D3F8008006FA04FC4CEA080CC3F8AF
:10D1700000C0D3F80CC000EA0C00D860D3F80CC093
:10D1800001FA04F040EA0C00102AD86004F102040D
:10D19000D8D1BDE8F08F2E4C666C35436564A5E7A9
:10D1A000002002464FF0010E4FF0030904E0013267
:10D1B000102A00F102003CD00EFA02F737EA05040B
:10D1C000F5D1D3F800A009FA00F4E4430AEA040A0E
:10D1D000C3F800A0D3F800B006FA00FA4AEA0B0A36
:10D1E000C3F800A0D3F808A004EA0A0AC3F808A00C
:10D1F000D3F808B00CFA00FA4AEA0B0AC3F808A000
:10D20000D3F804A02AEA07075F60D3F804A008FA5D
:10D2100002F747EA0A075F60DF683C40DC60DF68CE
:10D2200001FA00F401323C43102ADC6000F10200F4
:10D23000C2D1BDE8F08F064C266B3543256355E718
:10D24000034C266C3543256450E700BF48F10308C2
:10D250000038024010B50409013C032C17D80D4BCF
:10D2600033F8142000F00F0042FA00F313F001032A
:10D270000DD0012303FA00F0013810402EF0C6FA59
:10D28000054A064B125D104403EBC00010BD0020A0
:10D2900010BD00BFF0EF0308ECEF0308105E0020A4
:10D2A00001490248FEF714BF3C2600200020004040
:10D2B00001490248FEF70CBF14260020000400407C
:10D2C00002494FF08040FEF703BF00BFEC2500206D
:10D2D000F0B50668B30AA3F58013082B50D8384C74
:10D2E000E55C022D4CD84379A8009F08002952D054
:10D2F0009C080223B6F80CE0A340441907EB44074E
:10D3000043EA0E032F4C07F1040E9BB244F827109A
:10D3100044F82E20B381EFF31181502383F3128858
:10D320004219D200A7183B695BB33B620433421930
:10D3300004EBC202576917B11F60536904334219E5
:10D3400004EBC202976917B11F6093690433421955
:10D3500004EBC202D76917B11F60D36904330022FE
:10D36000C9B21A6081F31188284404EBC004236A0F
:10D370005BB9B38923F001031B041B0CB381F0BD1F
:10D38000F0BD02F120032344D1E7B3899BB243F0FF
:10D390000103B381F0BDB3890A4C4FF0020E0EFABF
:10D3A00007FE9BB223EA0E0300EB050E07EB4E07C8
:10D3B000B3813B1D44F8271044F82320ABE700BF9E
:10D3C00010D40308EC2500202B4B98423CD0B0F140
:10D3D000804F3BD0A3F57C43984239D003F580635E
:10D3E000984237D003F58063984235D003F58063C7
:10D3F000984233D003F58063984231D003F57043EF
:10D4000098422FD003F5705398422DD003F58063D6
:10D4100098422BD003F58063984229D0A3F5983326
:10D42000984227D003F58063984207D003F58063C4
:10D43000984208BF0D2202D0002070470C220F4BEB
:10D4400003EBC203187970470022F8E70122F6E7E0
:10D450000222F4E70322F2E70422F0E70522EEE7D6
:10D460000622ECE70722EAE70822E8E70922E6E7D6
:10D470000A22E4E70B22E2E70000014050F1030832
:10D480002DE9F04F013085B0C3B203930B460291F2
:10D490008B4C8C4E002B00F09A8032208A4D8B4FA3
:10D4A000DFF82C921FF06AF94FF4FA7A4FF0100C63
:10D4B0004FF47A70D9F80430C3F30803002B40F01E
:10D4C000DE80EFF31183002B40F0D9802968A26839
:10D4D00000BF2B689942F9D1D7F800E000FB0EF3AA
:10D4E0009B1AB3FBFEF300FB01314FF0010E0191DB
:10D4F000D9F80430C3F30803002B40F08780EFF322
:10D500001183002B40F082802B68A16800BF2A683D
:10D510009342F9D1D7F800B000FB0BF2521AB2FBDC
:10D52000FBF200FB0323019A9B1AB3F57A7FDFD34A
:10D53000BAF1010ABED1039B002B40F0BD804FF42D
:10D540007A7ADFF88C9150464FF0100CD9F80430FD
:10D55000C3F30803002B75D1EFF31183002B71D1B6
:10D560002968A26800BF2B689942F9D1D7F800E07A
:10D5700000FB0EF39B1AB3FBFEF300FB01314FF0EF
:10D58000010E0191D9F80430C3F3080313BBEFF384
:10D590001183FBB92B68A16800BF2A689342F9D1B7
:10D5A000D7F800B000FB0BF2521AB2FBFBF200FB03
:10D5B0000323019A9B1AB3F57A7FE3D3BAF1010AE8
:10D5C000C4D1029B013B0293002B7FF466AF05B0F0
:10D5D000BDE8F08FEFF311888CF31288A1682368FF
:10D5E000DB0344BFC6F800E0A1682B6832685FFA2D
:10D5F00088F888F31188D7F800801A4400FB08F3F4
:10D600005B1AB3FBF8F300FB0233D2E7EFF31188A8
:10D610008CF31288A1682368DB0344BFC6F800E0DE
:10D62000A1682B6832685FFA88F888F31188D7F808
:10D6300000801A4400FB08F35B1AB3FBF8F300FB0D
:10D64000023370E7EFF311828CF31288D4F808E00C
:10D650002368D90303D501233360D4F808E02B688D
:10D660003168D2B282F311883A68194400FB02F3A0
:10D67000A3EB0E03B3FBF2F300FB01317FE7EFF303
:10D6800011828CF31288D4F808E02368D90303D5FB
:10D6900001233360D4F808E02B683168D2B282F3FA
:10D6A00011883A68194400FB02F3A3EB0E03B3FBA5
:10D6B000F2F300FB013118E718461EF0E7FE3EE7E3
:10D6C00010E000E0D05D0020D45D0020D85D002097
:10D6D00000ED00E0204B5B68C3F3080330B4BBB936
:10D6E000EFF31183A3B91D4B1D4C1868A16800BF4F
:10D6F0001A689042F9D11B4B1C684FF47A7202FBF6
:10D7000004F3591AB1FBF4F130BC02FB001070476E
:10D71000EFF31182102383F3128811498C680B6890
:10D7200013F4803F104B02D0012018608C680B4925
:10D73000D2B20D68186882F311880A4B19684FF449
:10D740007A72284402FB01F31B1B30BCB3FBF1F3DC
:10D7500002FB0030704700BF00ED00E0D45D002008
:10D7600010E000E0D85D0020D05D00202DE9F84FEA
:10D770008046FFF7AFFF254E2549DFF8A0E0254A98
:10D78000254D844610274FF47A740120DEF80430CA
:10D79000C3F30803D3B9EFF31183BBB90B68D2F815
:10D7A00008A000BFD1F800904B45F7D1D6F800B0E3
:10D7B00004FB0BF9A9EB0A09B9FBFBF904FB039382
:10D7C000A3EB0C034345E1D3BDE8F88FEFF3118AD7
:10D7D00087F31288D2F808B01368DB0344BF2860CF
:10D7E000D2F808B00B68D5F800905FFA8AFA8AF38D
:10D7F0001188D6F800A0994404FB0AF3A3EB0B03AD
:10D80000B3FBFAF304FB0933DAE700BFD85D00206D
:10D81000D45D002010E000E0D05D002000ED00E0CD
:10D820002DE9F04FDFF830C1474A4849484E494D8D
:10D830008046102718F1FF38C0F08480DCF80430EF
:10D84000C3F30803002B5CD1EFF31183002B58D1F5
:10D850000B68946800BF08688342F9D1D6F800903D
:10D860004FF47A7000FB09FEAEEB040EBEFBF9FE2E
:10D8700000FB03EEDCF80430C3F308034FF47A74C2
:10D880000120FBB9EFF31183E3B90B68D2F808A0CC
:10D8900000BFD1F800904B45F7D1D6F800B004FB9B
:10D8A0000BF9A9EB0A09B9FBFBF904FB0393A3EB02
:10D8B0000E03B3F57A7FBDD2DCF80430C3F308035E
:10D8C000002BDFD0EFF3118A87F31288D2F808B06B
:10D8D0001368DB0344BF2860D2F808B00B68D5F8A2
:10D8E00000905FFA8AFA8AF31188D6F800A099446A
:10D8F00004FB0AF3A3EB0B03B3FBFAF304FB0933BA
:10D90000D5E7EFF3118487F31288D2F808901368F3
:10D91000D80303D501232B60D2F808900B68286840
:10D92000E4B284F31188D6F800A04FF47A7400EBC7
:10D93000030E04FB0AF3A3EB0903B3FBFAF304FBA6
:10D940000E3E97E7BDE8F08F10E000E0D45D0020C8
:10D95000D85D0020D05D002000ED00E030B4EFF392
:10D960001183102282F312880649074C0A6807487F
:10D97000013200250A602560DBB2026883F311885A
:10D9800030BC7047D45D0020D05D002010E000E086
:10D9900038B5264B5C69636B73B1A36DA26BD2B1D2
:10D9A000998A1A88C90592B201D5D20700D438BD28
:10D9B0004FF6F7721A8038BDA36D99891A888906C7
:10D9C00092B2EBD59206E9D5E26AD2B19888216B82
:10D9D00080B29047E1E799891A880D0692B2DFD5A7
:10D9E0001006DDD5A26A616A8A4219D0A16925694B
:10D9F000885C98800132B2FBF5F105FB1122A2622E
:10DA0000CEE79B88E2696169DBB28B54E269E0682A
:10DA1000A36D0132B2FBF0F100FB1122E261BDE720
:10DA2000DA6822F08002DA60BAE700BFBC5C00204E
:10DA300038B5264B9C68636B73B1A36DA26BD2B1F2
:10DA4000998A1A88C90592B201D5D20700D438BD87
:10DA50004FF6F7721A8038BDA36D99891A88890626
:10DA600092B2EBD59206E9D5E26AD2B19888216BE1
:10DA700080B29047E1E799891A880D0692B2DFD506
:10DA80001006DDD5A26A616A8A4219D0A1692569AA
:10DA9000885C98800132B2FBF5F105FB1122A2628D
:10DAA000CEE79B88E2696169DBB28B54E269E0688A
:10DAB000A36D0132B2FBF0F100FB1122E261BDE780
:10DAC000DA6822F08002DA60BAE700BFBC5C0020AE
:10DAD00038B5264B1C68636B73B1A36DA26BD2B1D2
:10DAE000998A1A88C90592B201D5D20700D438BDE7
:10DAF0004FF6F7721A8038BDA36D99891A88890686
:10DB000092B2EBD59206E9D5E26AD2B19888216B40
:10DB100080B29047E1E799891A880D0692B2DFD565
:10DB20001006DDD5A26A616A8A4219D0A169256909
:10DB3000885C98800132B2FBF5F105FB1122A262EC
:10DB4000CEE79B88E2696169DBB28B54E269E068E9
:10DB5000A36D0132B2FBF0F100FB1122E261BDE7DF
:10DB6000DA6822F08002DA60BAE700BFBC5C00200D
:10DB700070B4EFF31186502383F31288836B1A6815
:10DB8000D20720D45D686DB9446A826A944217D086
:10DB900081691144D9600ED9A21A5A6084620022A8
:10DBA00080F85C201A6842F00102F1B21A6081F339
:10DBB000118870BC704701698A1A5A608562EEE765
:10DBC000012380F85C30F3B283F3118870BC704796
:10DBD00003685B6A03B11847704700BF03681B6A9C
:10DBE00003B11847704700BF03682DE9F041DF69B2
:10DBF0001FB13B46BDE8F0411847002A164611DD2B
:10DC000004460D460E4400E023689B682046984772
:10DC10000028F9D0236815F8011B1B682046984797
:10DC2000AE42F1D1BDE8F08103689B69184700BF9F
:10DC300003685B69184700BF03681B69184700BF8A
:10DC40000368DB68184700BF03689B68184700BF7C
:10DC500003685B68184700BF03681B68184700BF6C
:10DC600038B50C46097849B1054601342B68284679
:10DC70001B68984714F8011B0029F7D138BD00BF75
:10DC8000064B53F820302BB11A689B8851690B4220
:10DC900001D1138370475383704700BFE05D0020BC
:10DCA000026802F13F4303F57E032DE9F04F9B0A22
:10DCB000544DEB5C03F01F055B090124032B04FAB0
:10DCC00005F400F09980042B00F09180022B3ED0E7
:10DCD00001F00306731E012BC1F3810CC1F3001880
:10DCE0008588C1F3411137D90024234601274FF01D
:10DCF000030E03E0102B04F1020426D007FA03F010
:10DD0000A84303F10103F5D1D2F800C00EFA04F0E4
:10DD1000C04300EA0C0CC2F800C0D2F8008006FA3A
:10DD200004FC4CEA080CC2F800C0D2F80CC000EAAF
:10DD30000C00D060D2F80CC001FA04F040EA0C00EC
:10DD4000102BD06004F10204D8D1BDE8F08F2E4B27
:10DD50005D6C2C435C64BBE7002003464FF0010E72
:10DD60004FF0030904E00133102B00F102003CD016
:10DD70000EFA03F737EA0504F5D1D2F800A009FA44
:10DD800000F4E4430AEA040AC2F800A0D2F800B0A2
:10DD900006FA00FA4AEA0B0AC2F800A0D2F808A074
:10DDA00004EA0A0AC2F808A0D2F808B00CFA00FA8D
:10DDB0004AEA0B0AC2F808A0D2F804A02AEA070728
:10DDC0005760D2F804A008FA03F747EA0A07576039
:10DDD000D7683C40D460D76801FA00F401333C4373
:10DDE000102BD46000F10200C2D1BDE8F08F064BC9
:10DDF0001D6B2C431C636BE7034B1D6C2C431C6495
:10DE000066E700BF48F10308003802402DE9F04FF3
:10DE10004A484B494B4B4C4C4FF0010A4FF002091A
:10DE20004FF004084FF0080C4FF0100E202740264A
:10DE3000802530F8022B12F0010F03D01960A3F8EF
:10DE400004A0083312F0020F03D01960A3F8049065
:10DE5000083312F0040F03D01960A3F804800833CC
:10DE600012F0080F03D01960A3F804C0083312F0B1
:10DE7000100F03D01960A3F804E0083312F0200F4C
:10DE800002D019609F80083312F0400F02D0196051
:10DE90009E80083312F0800F02D019609D800833F5
:10DEA00012F4807F05D04FF4807B1960A3F804B092
:10DEB000083312F4007F05D04FF4007B1960A3F8FB
:10DEC00004B0083312F4806F05D04FF4806B1960F2
:10DED000A3F804B0083312F4006F05D04FF4006BC0
:10DEE0001960A3F804B0083312F4805F05D04FF432
:10DEF000805B1960A3F804B0083312F4005F05D00A
:10DF00004FF4005B1960A3F804B0083312F4804F9B
:10DF100005D04FF4804B1960A3F804B00833D20B3E
:10DF200004D04FF4004219609A80083301F58061F3
:10DF3000A1427FF47EAFBDE8F08F00BFF0EF030891
:10DF400000000240105E002000100240002855D062
:10DF5000026802F13F4303F57E032DE9F04F9B0A6F
:10DF6000544DEB5C03F01F055B090124032B04FAFD
:10DF700005F444D0042B00F09780022B44D001F02C
:10DF80000306731E012BC1F3810CC1F300188588B1
:10DF9000C1F341113DD90024234601274FF0030E60
:10DFA00003E0102B04F1020426D007FA03F0A84383
:10DFB00003F10103F5D1D2F800C00EFA04F0C0431A
:10DFC00000EA0C0CC2F800C0D2F8008006FA04FC8B
:10DFD0004CEA080CC2F800C0D2F80CC000EA0C00F1
:10DFE000D060D2F80CC001FA04F040EA0C00102B0B
:10DFF000D06004F10204D8D1BDE8F08F70472E4BF9
:10E000001D6C2C431C64BAE72B4B5D6C2C435C6489
:10E01000B5E7002003464FF0010E4FF0030904E07E
:10E020000133102B00F102003CD00EFA03F737EA5F
:10E030000504F5D1D2F800A009FA00F4E4430AEA95
:10E04000040AC2F800A0D2F800B006FA00FA4AEAC0
:10E050000B0AC2F800A0D2F808A004EA0A0AC2F823
:10E0600008A0D2F808B00CFA00FA4AEA0B0AC2F883
:10E0700008A0D2F804A02AEA07075760D2F804A043
:10E0800008FA03F747EA0A075760D7683C40D460AC
:10E09000D76801FA00F401333C43102BD46000F13F
:10E0A0000200C2D1BDE8F08F034B1D6B2C431C63F3
:10E0B00065E700BF48F103080038024010B103686B
:10E0C00082885A83704700BF10B1036882881A8320
:10E0D000704700BF18B10368828809B95A83704736
:10E0E0001A8370470E4B1B8801463BB90D4B0E4AF5
:10E0F0001B7810680BB981F00101EBE70B4B5A69F3
:10E100001AB118B91A68106058747047084A18682C
:10E110001188084A92FBF1F201210260597470479C
:10E12000EC5D0020EE5D0020F05D0020F45D00203D
:10E130000C5E002020A1070010B40A4B0A4A1C788C
:10E1400001238340234052F8200029B9B3FA83F118
:10E1500049095DF8044BBDE7191C18BF01215DF8A2
:10E16000044BB7E7DC5D0020E05D002008B501212D
:10E170000220FFF7E1FF094B1B7803F00503052B95
:10E1800008D000210120FFF7D7FF00210846FFF744
:10E19000D3FFFEE712F0FCFDF3E700BFB85C002000
:10E1A00030B1036882881B691A4214BF0120002025
:10E1B000704700BF2DE9F0410B4E346873691C4075
:10E1C0000FD0DFF828800127B4FA84F3C3F11F03CE
:10E1D00007FA03F558F8230003689847AC437561C4
:10E1E000F2D1BDE8F08100BF003C01402C1F0020AF
:10E1F0002DE9F0410B4E346873691C400FD0DFF8F5
:10E2000028800127B4FA84F3C3F11F0307FA03F54A
:10E2100058F8230003689847AC437561F2D1BDE814
:10E22000F08100BF003C01402C1F00202DE9F0418F
:10E230000B4E346873691C400FD0DFF8288001272B
:10E24000B4FA84F3C3F11F0307FA03F558F8230067
:10E2500003689847AC437561F2D1BDE8F08100BF17
:10E26000003C01402C1F00202DE9F0410B4E34688A
:10E2700073691C400FD0DFF828800127B4FA84F3BB
:10E28000C3F11F0307FA03F558F823000368984702
:10E29000AC437561F2D1BDE8F08100BF003C0140A4
:10E2A0002C1F00202DE9F0410B4E346873691C408F
:10E2B0000FD0DFF828800127B4FA84F3C3F11F03DD
:10E2C00007FA03F558F8230003689847AC437561D3
:10E2D000F2D1BDE8F08100BF003C01402C1F0020BE
:10E2E0002DE9F0410B4E346873691C400FD0DFF804
:10E2F00028800127B4FA84F3C3F11F0307FA03F55A
:10E3000058F8230003689847AC437561F2D1BDE823
:10E31000F08100BF003C01402C1F00202DE9F0419E
:10E320000B4E346873691C400FD0DFF8288001273A
:10E33000B4FA84F3C3F11F0307FA03F558F8230076
:10E3400003689847AC437561F2D1BDE8F08100BF26
:10E35000003C01402C1F0020084A536C10B5084CAB
:10E3600043F4804353642046402200212EF08DFD6B
:10E370004FF0FF332364C4F8433010BD003802402F
:10E380002C1F00202DE9F041044618460D46164684
:10E3900098462CF041FD2768E6722844A072294671
:10E3A0007D69434632462046AC46BDE8F0416047B1
:10E3B000036810B504461B689847236820469B688D
:10E3C0009847A37B0133A37310BD00BF2DE9F04133
:10E3D0000578012D02D00020BDE8F08190F904E01D
:10E3E000BEF1FF3FF7D0BEF1030FF4DC4FEACE08D9
:10E3F000DFF898C008EB0E060CEB86067768002F56
:10E40000E9D04079326240000024C0B2B075F175A5
:10E410007476B576337675753475BB88F261990577
:10E4200014D43B88DA050CD44FF4805401E0013C4D
:10E430001FD03B889B05FAD43B889BB243F4807382
:10E440003B80BB889BB243F44073BB80F0440CEB31
:10E4500088024FF4805401E0013C0AD0537D002B28
:10E46000FAD10CEB880898F8144084F00100BDE85C
:10E47000F081054A1388013370469BB21380FCF784
:10E4800039FA2046BDE8F081903F0020DC5C002096
:10E490002DE9F04FBB4B1E788BB0002E40F08180F1
:10E4A000B94BBA4C1D78BA4FDFF808B305F0010537
:10E4B000A4F10A0954F80A0CB8B14FF0CC0808FBD3
:10E4C0000698FFF7C5FB80B154F80A0CFFF7B8FBBC
:10E4D00014F8023C024683B924283BD075B354F8A3
:10E4E0000A0CFFF7B5FB0028EED10136032E04F12C
:10E4F000CC04DFD10BB0BDE8F08F012B2ED0022B66
:10E5000033D0032B40D0042B00F06781052B00F0A3
:10E510005581062BE3D114F801ECBEF1000F00F099
:10E52000D881BEF1010F00F01B8201360023032EBB
:10E5300004F8023C04F1CC04BCD1DBE7232A54F8F4
:10E540000A0C00F08081934B93F822309342B8D1AB
:10E55000FBF772FE012304F8023CC0E74D2800F0EF
:10E560006581002304F8023CB9E700233C2804F845
:10E57000023C00F055813E28B1D10122032304F86A
:10E58000012C04F8023CAAE7C028EAD800210423A1
:10E5900004F8050C04F8040C04F8061C04F8023C0A
:10E5A0009DE77D4B18680028A4D0FAF7EFFBDFF851
:10E5B00008A27A4DDFF8F491DAF80000FFF748FB83
:10E5C000002897D0DAF80000FFF73AFB09281BD0A3
:10E5D0003F2819D02B68002B66D1042800F0BA819F
:10E5E0000C2800F0C8807F28E6D0A0F12002D2B22B
:10E5F0005E2AE1D80BB92028DED05A1C09F80300A6
:10E600002A6029F0DBF8D7E72C68002C59D1644B3D
:10E61000264603F51478002E08BF1E4610334345E6
:10E62000F9D1002E00F04F81A3F1100B3068DBF818
:10E630000020075D135D9F42204402EB040140F07F
:10E640004081671E4F4422460BB9FD2A5BD907F86B
:10E65000013F01322A6010F8013F11F801EF9E4599
:10E66000F2D00AB1B34512D04E4829F0AFF8B34505
:10E6700008D356F8100B29F0A9F8092029F09EF8C4
:10E680005E45F6D9484829F0A1F82A68002494424A
:10E6900092D2661E4E4416F8010F29F08FF82B68AF
:10E6A00001349C42F7D387E70C2864D00A2833D082
:10E6B0000D2831D07F2800F0BD80FF2B3FF67CAFC6
:10E6C00093E7374F4FF0000B07F514785E4602E0F2
:10E6D000103747450DD0224639684846FAF7B2FE52
:10E6E0000028F5D1BB46002EF2D13E4610374745F3
:10E6F000F1D1002E9AD1BBF1000F3FF45DAF294854
:10E7000029F064F8B5E7511C202009F802002960BF
:10E7100009F801300A46A5E729F0D9F82321234852
:10E720002EF0CAFB002800F01381A0EB090028603E
:10E7300090B1431E19F80310202940F02E8109EBF7
:10E74000030243B112F8011D202903F1FF304FD11C
:10E750000346002BF6D12B604FF48072002148460F
:10E760002EF093FB074B1B78002B3FF4C3AE0E48F3
:10E7700029F02CF820E70E4829F028F80A4829F05B
:10E7800025F819E7D9420020644A0020828E002033
:10E790002C1F0020C87100208C420020A0270020E0
:10E7A0009CD60308C8000408D0000408A026002056
:10E7B000D800040864D003089C26002014F8063C06
:10E7C00014F8051C994270D814F8043C83427FF475
:10E7D000C8AE062304F8023C9DE614F8043C04F895
:10E7E000030C5A40052304F8042C04F8023C76E696
:10E7F0002B606B4C002204F5147809F8032002E02A
:10E80000103444454DD02168484610F011FA0028D4
:10E81000F6D0444545D2E368984700232B609BE738
:10E82000032204F8013C04F8022C58E6022304F801
:10E83000023C54E6013B00225A482B6009F80320B1
:10E8400028F0C4FFB8E6584B5849DB78584ADFF83F
:10E850008CE11060003318BF01230B70554B564AF2
:10E86000CEF80030554BFA644FF0400E012187F886
:10E8700054E0B864386587F855505148197029F04C
:10E8800055FA504828F0A2FF4FF400600DF094FCB8
:10E890004D4B93F82230232B3FF45AAE14F8023C30
:10E8A00037E64A4828F092FFB7E714F8041C08EB53
:10E8B00003005140013304F8041C04F8063C827242
:10E8C0000DE62246CDE64248A3F1100B28F07EFF6C
:10E8D000CFE69BE80F000DF1280C0DF1080888E841
:10E8E0000F004CF824ED14F8053C14F803AC069422
:10E8F000624623444FF0010C414606A8ADF822E0E1
:10E900000793ADF820A08DF824C00AF0A7FE40B10F
:10E91000029A304B03924146A4F10A0002931CF084
:10E92000F1FEDDF80480002304F8023CB8F1000F8A
:10E930003FF4DBAD54F80A0C1CF0A4FF013654F888
:10E940000A0CC047032E04F1CC047FF4B3ADD1E52B
:10E950002868EDE620480FF0A7FC0BB0BDE8F08F6B
:10E9600014F8053C14F8032C0694234407936E2AEC
:10E970004FF0000308930993ADF820207FF4D5AD44
:10E9800006A8FAF7E1FD06A8FAF7D2FD06A8FAF7FD
:10E99000CFFD06A8FAF7CCFDC7E5034629E700BF7F
:10E9A0009CD603080001040805980020704F002041
:10E9B0009C260020781F002061C00008D94200205A
:10E9C00004010408D0000408C8710020E400040811
:10E9D000C80004080C990020A02600208C420020CA
:10E9E0002DE9F04F2DED068BA04BA14A1C7897B076
:10E9F00000F59C41203181460B911160002C00F004
:10EA000007879C4A1268904240F285809A4A069293
:10EA100016689A499A4A0591013C1C70994B0492D8
:10EA200006F480560893002E40F08380964B1B78A6
:10EA3000022B01F0AC81042B01F09B81012B01F032
:10EA40004F81924B9945089B9B7800F2B085002B33
:10EA500040F0B1858E4B0793069B1E6816F48057D5
:10EA600040F0A486DFF85892049BB3F90610059B8A
:10EA70005D8BA942B4BF00250125DFF83C82D8F8A0
:10EA8000003013F080535ED0079A127812F0010222
:10EA90005FD00598408C884241F31983002D5ED1E8
:10EAA0007C4C94F88C10002959D17B487B49006834
:10EAB00090F82D0000240C604C608C607849002890
:10EAC0004ED10870002A4FD0F1064DD5754A127804
:10EAD000D20649D4002F47D1002B45D1740243D42C
:10EAE000714B1B78002B02F0BC83704B9B78002D80
:10EAF00042F038843BB16E4A6E4B12681B689B1A19
:10EB0000002BC2F207841020624C2BF06DFA012317
:10EB100084F88D3028E0584B06931E68584B574AAE
:10EB2000049306F48056574B05920893002E3FF449
:10EB30007DAF00216048FBF72BFA00287FF476AF09
:10EB40000DF0BCFE72E770029ED4079A127802F0B4
:10EB50000102504C002184F88C10002DA5D05049A2
:10EB600001200870002AAFD1544B1A78002A40F0D7
:10EB7000C3800599049C488BB4F90070898BB4F963
:10EB80000240B842B4BF8026002646F04003B94296
:10EB9000D8BF33469B0843F08006A042B8BF334637
:10EBA000049F43F04006A142C8BF33469B08B7F913
:10EBB0000440B7F9066043F08007A042B8BF3B4667
:10EBC00043F04007A142C8BF3B469B0843F0800783
:10EBD000304C8642C8BF3B4643F0400794F88EE075
:10EBE0008E42B8BF3B469E4501F02585A4F8902093
:10EBF00084F892202C4984F88E300E78002E01F093
:10EC0000E3835F2B01F072846F2B01F08C84079BF0
:10EC10001B78DB0770D494F8921000296CD1B4F9FA
:10EC20009030322B68DD94F88E200120572A84F82A
:10EC3000920002F06880069B1B685D0741F13083FB
:10EC40005A2A41F02D8394F89430002B42F0BD8273
:10EC500094F8963083F0010384F89630002B42F04C
:10EC60004E830C202BF0C0F901F053BC6C4C0020FB
:10EC7000284C0020684C0020C07A00209C710020A5
:10EC800080910020442F002026490020404B4C005A
:10EC9000644A0020C41F00208465002088490020A9
:10ECA0001025002082650020D71C00209C950020A4
:10ECB000D45D0020642600203095002013450020FC
:10ECC000244D002092490F68450037B12E1803EB00
:10ECD00086067F787678BE4208D205448D4E8E48EF
:10ECE00003EB850300250B6035800560FA3A0023AD
:10ECF000A4F8902084F89230069B1B68874A884EBF
:10ED00000992590700F1D886864B0C930DF1500BF0
:10ED10001D460023CBF804300A96149340F6330ABC
:10ED2000192740F28334049E02E004354D4520D07B
:10ED3000A978EB78994217FB0140F6D26978043143
:10ED400017FB034336F911105145A8BF5146B1F5E1
:10ED5000617FB8BF4FF461718142E6DD9942E4DC26
:10ED600029782729E1D858460435FBF701F94D45A4
:10ED7000DED16D4B0A9E1B789BE8030088E80300F8
:10ED8000002B40F07286694B1B78002B00F0F28557
:10ED900001216748FBF7FCF8002840F0F482089B4B
:10EDA000DB78002B40F0EF82DFF8A09133881CB2B3
:10EDB00024F00104A7B2BB42378001F017805D4CFC
:10EDC0004FF002080E204FF0140B4FF0FF0A84F8AA
:10EDD000008084F801B084F802A02BF005F94146C8
:10EDE00053483788FBF7D4F8002841F04F8327F0C9
:10EDF00002039BB2BB4233800AD04E4B0220142147
:10EE0000FF2218700E2059709A702BF0EDF8378899
:10EE1000494B4A4A197850680A93BC0708BF81F0E9
:10EE20000201C1F340010B92FFF754F9242140483D
:10EE3000FBF7AEF830B9079A1378590744BF23F0AF
:10EE400004031370D9F8002012F00A0F1DD0052119
:10EE50003748FBF79DF8002801F00F8134886207DE
:10EE600041F1C78232480621FBF792F8002801F0F1
:10EE7000F180630641F1B58207212D48FBF788F840
:10EE8000002841F00D80D9F80020970600F1448554
:10EE9000B6F800802A4F26480C21FBF779F80028A5
:10EEA00000F08E8248F480734345338009D0214BB3
:10EEB000022214211A700E20FF2259709A702BF032
:10EEC00093F8204B1B78082B00F086820E2B00F065
:10EED0008382069B1C6860056FD51B4B1B79002B3A
:10EEE00000F0338214211248FBF752F8002840F05A
:10EEF000318220F097FC01202AF0C4FF00285AD06C
:10EF0000DFF84CA000244FF0CC0BA94625E000BF51
:10EF1000B8240020AC250020B02500208865002002
:10EF200080650020D44C0020AC670020D94200202E
:10EF30003095002090420020DC5D0020E05D002044
:10EF40009C7D0020D84900208C7D00202C6500206D
:10EF5000788E0020DCB2022C2CD80BFB04F8631C4A
:10EF60005AF80850002DF5D1032290F9023002958D
:10EF70000192C278E24951F82220009218462A46AE
:10EF80002B4601212AF0C8FD034604EB440000EBA8
:10EF900000100D9353B129460AEB8000CC222DF0CE
:10EFA00074FF0D9B4AF808300134E4B222F0E4FC0F
:10EFB0000028D0D14D46069B1C68079B93F800A003
:10EFC000D04B1AF0010A00F05A8201221A70099BF4
:10EFD00004991B68B1F906105A89CB484FF0010E0D
:10EFE000914280F800E080F23082C84B4FF07E52B0
:10EFF0001A60C74A059B0498B3F81880B0F900E07E
:10F0000092F90430107892F801C0002BAEEB08039F
:10F0100014BF01224FF0FF32002BB8BF5B42B3F5A3
:10F02000FA7FA8BF4FF4FA73984280F2B0821B1A9D
:10F0300007EE903AF8EEE77AC645C7ED007A03DAB4
:10F04000F1EE677AC7ED007A049BB3F902E0AEEB0C
:10F050000803002BB8BF5B42B3F5FA7FA8BF4FF49B
:10F06000FA73984280F2EE811B1A07EE903AF8EE9E
:10F07000E77AF045C7ED017A03DDF1EE677AC7ED77
:10F08000017A049BB3F90400A0EB0803002BB8BF7E
:10F090005B42B3F5FA7FA8BF4FF4FA736345CCBF68
:10F0A000A3EB0C03002302FB03F307EE903AF8EE08
:10F0B000E77A4045C7ED027ABCBFF1EE677AC7ED4B
:10F0C000027A14F4805400F09A81B1F5FA6F914BF2
:10F0D000A8BF4FF4FA61B1F57A7F1A78B8BF4FF440
:10F0E0007A71A1F57A71002A41F0A0818A4ADFF88D
:10F0F00040E282FB0130CB17C3EB6013581C6FF06A
:10F10000630C3EF910003EF913E00CFB0313A0EB77
:10F110000E0003FB00F382FB0312DB17C3EB621349
:10F120009E440FFA8EFE07EE90EAB8EEE78A87ED6E
:10F13000038A002C40F0AE8333885A0640F1FA80EF
:10F140007649774A91ED018AD2ED019A92ED026AF1
:10F1500091ED034A92ED030A91ED029A92ED007A45
:10F16000D1ED005AD7ED011A97ED002A6D4A6E498C
:10F1700038EE445A79EEC63A77EE007A65EE233AD5
:10F1800075EEC96A75EE890A37EE401A66EEA76A0F
:10F19000B0EE633AA0EE813A13F00303B0EE665A84
:10F1A00078EE044A79EE867AA0EE815AF0EE638A10
:10F1B000A4EEA73AD4EEA78AA4EEE75A33EE263A95
:10F1C000F0EE687AF0EE674AF6EE008A35EE88AA2D
:10F1D000E0EEC14A28EEC33A35EE635A77EE293A9B
:10F1E00077EEE67AAAEE233A25EE285A76EE403AF2
:10F1F00034EE49AAE0EE817A74EEA64AAAEE235ACA
:10F2000034EE094A37EE697A64EEA84A63EE036A7F
:10F21000E4EE074A75EEC85A36EE006A67EEA87A41
:10F22000B0EE667A95EE057AE5EE056AE5EE867A49
:10F23000B1EE648AF0EE665AF0EE476AB1EE674AC4
:10F24000E8EE246A63EE270A67EEA43AE4EE275A52
:10F25000B1EE450AB0EE609AB0EE631AA4EE277ADA
:10F2600023EE244AE7EEA76AA5EE249AA0EE031A3D
:10F27000E8EE245AB0EE448A31EEA16AE0EE240AA8
:10F28000A5EE278A66EEA16A72EE028AE5EE033ADF
:10F2900061EE211A26EE096AA4EEA47AA0EE274AAE
:10F2A0000CBFD7ED022ADFED212A82ED005AA2EE33
:10F2B000256AE8EEA06AE2EE081A73EEA33A27EE9A
:10F2C000227A34EE044AF0EE005AE3EEA26AA4EE8B
:10F2D000226AA1EEA57AC7ED016AC1ED376A81ED18
:10F2E000366A87ED006A81ED387A82ED013AC2ED27
:10F2F000027AC2ED034AEBB987ED027A1AE000BF49
:10F30000D4F00308654A002048250020C0240020CE
:10F3100074950020084F00201F85EB51A0000020AD
:10F32000B0000020E8000020C41F00200000000002
:10F33000882D0020BAF1000F40F02C812BF0F8FA54
:10F3400017B0BDEC068BBDE8F08F079B1B78D90783
:10F350007FF5CFAD4FF40F7021F054FD00283FF43E
:10F360002AAE1CF04FFB4FF40F7021F0B5FC0028C3
:10F370003FF421AE1CF046FB4FF40F7021F0ACFCC3
:10F380000028EED117E6DFF89093D9F800309907FE
:10F390007FF50CAD3788FA073FF529AD47F001033B
:10F3A0009F4233803FF423ADC54B022214211A70D3
:10F3B0000E20FF2259709A702AF016FE378816E543
:10F3C00028F480739BB2434533807FF470ADBD4B0E
:10F3D0001B78082B7FF47AAD328822F040039BB271
:10F3E0009A4233803FF475ADB54B022214211A7056
:10F3F0000E20FF2259709A702AF0F6FD69E5059BF0
:10F400005A8B9142C0F2EF84B1F5FA6FD4BFC2EBD0
:10F410000101C2F5FA614FF47A7303FB01F1AA48C6
:10F420000378C2F5FA62B1FBF2F1002B3FF45EAE55
:10F430004378A64A01FB03F182FB0123C917C1EB04
:10F44000631153E6DFEDA27A13E6B1F5FA6F80F2AD
:10F45000C384187A8B1A03FB00F3C2F5FA6293FB9C
:10F46000F2F3C3F1640307EE903AF8EEE77A9FED0A
:10F47000997A994B67EE877AC3ED007AB9E51B78E4
:10F480000693002B7FF4A3AD944A1268002A3FF440
:10F490009EAD934A079212F8030CDFF880B2114632
:10F4A000A2F1030912F0ACF89BF80080079A00283B
:10F4B00000F02886069BB8F1000F41F0D48509F1D1
:10F4C000080199F8050012F09BF8002841F06386C6
:10F4D000844999F80A0012F093F8002800F0278672
:10F4E000B8F1020F41F053867F4999F80F0012F0EE
:10F4F00087F8002841F05F867C4999F8140012F0E3
:10F500007FF8002800F02786B8F1040F41F04F86FD
:10F51000774999F8190012F073F8002841F04386F2
:10F52000744999F81E0012F06BF8002800F0278645
:10F53000B8F1060F41F033866F4999F8230012F0B5
:10F540005FF8002841F018866C4999F8280012F0FD
:10F5500057F8002800F02786B8F1080F41F0088618
:10F56000674999F82D0012F04BF800283FF42FADB1
:10F570000922134602EB82029144624A99F8010083
:10F5800099F802108BF80030107051701FE5DFED14
:10F59000507A51E50A9B19780B9B01F0010118681C
:10F5A000FEF798FD17B0BDEC068BBDE8F08F13B9E0
:10F5B000089A01239370544B089A1D7892F82140C1
:10F5C00007931B2012F046F8012C05F00108814634
:10F5D00000F0A68705F00205089A4C4E92F82030FC
:10F5E000DFF83CA14A4F09959346052B01F23B8079
:10F5F000DFE813F0C100B7000600FF000101F400CE
:10F60000012C04BF05238BF82030B8F1000F12D075
:10F61000059B3088B3F918100022134661F30F02DE
:10F6200060F31F4261F30F03049861F31F4303600B
:10F63000032342600993374DDBF814102A68914286
:10F6400080F0B28647F230510322CBF81C108BF8C1
:10F65000202002200CF0B0FD0DF030F92968DBF815
:10F660001C200A440421CBF818208BF82010012C10
:10F6700041F03F802A68DBF81810914280F0F38750
:10F680009AF8000020B911F0E5FF002840F0EB8760
:10F690003A6822F002023A602A687388642101FB0A
:10F6A00003234FF480600022CBF810308BF8202029
:10F6B0008BF803200CF050FD9BF8203095E700BF3D
:10F6C00090420020D8490020084F00201F85EB51B0
:10F6D000000000000AD7233CC0240020684A002014
:10F6E0003A42002044420020494200204E4200207D
:10F6F00053420020584200205D4200206242002018
:10F70000674200206C4A0020644A0020802D0020BF
:10F710007C650020D45D00202C6500201C000020AA
:10F72000D71C002011F09CFF012807D1834D72885F
:10F730002B68642101FB0233CBF81030B9F1000FC4
:10F7400002D0B379002B4BD1012C00F08C877B4D7C
:10F75000DBF810102A689142C0F0D88701238BF89B
:10F760002030012C3AD0F379012B46D011F006FF5E
:10F770009BF8203039E7B8F1000FD3D1099D4FF441
:10F780008060B9F1000F00F04F830CF0FDFC089A87
:10F7900000231361002D3FF45FA928462AF024FCC2
:10F7A000069B1E6816F480573FF45CA91D2164482F
:10F7B000FAF7EEFB00287FF455A9624B03F15009DC
:10F7C00003E00433994500F054871A78262AF8D1CB
:10F7D0009978DA789142F4D2FFF746B9574D5BE752
:10F7E00011F0CCFE03224FF47A738BF82020CBF873
:10F7F0001C30524D2DE7514D39E711F0BFFE032269
:10F8000040F6B8338BF82020CBF81C304B4D20E766
:10F810004D4F3B78002B01F05D834C4BDFF8488166
:10F82000DFF848B1DFF848A1059345465E460490ED
:10F8300099460EE019F804109847032C28DC88B983
:10F840003B782AF8020F01349C4205F1040580F24E
:10F850006D81072CE1B23046DBF80430EADD9847D1
:10F8600000B2EDE738F824206B88801A4FF47A71E3
:10F870009B1A01FB00F040F6CA0290FBF3F008442B
:10F88000904240F2EE23A8BF10469842B8BF1846F7
:10F8900000B2D5E71D212A48FAF77AFB002840F08C
:10F8A000A3860C9B03E00433AB423FF445AC1978CC
:10F8B0002629F8D19878DA789042F4D2089BDB7840
:10F8C000002B7FF439AC1E48FAF762FBDFED207A9B
:10F8D000002801F0168338EE678A1E4A1E49FDEEA5
:10F8E000C87ACDED047ABDF910301B0382FB030208
:10F8F000DB17C3EBA212C8F57A731BB203FB02F34A
:10F9000043F30F33434407EE903AF8EEE77A0123CE
:10F91000C7ED037A0B700FE4104B1B789C0704D5DE
:10F920000F4C237D042B00F2FC86B6F8008018F003
:10F93000300F40F046840B4FFFF7ADBAD45D002086
:10F9400030950020D44C00209C4D00209C7100205C
:10F9500000007A44D34D62103C25002082650020CF
:10F96000286B00209C7D0020B04D0020389800209E
:10F97000C21F0020DFF8ACB1DFF8AC91614C9846B3
:10F980000BF15A074FF0010A59461BF8010C11F010
:10F9900037FEF8B19BF804009BF802309BF803E0B7
:10F9A00000EB400104EB8101013BD1F8A02003EB07
:10F9B00043034B4493420DD094F8CC2081F89CE053
:10F9C0000AFA00F022EA0000C1F8A030C1F8A480D1
:10F9D00084F8CC000BF1060BBB45D5D14A4B4B4A02
:10F9E0001B780A93099B4A4C1B68D2F800900B9332
:10F9F000A4F19C0B4FF0000A63686BB31F785FB3F0
:10FA0000A268A9EB0202002A0BDB9BF8CC200121A3
:10FA100001FA0AF122EA010209F5FA718BF8CC2009
:10FA2000A1600A9AC2B1227859780432D2B2002970
:10FA300040F0538305990498098B30F9122001F1A5
:10FA4000C800824240F327869BF8CC109A7841FA8E
:10FA50000AF3DB0740F1D4860AF1010ABAF1040F78
:10FA600004F10C04C8D1FFF793B92A4B03E0043327
:10FA70009D423FF488A919782329F8D19878DA783B
:10FA80009042F4D22448FAF783FA00283FF47BA985
:10FA9000224B1B6813F4003341F0FD820022204BFF
:10FAA0001046995C142902F10C0201F0C381013067
:10FAB0001828F6D1FFF767B9124C94F896305BB16D
:10FAC000079B1B78DA0707D5049BB3F90620059B33
:10FAD0005B8B9A4200F3868611210F48FAF758FA99
:10FAE000002800F0DF8294F89A302BB994F8943013
:10FAF00013B93223A4F89830012384F89A30FFF721
:10FB000003B900BFC41F0020352F0020D45D0020A2
:10FB100060200020D44C002030950020444100207B
:10FB2000A4E503085141002074D00308DDF81090CB
:10FB3000BF4A0692BF49126842F2010AA1FB091BA3
:10FB400012EA0A0A4FEA9B1B00F0BE82BA4DBB487C
:10FB5000BB4CBC492E780078267008701EB1B9499C
:10FB60000E7886F00106B84C0F2184F82410002B83
:10FB700000F05F84059DB54BB5F826C0B5F824E0CC
:10FB8000059D109318462D8B0078B14B129594F873
:10FB900025500995AF4D0495A3FB00535B0803EB7B
:10FBA0004303C31ADBB20F90CDF834C002F4805285
:10FBB0000C9304F128000BF59673CDF8449097F858
:10FBC0000080DDF82490DFF8D0C20994A14C0E919A
:10FBD000139200210A930896CDF81CE0089B002B95
:10FBE00000F08483099B079D33F911201FFA82FEE0
:10FBF000AE454FEA410303D30D9DAE4540F2BB83B2
:10FC00005CF82120934580F07B83E25EBAF1000F1F
:10FC100040F0908301314145E25200F10600DDDB06
:10FC20000E9A099C8C4B84F824200F2A49460CBF5D
:10FC300001220022DDF8449084F825101A7000F0AB
:10FC4000FF83864B7D497F4ADFF850B208931C46FC
:10FC5000042001230B7013700CF0AEFADBF80030B7
:10FC6000A1686268E3605B1A934284BF002384F852
:10FC70002130069B3C781E68002C01F03E81059ADD
:10FC8000774DB2F824E0178B724916F48056284657
:10FC900040F00E8432460EE0437803EB830303EB1F
:10FCA000830303F2EE239BB20132A24221F8023B0E
:10FCB00000F102000ED015F81230002B00F05F8327
:10FCC000022BE9D001320B8821F8023BA24200F15D
:10FCD0000200F0D1109A137801331370FEF7A3BE1F
:10FCE000594CD4F88830A9EB0303002BFEF6A9AEDB
:10FCF0005C4A5D4B527C059933F812308A7DDFED0A
:10FD00005B6A9FED5B6AC97D9BB207EE102A07EE26
:10FD1000903AB8EEC77AF8EEE77A27EE267A67EEE1
:10FD2000867A0B9AC4F88820C7EE876A40F2FF32C1
:10FD3000FCEEE67ACDED077ABDF81C30934228BF81
:10FD4000134609B1D31A9BB24A484B4D01784B4C2C
:10FD500035F81160226825F81130921B13440131E7
:10FD6000474D236001F00F021B0902702B80FEF744
:10FD700068BEFDF7AFFC434B434A1B68C31A93426E
:10FD80007EF75FAE3E4B00221A80FEF75ABE059A00
:10FD90000499537DD27D013B31F913301AB1C3F57B
:10FDA0003B6308331BB2A3F57A7307EE903A9FEDDD
:10FDB000377A334AF8EEE77A40F2FF3167EE877A16
:10FDC000FCEEE77ACDED077ABDF81C308B4228BFF8
:10FDD0000B461380FEF735BE1B7AC3F1640307EEB2
:10FDE000903AFFF742BB2146FFF719BB0221284892
:10FDF000FAF7CEF800283EF4FAAF3480BB073FF59F
:10FE000007A847F00203BB4233803FF401A8214B0F
:10FE1000022214211A700E20FF2259709A702AF0C3
:10FE2000E3F83788FEF7F4BF0CF096F9AFE400BFB3
:10FE3000C07A0020D34D6210044C00202001002025
:10FE4000352F002021010020C41F0020894C0020F4
:10FE5000ABAAAAAA8091002056980020442F002027
:10FE6000E44D0020985F0020B85F00200000C842E9
:10FE700000008044274900202C4900202849002008
:10FE80003E2F0020D825002060E316006F12833F2C
:10FE900030950020904200208C4C0020D45D002042
:10FEA000DE4AB2F90030002BB8BF5B42B3F5E17F08
:10FEB000BEF6E9AFB2F90230002BB8BF5B42B3F532
:10FEC000E17FBEF6E0AFD64B93ED096AD3ED076A4A
:10FED00093ED057AD3ED037A76EE866A77EE877A2C
:10FEE00076EEA66AB7EE007A37EE666A77EEA77A04
:10FEF000B0EEC66AF0EEE75AB4EEE56AF1EE10FA3B
:10FF0000B4BFB0EE655AB0EE465AB5EE405AF1EEC7
:10FF100010FA40F037849FEDC37AB4EEE56AF1EE53
:10FF200010FA44BF9FEDC06A36EE477AB7EE006A1A
:10FF3000F4EEC66AF1EE10FAC8BFDFEDBC6AF5EE6A
:10FF4000C07AC8BF36EEC77AF1EE10FA48BFB1EEFC
:10FF5000477AF6EE007A27EE677ADFEDB37A77EE2E
:10FF6000276ABDEEE66A16EE103A2033402B40F2C7
:10FF7000FE86DFEDAF6AAF4ADFEDAD7AC2ED006A13
:10FF8000FDEEC76AC2ED017A16EE903A2033402B9F
:10FF9000C2ED027A49D8DFEDA57AB4EEE77AF1EE48
:10FFA00010FA41F37F819FEDA46ADFEDA46A01E0BE
:10FFB000B0EE677AB4EEE67AF1EE10FA77EE467AB2
:10FFC000F6DC9FED9F7AF4EEC77AF1EE10FA41F17C
:10FFD00065819FED996ADFED9B6A01E0F0EE477A5B
:10FFE000F4EEE67AF1EE10FA37EE867AF6D4DFED2B
:10FFF0008E7AB4EEE77AF1EE10FA40F35587DFED32
:020000040801F1
:100000008B7A37EEC77A27EE076ADFED8F5ADFED7E
:100010008F6ADFED8F7AE6EE256A67EE065AE6EE26
:10002000267AA5EEA77AF0EE477A8A4BC2ED037ADC
:100030001A6812F4003240F01487874B1046995C1E
:100040000A2902F10C0200F0038601301828F6D1CB
:10005000FEF719BF24F040039BB2A34233803EF465
:100060000BAF7E4B022214211A700E20FF22597012
:100070009A7029F0B9FFFEF7FFBE338823F004041D
:10008000A4B2A34234803EF4EDAE744B022214219C
:100090001A700E20FF2259709A7029F0A5FF34883B
:1000A000FEF7E0BE94F89430002B3EF42DAE079B93
:1000B0001B7813F001037EF427AE012284F89430FC
:1000C00084F89520FEF720BE65490E7846E5654C1C
:1000D000012184F88C10FEF742BD012900F0D4857F
:1000E0009BF8CC20012303FA0AF30AF1010A134317
:1000F000BAF1040F8BF8CC3004F10C047FF47CAC23
:10010000FEF746BE511D99F8050011F079FA002856
:100110003FF4DEA9B8F1010F41F03D8009F10D0176
:1001200099F80A0011F06CFA002841F030804E492D
:1001300099F80F0011F064FA00283FF4DDA9B8F136
:10014000030F41F03880494999F8140011F058FA2A
:10015000002841F02C80464999F8190011F050FA16
:1001600000283FF4DDA9B8F1050F41F01C8041499A
:1001700099F81E0011F044FA002841F010803E4921
:1001800099F8230011F03CFA00283FF4DDA9B8F1FA
:10019000070F40F0F187394999F8280011F030FA3B
:1001A000002840F0E587364999F82D0011F028FA2B
:1001B00000283EF40CAFB8F1090F3EF408AFFFF78A
:1001C000D7B910200BF0C8FF20200BF0C5FF2D4B36
:1001D000B6F800802C4F00221A702C492C4A2D4C66
:1001E0002D4800230B602D4923604FF0000E036063
:1001F00053609361C2F800E0C2F808E0C2F814E06E
:10020000C2F81CE0C1F800E04B60C1F808E0C1F89A
:1002100014E08B61C1F81CE0FEF73DBE30650020A4
:10022000C0000020A7DFA834DB0FC93FDB0F494027
:1002300000000000A0000020DB0FC940E4CB164105
:10024000DB0F49C0E4CB16C192E741B99730083CB7
:1002500015A82ABE44410020A4E5030890420020CE
:10026000352F0020C41F0020494200204E420020AC
:1002700053420020584200205D420020624200208C
:10028000674200203E3D00209C7D0020283E00204B
:10029000D83D0020E4240020A4250020003E0020BA
:1002A0005D2A00F0B2825B2A00F04C865E2A00F0E4
:1002B000D586562A00F0DA86972A00F04E87A72ABC
:1002C00000F0C086B44E3388980740F07F86A2F1D4
:1002D000B703072B00F2D382DFE813F0C302D10289
:1002E000D102D102B502D102A702A702079B002BBF
:1002F0003FD05CF8212093454FEA4103FFF485ACE1
:10030000A64AA64DD25C05EB030E002A00F0B18090
:10031000022A47D19EF8012002EB820202EB820200
:1003200002F2EE2292B2032933DD12B2BAF1000FCB
:100330003FF470AC0C9D20F81520B9F1000F03D1EB
:100340000F9D022D7FF666ACB0F802900288B0F8DF
:1003500004E04A449644924A0FFA8EFE82FB0E5203
:10036000904DA2EBEE7225F803E012B24FF00109B6
:1003700050E41A464B000A9D4CF8215046E4D3B293
:10038000022B04D9032B7FF49DAC73468CE43B46CF
:100390008AE4012505FA01FE0E9D25EA0E0512B23A
:1003A0000E9533E4E25ABEE77F4A1278002A7FF4C2
:1003B00049A9B8F1000F3FF445A9012C40F0538141
:1003C0009BF82030FFF711B931467848F9F7E0FD86
:1003D000002800F0BC8084F893600CF069FDFEF703
:1003E00016BC44F04003A34233807FF43AAEFEF7DC
:1003F00043BD44F004039C4233800AD06C4B02227C
:1004000014211A700E20FF2259709A7029F0ECFD09
:100410003488684B684AB3F90430684982FB0302A8
:10042000DB17C3EBA2030B80FEF71CBD5B78FFF765
:1004300000B8634B634A109201221A70624B049316
:100440001B215A48F9F7A4FD00287FF4FAAB5F4B53
:10045000DFF88CB108931946DBF80030CA688B606E
:100460009B1AC82B00F23A85069B1E6806F480563C
:1004700030E4CAB2022A40F20484032A92D1129ACA
:10048000139D079E002D08BF32464CE727F001035D
:100490009BB2BB4233803FF4B1AC0E2084F80080A5
:1004A00084F801B084F802A029F09EFD3788A5E405
:1004B00000220FE0437803EB830303EB830303F293
:1004C000EE239BB20132A24221F8023B00F102006E
:1004D0003FF400AC15F812301BB1022BEAD00B88A8
:1004E000F0E7D3B2032BFAD83B46EBE7B2F5FA7F3D
:1004F000FEF602AC94F89230002B7EF4FDAB079B25
:100500001B7801210B4084F8921000F01D840CF040
:10051000D5F9214E069B2E4A1B680992FEF7F1BBC6
:100520000025FFF759B8B2F5FA7FFEF6E5AB94F86F
:100530009220002A7EF4E0AB079B1B78012184F80F
:100540009210D90700F1BD840CF0B2FCE1E7079BE3
:10055000204A1B781060D8077EF55DAB1E4B1B78D8
:10056000002B3EF4C9AB089BDB78002B7EF4C4ABB8
:1005700094F893300133DBB2032B84F893307EF68A
:10058000BBAB164B5B7813B9002D7EF4B5AB0CF00A
:1005900095F9FEF73CBB00BF80650020E44D0020CC
:1005A0005655555534200020002500203095002058
:1005B000904200203065002067666666483E002055
:1005C00056980020894C002080910020442F002064
:1005D0008865002068260020352F00209C9500208B
:1005E000D45D002000007A44089BDB78002B7FF468
:1005F00058A95FED047AC54938EE678AC8F5FA63F1
:10060000FDEEC87A1BB2CDED047ABDF910201203BD
:1006100081FB0201D217C2EBA11203FB02F343F3E9
:100620000F33434407EE903AB8EEE78A0C9B87ED10
:10063000038AFFF73CB9B64AB4491068B4F9902070
:10064000C66981FB06018911F617701A00F5FF4093
:100650007F3082423EF7CEAA891B0A4412B2A4F828
:100660009020FEF7C7BA099D002D3EF4F5A9FFF7CB
:1006700094B8A84A059BD588049A1B8BB2F906103A
:100680005A1B914240F3AB802B449942B4BF0025E2
:100690000125FEF7F2B9C8398A4265DA9BF8CC1019
:1006A0009A7841FA0AF3D8073FF5D6A952420120B9
:1006B0000D9229F0BFFD7B1E0D9A162B00F27C8156
:1006C000DFE813F05E02740245029D028A02B10265
:1006D00030021B020402ED01D6017A019D02C10124
:1006E000B10230021B02AA0193017D016801500191
:1006F0000C01AB460899DBF80020CB69099D134437
:100700008B61002D3EF4A8A9FFF747B810F036FF23
:10071000032140F6B8328BF82010CBF81C20FEF7EE
:1007200098BF0A2010F096FFB6F800808146002896
:1007300000F0658318F0100F00F0F984764C94F8FF
:10074000D490B9F1000F7FF4F6A8744F0D2029F072
:100750004BFC012384F8D430B6F80080B9F1000FC7
:100760007FF43BADFEF797BB9BF8CC30012202FA39
:100770000AF223EA020309F5FA728BF8CC30A26080
:10078000FFF76AB9B4EEE56AF1EE10FA8CBFB0EE8D
:10079000654AB0EE464AC4EE054A9FED612A9FEDD8
:1007A000615ADFED611ADFED612A9FED613ADFEDFD
:1007B000613A9FED614AA4EE825AE4EEE12AA4EE8A
:1007C000857AA4EEA23AB0EE475AB0EE637AA4EE70
:1007D000837AA4EE874A84EE057AFFF79EBB012553
:1007E000FEF74BB900215548F9F7D2FB00287FF4FA
:1007F00073A9322384F89600A4F89830FFF76CB9F7
:10080000002A0CBF0120022052E74D4B002201209C
:100810004C494D4C0B604D4B0993227029F00AFD59
:10082000069B4B4E1B68FEF76CBA484A464B099232
:100830001146484A0A6002225A7010F06FFF069B68
:100840001B68FEF75EBA414A3F4B09921146424A85
:100850000A6000225A7010F061FF069B1B68FEF7C9
:1008600050BA3A4A384B099211463C4A0A60012272
:100870005A7010F053FF069B1B68FEF742BA792AA4
:1008800000F0E8847A2A00F0DE849E2A00F0D38407
:100890009D2A00F0C884AE2A00F0BD84AD2A00F085
:1008A000B284EF2A00F0AC84FD2A00F09784FB2A82
:1008B00000F06F85FE2A00F06985F72A00F0FE84BB
:1008C0007B2A7FF427AE4FF4FA6102200DF026F95F
:1008D0001E4B0993069B1B68FEF713BADBF8D0008A
:1008E000DFF87C8090F8361098F8023011446429C3
:1008F000A8BF642121EAE17180F83610002B40F096
:10090000E7840FF0DBFFFFF7EBBB00BFD34D6210B6
:1009100078660020682D0020C41F00209C7D0020E8
:1009200099FB243F69A2163E39094E3DE3B59E3E30
:1009300088FA163E45FE7F3FA7DFA8343095002099
:10094000E45F002084650020059800208865002071
:10095000806500202A980020129800201E98002010
:1009600004610020DBF8D000DFF85C8690F83710D7
:1009700098F802301144FE29A8BFFE2121EAE17156
:1009800080F83710002BBCD0162010F0ADFEDBF83D
:10099000D000B6E70B98DFF8308641781144B1F506
:1009A000967FA8BF4FF4967121EAE171417098F8E3
:1009B0000230002B40F08584DBF8D000A1E7DBF8A3
:1009C000D000DFF8048681781144C829A8BFC82167
:1009D00021EAE171817098F80230002B91D0142047
:1009E00010F082FEDBF8D0008BE7DBF8D000DFF8F8
:1009F000D88541781144C829A8BFC82121EAE171EE
:100A0000417098F80230002B3FF47BAF132010F0B8
:100A10006BFEDBF8D00074E7DBF8D000DFF8A885C8
:100A200001781144C829A8BFC82121EAE1710170E9
:100A300098F80230002B3FF464AF122010F054FEFF
:100A4000DBF8D0005DE7DFF880850B9898F802307E
:100A5000417911446429A8BF642121EAE1714171FF
:100A6000002BA9D00E2010F03FFEDBF8D00048E7A5
:100A7000DBF8D000DFF85085017A98F80230114495
:100A8000C829A8BFC82121EAE1710172002B3FF4F7
:100A900038AF0B2010F028FEDBF8D00031E7DBF890
:100AA000D000DFF82485C17998F802301144C829B4
:100AB000A8BFC82121EAE171C171002B3FF421AF29
:100AC0000A2010F011FEDBF8D0001AE7DBF8D000A6
:100AD000DFF8F484817998F802301144C829A8BF5E
:100AE000C82121EAE1718171002B3FF40AAF09208E
:100AF00010F0FAFDDBF8D00003E7DBF8D000DFF8F8
:100B0000C884417998F802301144C829A8BFC82187
:100B100021EAE1714171002B40F0DF83112F7FF456
:100B200052AFEEE6DBF8D000DFF89C84017998F84C
:100B300002301144C829A8BFC82121EAE17101711E
:100B4000002B40F0DF83102F7FF453AFD9E60B99D1
:100B5000DFF874840F791744642FA8BF642727EA4D
:100B6000E7770F7110F0DAFD98F80230002B3FF4B0
:100B700023AF0320394610F0B7FDDBF8D000C0E604
:100B80000B98DFF8448401781144FA29A8BFFA21B0
:100B900021EAE171017098F80230002B3FF40CAFAC
:100BA000012010F0A1FDDBF8D000AAE60B98DFF8D9
:100BB0001884817811446429A8BF642121EAE17175
:100BC000817098F80230002B3FF4F6AE022010F04E
:100BD0008BFDDBF8D00094E60B98DFF8EC83C1794D
:100BE00098F80230114481F30801C171002B3FF4E1
:100BF000E3AE052010F078FDDBF8D00081E60B9B1A
:100C0000DFF8C483997998F8020011446429A8BFD9
:100C1000642121EAE1719971002840F066830D2F6B
:100C20007FF413AFC8E6DBF8D000DFF89C83C1780F
:100C300098F802301144C829A8BFC82121EAE171FF
:100C4000C170002B40F09A830F2F7FF4E9AE58E675
:100C5000BE490C6847003CB13A1803EB8202647845
:100C60005278A242BEF40FA90744B94CB948D9F84A
:100C7000002003EB870300270B6027800760FEF747
:100C800004B9129AFFF74FBB049931F912209978F1
:100C9000B2F5617F4FF4966393FBF1F3C0F2E98004
:100CA00040F633019142A8BF11460C2FA1F56171A6
:100CB00091FBF3F100F08382182F7FF411AAC9B2DF
:100CC000C8290B46A8BFC823DBF8D000C27DDFB21D
:100CD00097423FF405AA9A1ADFF8EC82C77548BF1D
:100CE0000732D71098F802300137FFB23BB9002F16
:100CF0003FF4F6A9384629F09DFAFFF7F1B918201C
:100D000010F0F2FCF3E7944B94491A684FF47A73AD
:100D1000B3FBF2F3C3EB431203EB8202069B1B68A7
:100D2000D2001F06A1F8A8207DF5E8AF8C4A127802
:100D300096077DF5E3AF8B4A127D042A7DF6DEAF80
:100D400012F0B8F8FFF7E5BB8749096811F40031E4
:100D500040F0FC81854B08465D5C0F2D01F10C01D4
:100D60003DF4B0AF01301828F6D1FDF7BFBFB4EEA7
:100D7000E77AF1EE10FA40F39E82DFED7D5A9FEDA7
:100D80007D6A01E0F0EE676AF4EEC66AF1EE10FAF1
:100D900076EEE57AF6DCDFED786AF4EEE67AF1EEEF
:100DA00010FA40F18582DFED725A9FED746A01E01E
:100DB000F0EE667AF4EEC67AF1EE10FA77EEA56AF6
:100DC000F6D4DFED6F7AF4EEE76AF1EE10FA40F355
:100DD0002D81DFED6C7A77EEE66A66EEA65A9FED1E
:100DE0006A5A9FED6A6ADFED6A7AA5EE856A26EE99
:100DF000A55AE5EE867AE5EE276AFFF7BCB818F04B
:100E0000100F40F089810B2010F024FC002840F0E6
:100E10004B81604F18F0200F40F0B2815E4C94F887
:100E2000D430002B3FF492ACB9F1000F7FF4D5A978
:100E3000FEF731B845490F6842003FB1141803EB83
:100E400084047F786478BC42BDF49DAF0244404C7A
:100E5000404803EB820300220B6022800260FDF712
:100E600092BF4E4B1B78032B00F0AB810022FFF7A3
:100E7000E4B80C2F40F0098100273946484B0D910A
:100E80005B78BB423FF42CA9DFF83C8138460CF07C
:100E90001FFF98F802300D991BB1C9B20C2010F059
:100EA00023FC0137FFB222E7DFED3E7AB4EEE77AAA
:100EB000F1EE10FA44BFDFED307A37EEC77AFFF774
:100EC000A2B83949069B0A60384A1B68384E099215
:100ED000FDF717BF374A0592FEF72ABE364A069B32
:100EE0001E68136823F004031360089A012306F4B4
:100EF000805682F82130FEF7EDBE06F48056FEF7EC
:100F0000E9BE38EE678A2D4B2D491870FDEEC87A80
:100F1000C8F5FA63CDED047ABDF91020120381FB08
:100F20000201D217C2EBA1121BB203FB02F343F37F
:100F30000F33434407EE903AF8EEE77AC7ED037AB1
:100F4000FEF7FAB81F4B0122022061E4B82400200A
:100F5000AC250020B0250020B07A0020D4720020FB
:100F600082650020286B002044410020A4E503088E
:100F7000DB0FC940E4CB1641DB0F49C0E4CB16C1FF
:100F8000DB0FC93FDB0F494092E741B99730083C7E
:100F900015A82ABE9C7D0020C41F0020412F0020E0
:100FA00005980020DB0FC9BF682600208865002057
:100FB000806500209C7100207C6500203C2500207D
:100FC000D34D621032600020046100200023BB2A50
:100FD000149300F06081B72A00F05981BE2A00F016
:100FE0006581BD2A7FF44BAC4FF6FE71CD4ACE48E9
:100FF000D589099090892B4401449181D38118F0BF
:1010000015FFF7F7D7FF18F0F9FEFBF765FB012096
:1010100029F010F9B4F89020069BFA3A00211B68D9
:10102000A4F8902084F89210FDF76BBEDFEDBF7A34
:10103000F4EEE76AF1EE10FA44BFDFEDBD7A77EE29
:10104000E66ACAE6BB49069B0A781B68BA4E42F0BC
:1010500004020A70B44A0992FDF753BEB74B02224C
:101060000320FFF7D5BB1A46FEF784BA18F0DEFE60
:10107000F7F7A0FF18F0C2FEFBF72EFB012029F0C6
:10108000D9F894F88E20FFF717B9182F7FF428A805
:1010900000210B4618E6AA4B1B78032B7EF4FEAC0E
:1010A00028F086FFFDF76FBEA64BA74F5B8997ED33
:1010B000007A07EE903AF8EEE77AB0EEC77AB4EE2F
:1010C000E77AF1EE10FA7FF5A5AE97ED017AB0EE72
:1010D000C77AF4EEC77AF1EE10FA7FF79BAE18F0FC
:1010E000200F7FF49BAE20200BF04EF894E80C000C
:1010F00096490A60084641F8043F27F0B3FD944B37
:1011000001221A70934C94F8D430002B00F0F38035
:10111000B6F80080FFF761B810200BF01DF88C4B7B
:10112000B6F8008083F800904FF001096BE61020BC
:101130000BF02AF820200BF00FF88749824F081F88
:1011400027F090FD824B02221A70DBE77C49097878
:10115000032900F096801946FCE5804A069B764EEE
:101160001B684FF4C87111806F4A0992FDF7C9BD21
:1011700008221346FEF7FEB907221346FEF7FAB916
:1011800020200AF0E9FF724B00221A70BAE702220F
:101190001346FEF7EFB901221346FEF7EBB906221C
:1011A0001346FEF7E7B905221346FEF7E3B904221A
:1011B0001346FEF7DFB903221346FEF7DBB9CFB2C1
:1011C0005CE628F0F5FEFDF75EBE574B84F8941000
:1011D00084F89500584E0993FEF76FBC002101205A
:1011E0000CF09CFCB4F89020069B4F491B680991B9
:1011F000963AA4F89020002284F89220FDF781BD51
:1012000000210846ECE7FF21002017F014FD94F8B8
:101210008E20FFF746BB0121002017F00CFD94F84B
:101220008E20FFF73BBB0021FF2017F004FD94F850
:101230008E20FFF730BB0021012017F0FCFC94F852
:101240008E20FFF725BB464A137A43F00103137241
:10125000FFF760B9424A137A23F001031372FFF7D4
:1012600059B9002D3DF44FAC3A4C94F88D30002B19
:101270003DF47AAC28F09CFE002384F88D30FDF715
:1012800073BC28F095FEB4F99020FDF72FBD1946E8
:101290004FF6FE73AAE619460223A7E6B0EE677A78
:1012A000FEF7A5BEF0EE477AFEF78BBE02219DE663
:1012B000F0EE676A85E5F0EE667A6CE500210420C1
:1012C0008EE7152010F010FADBF8D000FFF719BBFD
:1012D000172010F009FAFFF76FBB11200D9210F0E4
:1012E00003FADBF8D0000D9A18E40D200D9210F0EF
:1012F000FBF90D9A93E44FF00109FFF727BA0B2091
:10130000FDF7B0BC10200D9210F0EEF9DBF8D00024
:101310000D9A18E40F4C0BF0D1FA002384F88D30AD
:10132000FDF722BC7C95002088650020DB0FC9BF3B
:10133000DB0F49C0826500208065002080600020AE
:10134000412F0020CC3D00209C7D0020BC250020AA
:101350003E3D0020C41F0020183D0020E6980020DC
:10136000503E0020002B3FF47FAF0B490B4A096829
:101370004FF47A7000FB0313136075E70F200D9292
:1013800010F0B2F9DBF8D0000D9A5DE400210320E3
:1013900026E70021022023E7D45D002064260020F8
:1013A0002DE9F047C74C636820469847002800F0B5
:1013B000C380C54B1B780122042B84F83C2000F02D
:1013C000BD80B4F91610B4F91820B4F91A302163AD
:1013D0006263A363BD4B1B88002B69D0BC4DD4ED69
:1013E0000C7AD5ED004A95ED050A95ED015A95ED7B
:1013F000067AD5ED035A95ED026AF8EEE76AD5ED67
:10140000047AA4EEA60AA5EE267A67EEC07AA5EEC7
:10141000C07AE6EE267A85ED057AC5ED067A2AF0E1
:1014200079FDD4ED0D6AD5ED094A95ED0E0A95EDDD
:101430000A5A95ED0F7AD5ED0D7AD5ED0C5A95ED4A
:101440000B6A2063F8EEE66AA4EEA60AA5EE267AF9
:1014500067EEC07AA5EEC07AE6EE267A85ED0E7AC2
:10146000C5ED0F7A2AF056FDD4ED0E6AD5ED124A7D
:1014700095ED170A95ED135A95ED187AD5ED167A74
:10148000D5ED155A95ED146A6063F8EEE66AA6EE9E
:10149000A40AA6EE857A67EEC07AA0EE657AE6EE3B
:1014A000867A85ED177AC5ED187A2AF033FDA063A8
:1014B000884FA17F884816F017F93B88002B40F031
:1014C0008480864ED6F8E450854B1B685B0743D476
:1014D000B5F90070216B636BA06B824A824E92ED6E
:1014E000026AD2ED006AD2ED015AC91B2163B5F937
:1014F0000270DB1B6363B5F904703568C01B07EE2F
:10150000900AB8EEE75A07EE901AB8EEE77A07EEBF
:10151000903AF8EEE77A36EE056A36EE877A77EE9D
:10152000A57A0135A06382ED026A82ED007AC2EDF0
:10153000017A3560BDE8F087BDE8F0876B4BB4F900
:101540001600B4F91810B4F91A20188020635980D5
:1015500061639A80A2633DE7B6F89820322A00F0D2
:101560008880002A66D196F89530002BB0D060486C
:10157000D6F800215F4980FB0273D217C2EB231219
:101580002A80D6F8042180FB0273D217C2EB231203
:101590006A80D6F80831A78A80FB0302DB17C3EB09
:1015A0002213DB1BAB800023CB6086F8953018F04C
:1015B0003DFCF7F7FFFC18F021FCFBF78DF801204C
:1015C00028F038FED6F8E45082E7444E226BD6F875
:1015D000E450B3F5C87F4FF0000323632B803988B4
:1015E00018BFD6F8E800B7F8008008BF0020B1F5B2
:1015F000C87F18BFD6F8EC30616B02440B44002062
:10160000B8F5C87F6063C6F8E820C6F8EC3068809B
:1016100052D0D4F838E0D6F8F010A0637144B8F195
:10162000010FA880C6F8F01068D008F1FF38A7F8BD
:10163000008049E7D6F80001236B00210344C6F877
:10164000003121632980D6F80401636B6163034490
:10165000C6F804316980A36BD6F80801A16303447E
:10166000012AC6F80831A98075D0013AA6F8982059
:1016700079E72B8820491F48276BA6F8F430002310
:10168000B5F802E0B5F804C0C0684B608B60236316
:10169000C6F800712B80616BC6F8041163636B8020
:1016A000A16BC6F80811A363A6F8F6E0A6F8F8C087
:1016B000C6F8FC00AB80D8E7A36BC6F8F030A06397
:1016C000A880B2E7386500208C7C00203E450020D1
:1016D00040450020E698002068650020C41F0020D7
:1016E000C07A0020E0270020DC270020907C00202A
:1016F0001F85EB517C950020C4200020DFF804C139
:10170000DFF8F0E0C8328CFB02A9C833D217C2EB75
:10171000E9128CFB03A9DB17C3EBE913C8316B801B
:101720002A808CFB013CA28ACB17C3EBEC139B1ADB
:10173000AB80CEF80C0018F079FBF7F73BFC18F003
:101740005DFBFAF7C9FF404628F074FDB7F800804A
:10175000D6F8E45069E7254B86F89A101B6886F89E
:10176000942013F4003334D119462148475C0B2FE1
:1017700001F10C0110D00133182BF7D1B6F8F41099
:101780001C4B2980B6F8F670B6F8F800D6F8FC10B5
:101790006F80A880D96068E7174FD7F800C059005C
:1017A000BCF1000F09D001EB030E00EB8E0E9CF88C
:1017B00001C09EF801E0E645E0D20B44DFF848E0C6
:1017C0000E4900EB830000233860AEF800300B6058
:1017D000D4E70B4B1B78032B01D00B46C5E728F051
:1017E000E7FBD6F8E450B6F89820C7E7444100205C
:1017F000A4E503087C950020B8240020B025002033
:10180000412F00201F85EB51AC2500202DE9F0472A
:101810008C4B1B78DB07074644D58B4B8B4D1C78D4
:101820008B4E012C59D01CD3022C07D189498A4AEE
:1018300009881288914201D901241C70EB7AE3B126
:101840002B89D3B1854B1B78BBB119F04DFD002816
:1018500000F09B802B7B83422CBF01210021317043
:101860000CE07C497E4A098810886A7B801A88428D
:10187000E2DAEB7A0024002BE2D131782A79632A6C
:1018800006D8022C774E00F0BA803378002B5DD159
:10189000754AAB7A8C4238BF0C461470002B4CD181
:1018A000BDE8F0876B4B694D19885B88E878CB1AE7
:1018B00083EAE3728142A2EBE3721DD32B788B4261
:1018C0001AD3614B1C78E01E012861D96749097859
:1018D00002294FD0012C5E4EA5D15F4A5D49128886
:1018E000687B0988121A914239DD5D4A12888A4262
:1018F000A4D200241C70A1E7B1EB400FE1DC524BF5
:101900001C78E11E012940F29480022ADEDC57494E
:101910004F4E0878DFF84481DFF844C1DFF838E142
:1019200000210324022834701C7088F80010ACF8E1
:101930000010AEF8001081D11FE0012C71D0022CF4
:101940000BD10720BDE8F04728F04EBB7068381A6D
:10195000474B984258DD72709AE7BDE8F087022441
:101960001C706BE7022AD2DD4049097802294FF04A
:10197000040464D13949364E09783E48022ACCBF66
:1019800000220122C28081804BE70221317075E77D
:10199000022A9BDC95F800C091FBFCFC0CF1010CC9
:1019A000BCF1080FDFF8B4A0304EA87895F801E03C
:1019B00096F800802A4CDFF8A090254EA8BF4FF083
:1019C000080C8AF800C01FFA8CFA10FB0AF01EFB04
:1019D0000AFE80B2DFF88CA02080A9F800E0002485
:1019E0004FF0640EB8F1020F34701C70CAF8044056
:1019F0008AF801E07FF439AF0FFA8CF1BDE7307857
:101A0000A0B9012377603370C2F164021A4B00FB66
:101A100002F083FB0023C017A0EBA350643070706A
:101A200036E70820BDE8F04728F0DEBA7368F81AF8
:101A30008EE7032C96D10D49097802299AD0044EDD
:101A4000FCE600BF644A0020004F00201C65002017
:101A5000104F0020847D0020044F00209A7D00203C
:101A6000024F0020084F0020412F00208C7C0020D6
:101A70007F969800907C00206BCA5F6B2DE9F04F39
:101A80002DED028B93B006461DF0CCFE9A4B1D78CF
:101A900025B113B0BDEC028BBDE8F08F974B1B68EE
:101AA0005C05F6D5964F3A68002A00F02181954CE6
:101AB000D4F8283103F5F43348339E42C0F018813E
:101AC000DFF8888294F82C31D8F80010C4F8286127
:101AD0000133DBB2880784F82C3101F1B88608079E
:101AE00000F1BE8113F0070901F06C85282B864BAD
:101AF000029301F0FA875E209047844B1B78002BFD
:101B00006BD0804C824AD4F83431F31A934201F2FC
:101B10001F84DFF83CA29AF80090B9F1000F33D18E
:101B2000DFF8FC81D8F80000FCF792F8C0B2012879
:101B30000ED90228774F42F095803B78002B42F077
:101B40006781D4F83C31F31AB3F57A6F82F00282E0
:101B500071480268002A40D09AF80030BBB96F4B38
:101B6000D8F800001B689B781E3B012B4FF0020148
:101B700042F2A38104301DF027FD012200238AF8E0
:101B8000002084F8483126E0634802682AB3D4F87C
:101B9000443140F6B731F31A8B421ED994F84031E4
:101BA000002B02F05580013BDBB284F84031002B62
:101BB00001F0BB8612F8011B94F84871026094F89A
:101BC00049315748CA190133006884F8482184F81C
:101BD0004931FCF741F8C4F84461524A029B12783B
:101BE0001B68012A03F101030A9301F0DB824E4BCB
:101BF0001B786BB14D4F3B6853B1029B414CD3F8FE
:101C000000B0D4F85C31ABEB0303632B01F2FF812E
:101C1000DFF8408198F80090B9F1020F01F05F867B
:101C20003C4F97F87430032B01F09584404B1B78A0
:101C300073B1404D2B685BB1324CFBF74BFDD4F8D0
:101C40006831039044F61F62C31A934200F25C812C
:101C5000394B1B78002B7FD1384B1B7843B1294C73
:101C6000D4F8B83203F50043E8339E4281F0108384
:101C7000334B1B78002B3FF40CAF224E314C324DCE
:101C800006F2C1272068FBF7E3FF00283FF401AF0D
:101C90002068FBF7D5FF2B7880465A1E33B12068A9
:101CA0002A70FBF7D5FF0028F2D1F2E6032239466D
:101CB000781E2BF0D0F896F8C03296F8C12286F83C
:101CC000C38283F47F4383F0FF039B1A1FFA88F8D3
:101CD0009BB2B8EB132FD5D196F8C222DBB29A4251
:101CE000D0D1781E21F06EFE2B7818442870C9E7F9
:101CF000054B029301E700BFD9420020C07A0020C3
:101D0000A4650020D0200020D45D0020366600208D
:101D10003F0D0300200000209C65002098650020F6
:101D2000946500203766002044660020146500207A
:101D30004C66002050660020746600207566002006
:101D4000566600205C660020606600202C6500203E
:101D5000A06500201C9300205E4C2278002A41F0F0
:101D600018825D4F3C78002C40F0A7805B4D2878AE
:101D7000002841F0CD875A4C5A4DD4F8B0122A7839
:101D8000594B93FBF2F30B449E42FFF465AF574A65
:101D900094F8B432C4F8B062D75CFA0702F1FF805D
:101DA000BB0702F1A381780702F166813A074CD59F
:101DB0004F4BDFF850810B930DF14809A3F13D0221
:101DC00049F8202D0021A3F1400203F8401C022312
:101DD0001121517093704846D8F80010F7F7C4FBF2
:101DE0004846D8F80410F7F7BFFBB8F80E30414961
:101DF00003EBC3039B00053381FB0321DB17C3EB1C
:101E0000A10189B24846F7F7C7FBB8F8103003EBD9
:101E10008303590089B24846F7F7BEFB364B1B785F
:101E20009B0743BFB8F8081001F57A7189B24FF4E7
:101E30007A714846F7F7B0FB0A9B98F81420591CB2
:101E40000A9148461A701DF0ADFC94F8B432297816
:101E5000013393FBF1F201FB123384F8B432FBE659
:101E600013F0030A7FF43EAE5E2090473B681420D7
:101E70009847224B1F4AB3F9043082FB03124FEA02
:101E8000E379C9EBA2090FFA89F95FFA89F01DF02D
:101E9000EFFBC9F307201DF0EBFB3B685E20984782
:101EA0003B681C20984750461DF0E2FB50461DF051
:101EB000DFFB94F82C313A6814E6114D286E0028A7
:101EC00041F0EE858146064B87F80090C3F8B0627A
:101ED000C2E600BF28660020F92F0020F82F00205E
:101EE000D020002000300020A0860100FC2F002020
:101EF000E865002067666666826500203065002020
:101F000008300020286B002094F86E31002B41F03F
:101F10002485DB4B1A6802F00803002B48F60341C6
:101F20004AF60B404BF60F4349F6074704BF0346FA
:101F30000F4612F0040F4FF0190118BF1F46930609
:101F400084F86E1103D547F4804747F0200719F055
:101F5000BDF9C7F30909002842F01681C94B9B79E6
:101F6000002B42F0F582984664204FF0FF3A4FF084
:101F7000000C0A970B97ADF834C0CDF83AC0CDF8F5
:101F80003EC0CDF842C0CDF83090ADF83680ADF807
:101F900038A08DF846000AAF0FCFDFF800E384F8D1
:101FA00005C0AEE80F0097E80F00AEE807002EF876
:101FB000023B71464FF0010C1B0CFE271F20C8226C
:101FC00001F81E39A770A27184F807C0E07094F878
:101FD0007E01207180F0F10383EA0313DAB2130962
:101FE00083F0E70343EA022383EAC2031BB283EAD6
:101FF0000312D2B2C3F3072383EA121343EA022384
:1020000083EAC2031BB283F0C80282EA0212D2B290
:10201000C3F3072383EA121343EA022383EAC203CA
:102020001BB283EA0C0787EA0717FFB2C3F3072244
:1020300082EA171242EA072200EB0C0382EAC70782
:102040000EEB0C0084F87E31278011F8013B7B40B9
:1020500083EA0313DBB21A0982EA172242EA032257
:1020600082EAC3031BB29FB281422780EDD183F085
:102070007C0383EA0313DBB24FEA131E8EEA172EAA
:102080008EEA032E8EEAC30E0FFA8EFE1FFA8EF929
:10209000DFF80CC2A4F800905FFA8EFE4FEA19290F
:1020A00084F8289084F827E00CF5D37804F1220A0C
:1020B000DCF80000DCF80410DCF80820DCF80C3058
:1020C00047460FC70CF1100CD445B846F0D1DCF8E8
:1020D000000038606C4F9CF8043088F8043007F139
:1020E000270884F8CDE184F8CE9117F8011F2868FD
:1020F000FBF7B2FDB845F8D194F86F31002B41F0F1
:1021000031846249029A097812680A2084F86F01C2
:10211000002901F0BE855E4F01293888069042F201
:102120000F820229B7F802E002F00181B888059019
:10213000032902F023820429B7F806B002F01982BD
:1021400038890490052902F010820629B7F80A9010
:1021500002F008820729B7F80C8000D0FB8994F8B8
:102160007E110A92084680F0300282EA0212D2B250
:1021700017094849079087F07A0747EA0227098834
:10218000207187EAC202444FC1EB012187FB010A9B
:1021900006984FF0000C60F30F0C05986EF31F4C7F
:1021A0004FF0000E60F30F0E0498CDF82CC012B261
:1021B0008A440027C917C1EB6A2A60F30F0782EA35
:1021C00002110020C9B268F30F00C2F3072269F3BD
:1021D0001F4782EA11126BF31F4E63F31F404FF04B
:1021E0000009CDF830E00D978DF83DA00E908DF8E8
:1021F0003C9042EA01220DF1280C82EAC107BCE8BA
:102200000F003FB287F0C80888EA0818DFF88CE0B2
:1022100084F805905FFA88F8C7F30727AEE80F0047
:1022200087EA181747EA08239CE8030083EAC803F3
:102230001BB283F023024EF8040B82EA0212D2B2E0
:10224000C3F30723079F83EA1213704643EA02236E
:1022500083EAC20207F1010C20F814194FF0230899
:102260001621FE27C82384F87EC1228084F80780C7
:10227000A7700EF1020EE170A371114612E000BFCB
:102280002C6500201C650020772200203898002053
:10229000809100203E2F002003082080D8200020BD
:1022A000D220002010F8013B4B4083EA0313DBB23D
:1022B0001A0982EA112242EA032282EAC3031BB20C
:1022C00099B270452180EDD183F0F40383EA0313C2
:1022D000DBB24FEA131E8EEA112E8EEA032E8EEA2F
:1022E000C30E0FFA8EFE1FFA8EF8CC4FA4F80080B2
:1022F0004FEA182C5FFA8EFE84F81EE084F81FC0A7
:102300007968BA683868FB6807F5D378A8E80F00E1
:1023100038697969BA6904F2A717A8E8070004F2D6
:10232000C51884F8C5C184F8C4E117F8011F2868EE
:10233000FBF792FCB845F8D194F87231002B41F0CC
:102340000783B74B1B681922980684F8722140F165
:102350000B83B44BDFF8DC821B78990741F11C86B4
:1023600098F81430042B8CBF03270227FBF7B2F92F
:10237000B8F81030B8F808200A9003EB83035B002C
:10238000ADF842304FF47A70D8F800300C93B8F8BA
:102390000E1098F814C0D8F804308DF8447000FB83
:1023A00002F24FF0000E4FF0FF300DF128098DF8CA
:1023B00045C0CDF82CE00E920D93ADF840100F9073
:1023C000CC46BCE80F00984F0FC79CE80F0007C72A
:1023D0003A46182122F81C39E17194F87E1184F8EC
:1023E00005E081F0780383EA0313D8B2030983F090
:1023F000F60343EA002383EAC0031BB283EA031017
:10240000C0B2C3F3072383EA101343EA002383EA2D
:10241000C0031BB283F0C80080EA001E5FFA8EFE84
:10242000C3F3072080EA1E1040EA0E2080EACE00A7
:1024300000B280F0180383EA0313DBB2C0F3072075
:1024400080EA131040EA032080EAC30301F1010C83
:102450001E204FF0FE0E4FF0C80AE07002372171C7
:1024600084F87EC1238084F802E084F806A0184630
:1024700012F8011B414081EA0111C9B20B0983EA3C
:10248000102343EA012383EAC10109B288B2BA42A8
:102490002080EDD181F0180181EA0111C9B24FEA23
:1024A000111B8BEA102B8BEA012B8BEAC10B0FFA65
:1024B0008BFB1FFA8BF3594A23805FFA8BFB1B0AB5
:1024C0000492059384F8273084F826B0964602F5E6
:1024D000D37C04F1220ADEF80000DEF80410DEF8F6
:1024E0000820DEF80C3067460FC70EF1100ED645F7
:1024F000BC46F0D14D4BDEF8000038601A4603F1BF
:10250000260A9DF8143084F8CCB184F8CD31934676
:1025100017461BF8011F2868FBF79EFBDA45F8D128
:10252000FBF7D8F8424BDFF810C1B3F90410B8F844
:1025300008E00A9098E80C008CFB010CC9174FF4D6
:102540007A704FF0000800FB0EF0C1EBAC01ADF863
:102550003C80ADF83E80ADF84080ADF842100D9063
:102560000E900B920C93CC46BCE80F00DFF8B8E05D
:1025700084F80580AEE80F009CE807004FF02108C2
:102580008EE807001C23C8224FF0FE0CE370A271F6
:1025900084F8078084F802C094F87E11217181F0DC
:1025A0006A0383EA0313DAB2130983F0D50343EA1B
:1025B000022383EAC2031BB283EA0312D2B2C3F33B
:1025C000072383EA121343EA022383EAC2031BB2FE
:1025D00083F0C80282EA0212D2B2C3F3072383EA6D
:1025E000121343EA022383EAC2031BB283EA0802FE
:1025F00082EA0210C0B2C3F3072282EA101242EA52
:102600000022013182EAC0020EF10C0E84F87E1124
:102610002280AEF11C01104610E000BFD220002045
:102620002C65002082650020D82000207722002021
:1026300030650020286B00206766666611F8013B54
:10264000434083EA0313DBB21A0982EA102242EA0A
:10265000032282EAC3031BB298B271452080EDD1F8
:1026600083F0680383EA0313DBB24FEA131B8BEAA0
:10267000102282EA032B8BEAC30B0FFA8BFB1FFAA3
:102680008BF3DFF800E423805FFA8BFB1B0A0593D2
:1026900084F8253084F824B00EF5D37A04F12208AA
:1026A000DEF80000DEF80410DEF80820DEF80C305A
:1026B000D446ACE80F000EF1100EC645E246EFD14D
:1026C000BEF80030ACF800309DF81430DFF8B88365
:1026D00084F8CAB1BA4684F8CB311AF8011F2868C9
:1026E000FBF7BAFAD045F8D194F87EA1E14A84F814
:1026F00004A08AF0EB0383EA0313D9B20B0983F039
:10270000C50343EA012383EAC1031BB283EA031032
:10271000C0B2C3F3072181EA101141EA002181EA26
:10272000C00109B20CCA81F0C80C8CEA0C1C5FFA1B
:102730008CFC4FF0000EC1F307210B93CDF830E075
:1027400081EA1C130A9299E8070043EA0C2383EA02
:10275000CC03BB461BB2C84F84F805E083F0310CB4
:1027600087E807008CEA0C1C5FFA8CFCC3F3072394
:1027700083EA1C1343EA0C2383EACC0394F808C0D1
:10278000607AA17AE27A94F80CE094F811801BB296
:102790008CEA030C8CEA0C1C5FFA8CFCC3F3072355
:1027A00083EA1C1343EA0C2383EACC031BB2584090
:1027B00080EA0010C0B2C3F3072383EA101343EA90
:1027C000002383EAC0031BB2594081EA0110C0B262
:1027D000C3F3072181EA101141EA002181EAC00117
:1027E00009B24A4082EA0212D2B2C1F3072383EA55
:1027F000121343EA022383EAC2031BB28EEA030EDA
:102800008EEA0E1E5FFA8EFEC3F3072383EA1E13C1
:1028100043EA0E23607BA17BE27B94F810C083EA3D
:10282000CE031BB2584080EA0010C0B2C3F30723A6
:1028300083EA101343EA002383EAC0031BB2594022
:1028400081EA0111C9B2C3F3072383EA111343EAF2
:10285000012383EAC1031BB25A4082EA0212D2B2B8
:10286000C3F3072383EA121343EA022383EAC20372
:102870001BB28CEA030C8CEA0C1C5FFA8CFCC3F3D1
:10288000072383EA1C1343EA0C2383EACC031BB21D
:1028900088EA030888EA08185FFA88F8C3F3072370
:1028A00083EA181343EA082383EAC803A17CE27C85
:1028B0001BB2594081EA0111C9B2C3F3072383EA6D
:1028C000111343EA012383EAC1031BB25A4082EA8F
:1028D0000212D2B2C3F3072383EA121343EA02239C
:1028E00083EAC2031BB283F0270989EA0912D2B234
:1028F000C3F3072989EA121949EA022989EAC209B8
:102900000FFA89F90AF101031FFA89F231205FFAFF
:1029100089F94FF0FE0C0C2184F87E31C8234FEA70
:10292000122E07F5D0782280E07184F802C0E170A1
:10293000A37184F81490049F84F815E07968BA684C
:10294000FB683868B7F810C0A8E80F005F4628F8A1
:1029500003CB84F8BBE184F8BA9117F8011F28680B
:10296000FBF77AF9B845F8D194F87671002F40F06A
:10297000EA87424B94F87EC1B3F90010B3F9022004
:10298000B3F904309FED3E6A677107EE103A029B7F
:102990001B680A938CF06A0383EA031306EE901A0D
:1029A000D9B20B0983F0D50343EA012383EAC103BB
:1029B0001BB283EA03115242C9B207EE902AC3F355
:1029C000072383EA111343EA0123F8EEE77AF8EECE
:1029D000E66AB8EEC77A83EAC1031BB267EE867A6D
:1029E00066EE866A27EE067A002083F0C808CDEDF1
:1029F0000C7ACDED0B6A8DED0D7A0E900F90109044
:102A000088EA081E0DF128095FFA8EFEC3F3072835
:102A1000B9E80F0088EA1E1848EA0E2888EACE08AE
:102A2000DFF854E00FFA88F8AEE80F0088F01E07D0
:102A300099E8070087EA0717FFB2C8F3072383EA7C
:102A4000171343EA07238EE8070083EAC707C82164
:102A50004FF005094FF01E08FE231C200CF1010267
:102A600084F8769184F80780A370E070A171AEF1CC
:102A700010010BE0143D0020D8200020306500201C
:102A800088C3E43AD22000209B22002084F804C0AE
:102A90000EF10C0E278084F87E2111F8013B7B405B
:102AA00083EA0313DBB21A0982EA172242EA0322FD
:102AB00082EAC3031BB29FB271452780EDD183F038
:102AC000270383EA0313DBB24FEA131E8EEA172EA5
:102AD0008EEA032E8EEAC30E0FFA8EFE1FFA8EF9CF
:102AE000DFF8DCC3A4F800905FFA8EFE4FEA1929E4
:102AF00084F8259084F824E00CF5D37804F1220AB8
:102B0000DCF80000DCF80410DCF80820DCF80C30FD
:102B100047460FC70CF1100CD445B846F0D1E04F32
:102B2000BCF80030A8F8003007F1240884F8CAE1A6
:102B300084F8CB9117F8011F2868FBF78DF8B8458A
:102B4000F8D194F877B1BBF1000F40F0F686D54B81
:102B50001B68052284F877219A0641F19480D24BB4
:102B6000DFEDD26ADA891B8907EE902A07EE103A68
:102B7000F8EEE77AB8EE477A67EEA67A94F87E81A7
:102B8000CB4BCC4AB3F90410B2F90620CA4FCB485C
:102B9000CDED0B7A88F0220383EA03135FFA83FEFC
:102BA0004FEA1E1383F0590343EA0E2383EACE0350
:102BB000B2F5FA6F1BB2A8BF4FF4FA6283EA031EA4
:102BC0005FFA8EFEB2F57A7FC3F3072383EA1E1302
:102BD000B8BF4FF47A724FF0640C43EA0E23A2F5AB
:102BE0007A720CFB02F283EACE0E87FB02C780FBEF
:102BF00001C00FFA8EFEC917D217C2EBA7124FF011
:102C0000000AC1EBA0038EF0C8070DF128098DED75
:102C10000C7AADF83A20ADF83830CDF828A0CDF8D0
:102C200034A0CC4687EA0717BCE80F00FFB2CEF30A
:102C3000072E8EEA171E4EEA072E8EEAC707DFF828
:102C400094E2DCF800C084F80480AEE80F003FB2E4
:102C500087F04A0383EA0313DBB2C7F3072181EA53
:102C60001311724641EA032108F1010881EAC30306
:102C7000142042F810C9FE274FF04A0C002184F8B6
:102C80007E814FF0C808E07023800EF1040E84F8B6
:102C900007C0A770617184F80680184612F8011BFE
:102CA000414081EA0111C9B20B0983EA102343EACA
:102CB000012383EAC10109B288B272452080EDD1B7
:102CC00081F0140181EA0111C9B24FEA111E8EEAA6
:102CD000102E8EEA012E8EEAC10E794B0FFA8EFE6F
:102CE0001FFA8EFC1F464FEA1C2A5FFA8EFE84F8FC
:102CF0001DA084F81CE0596838689A68DB68A4F85D
:102D000000C007F5D37CACE80F0038697969B7F8E3
:102D100018800497ACE8030004F2A717ACF8008011
:102D200084F8C3A1B84684F8C2E104F2C31A18F8C3
:102D3000011F2868FAF790FFC245F8D1614B624A3B
:102D40001B781278013B12F00100DBB214BFC021E6
:102D50004021172B03D85D4A134493F814B05C4B01
:102D60001A8893071ABF002341F01001012312F4BF
:102D7000027F18BF022312F0100F18BF062312F0B3
:102D8000200F18BF1023002841F0D4804FF0030813
:102D900094F87EE10A938EF0460383EA0313DAB2D5
:102DA000130983F0920343EA022383EAC2031BB2AE
:102DB00083EA0310C0B2C3F3072282EA101242EA88
:102DC000002282EAC00212B282F0C80C8CEA0C1C0B
:102DD00000235FFA8CFC0320C2F307228DF82CB08D
:102DE0008DF82F8082EA1C128DF82D308DF82E1070
:102DF0008DF8300042EA0C2899E8070088EACC0CEC
:102E00000FFA8CFCDFF8CC80E3718CEA0C19A8E88F
:102E100003005FFA89F9CCF3072C8CEA191C4CEA01
:102E2000092181EAC90994F808C088F800200FFA3E
:102E300089F98CEA090C8CEA0C1C5FFA8CFCC9F34A
:102E4000072282EA1C1242EA0C22607AA17A94F8E4
:102E50000B90637182EACC0C0FFA8CFC80EA0C00B8
:102E600080EA0012D2B2CCF3072080EA121040EAC6
:102E7000022080EAC20000B2414081EA0111C9B2D9
:102E8000C0F3072282EA111242EA012282EAC10259
:102E900012B289EA020989EA09195FFA89F91BE085
:102EA000772200202C650020286B00200AD7233CC5
:102EB0003065002080910020D34D62106766666601
:102EC000D2200020D8490020644A0020BCD003084A
:102ED00080650020D8200020C2F3072282EA191260
:102EE00042EA092294F80CC0607BA17B84F804E0DC
:102EF00082EAC90212B28CEA020C8CEA0C1C5FFA5C
:102F00008CFCC2F3072282EA1C1242EA0C2282EAFB
:102F1000CC0212B2504080EA0010C0B2C2F30722C5
:102F200082EA101242EA002282EAC00212B2514042
:102F300081EA0111C9B2C2F3072282EA111242EA00
:102F4000012282EAC102E17B94F8109013B281EA77
:102F5000030282EA0212D2B2C3F3072383EA1213F6
:102F600043EA022383EAC2031BB289EA030282EA2C
:102F70000212D2B2C3F3072383EA121343EA0223F5
:102F800083EAC2031BB283F0320282EA0212D2B297
:102F9000C3F3072383EA121343EA022383EAC2033B
:102FA0001BB29AB24FF0FE0C5FFA83FB0920C821D6
:102FB0000EF1010E84F802C04FEA122CE070A171EC
:102FC00084F87EE1228084F812C084F811B0049B5A
:102FD000186859689A68B3F80CA008F5CC7EAEE87A
:102FE000070008F5D4788EF80290AEF800A084F8B7
:102FF000B8C184F8B7B117F8011F2868FAF72CFE9A
:10300000B845F8D1039BC4F86831FEF721BEDFF85C
:1030100028A3DFF82883DFF8289341201BF05AFF0C
:10302000BAF9023088FB0320DB17C3EBA00080B2A3
:103030001BF034FFBAF9003088FB0320DB17C3EB29
:10304000A00080B21BF02AFFBAF9043088FB0320ED
:10305000DB17C3EBA00080B21BF020FF99F8001033
:103060003868FAF7F9FD94F860A11AF0010800F049
:10307000A184A44B1B689A067AD5A34BDFF8C482BF
:103080001B789B0740F11D8798F81430042B8CBFE8
:103090004FF0030A4FF0020A47201BF01BFFD8F83D
:1030A00000001BF0C7FED8F804001BF0C3FEB8F800
:1030B0000E30964A3868A2FB0323C3F34713194620
:1030C0000393FAF7C9FDB8F8082099F80010039B9C
:1030D00064204B4000FB02F089F800301BF0AAFE90
:1030E00098F8148038684AEA88085FFA88F84146F8
:1030F000FAF7B2FD99F80030386888EA03084146CB
:1031000089F80080FAF7A8FD94F860A1BAF1000FE1
:103110002ED1DFF834824F201BF0DCFED8F80000FF
:103120001BF088FED8F804001BF084FE50461BF00C
:1031300081FE01213868FAF78FFD734A99F8003053
:1031400092F80080386808F0010883F001034146D6
:1031500089F80030FAF780FD99F80030386888EA7D
:103160000303194689F80030FAF776FD94F860A158
:10317000674AC4F85CB10AF10103DBB2A2FB031297
:10318000D20802EB8202A3EB420384F86031FEF71F
:103190003FBD604B60491868FAF726FD0023237095
:1031A000FEF7DFBD5D4F386800283EF420AD4FF0DC
:1031B000000ADFF898815A4CAB465546FAF748FDAD
:1031C000F8B1F5B94FF00109AA463868FAF738FDA9
:1031D00083B27E2B00F09A8398F80120002A49D10F
:1031E00094F84C11B1B11B2B84F84C2100F066838C
:1031F0000D2B45D0386888F80190FAF729FD002892
:10320000E3D1AA4650460AAA46495D461BF07CFE19
:10321000FEF7EDBC7D2B00F0468594F8502122B1DD
:1032200080F02003DBB284F8501194F84B21062A79
:1032300010D8B4F84E1138681944A4F84E11A118EA
:10324000013281F8543184F84B21FAF701FD00284E
:10325000BBD1D6E7B4F84E2188F8019013449BB255
:103260001A0A52FA83F3FF2BA4F84E31386802D1C0
:103270002D4DA3E73868FAF7EBFC0028A5D1C0E78D
:103280003868A4F84E21FAF7E3FC00289DD1B8E78E
:1032900094F8BC32C4F8B862012B40F2DD8494F893
:1032A000BD222249981801EB8001013202F001028F
:1032B000CF6A84F8BD22BFB11D4D0B950DF14809B1
:1032C000123DA52349F8205D802284F81031152392
:1032D0003146484684F8112184F81231B847002855
:1032E00040F03B8494F8BC32124A013382FB031253
:1032F000A2EBE37202EB42029B1A84F8BC32FEF7A7
:10330000B7BC00BF2C650020826500201F85EB51F3
:10331000CDCCCCCCF42F0020E865002090650020B7
:10332000D02000201A22002024220020BCD0030834
:10333000F5210020565555553065002067666666B4
:1033400018650020286B0020143D0020200000207C
:103350008B4A8C4B92F80BC0029A1B881168D4F8E8
:103360003801894A5FFA83FE1F0A4FF47A73091AFB
:1033700003FB0CF30020994282F81EE0D77782F815
:1033800014E057759070107180F052847F49DFF817
:103390001CE20B688F687E49DFF81482087898F881
:1033A00014908EFB03C1DB17C3EBA1018EFB07CE8C
:1033B0001177FF170912C7EBAE075177F4214FEAD7
:1033C000272E82F82070917601273021D77682F857
:1033D0002210704B82F821E07527782182F8237043
:1033E00082F82410820783F81A9040F11E84D8F8DE
:1033F00000E0694AD8F80470DFF8B8B1DFF8B8C166
:1034000082FB0E1A4FEAEE7082FB0712C0EBAA5045
:10341000F917C1EBA2510BFB00E202EB4202520092
:103420000BFB017B00EB8000049201EB810100EBC0
:1034300080000BEB4B0B4FEA4B0B059001EB81002F
:10344000049907908CFB022A8CFB0B2C4FEAAC42B0
:103450004FEAAA4AC9174FEADE7E069283F809E0CE
:103460004E4AB8F80EC0B8F80880AAEB010E0499CD
:10347000F24602FB1A1A05994FFA8EFE0EEB810EE8
:1034800006994FEAEB7008F5FA780A1A1FFA88F8DD
:10349000FF0F4249CDF80C8010469F730CEBCC0C0B
:1034A000079FDFF8188101FB12B24FEA8C0C3C49F0
:1034B00040B200EB870088FB0C789DF80C705F75BC
:1034C0004FEAEC7CCCEBA81C81FB0A7881FB0271F3
:1034D000D217B9F1050FC2EB6112DFF8E49003993E
:1034E000B9F800B05A744FEAEA7ACAEB681A1FFAC0
:1034F0008EFE80B24FEA11282A4983F80AE04FEA8B
:103500001E294FEA102E4FEA2A2783F80CA00988BB
:1035100083F80B90D87383F810E04FEA2229CCF39C
:1035200007204FEA1B2E34BF4FF0320A4FF0330A08
:103530005F7383F8129083F8168083F807C01872BF
:1035400083F813B083F814E083F81BA01977C4F84C
:103550003461FEF7DEBA144B03931868FAF768FB80
:1035600000283EF463AB039B01211868FAF75CFB6B
:103570000222002387F8742088F80030FEF756BB3B
:103580008C7D0020847D00209C2F0020586300202B
:1035900082650020C82F00206BCA5F6B40420F007D
:1035A0001F85EB51803D0020744D002067666666E4
:1035B000286B0020806967FF83DE1B43D34D6210B8
:1035C0008C6500205E2090473B6802209847FF20D2
:1035D00020F07AF90378FF2B00F06C8490F9013029
:1035E0004FEAE3795FFA89F9D8B21CF041F848460E
:1035F0001CF03EF83B685E2098473B6803209847E4
:10360000FF2020F061F90378FF2B00F00784B0F968
:103610000830D8B2C3F307291CF02AF848461CF03A
:1036200027F8D34B1B78042B75D0DFF86CB3B4F8B4
:103630002E319BF80010DFF864A393FBF1F201FB3D
:10364000123292B2BAF80030A4F82E21120164208E
:1036500092B200FB03134900B3FBF1F342EA0329E2
:103660005E20C3F303221FFA89F93B6849EA020985
:1036700098473B68062098475FFA89F01BF0F8FFEF
:103680004FEA19201BF0F4FFBA49B4F82E214B7A07
:10369000BAF800900132012BA4F82E2100F05F86C9
:1036A0004A7B09EB89031FFA83F9002A40F04C8416
:1036B0003B685E2098473B683A209847AE4BA3FB97
:1036C00009234FEA531A1FFA8AFB5FFA8BF01BF0AB
:1036D000CFFF4FEA1B201BF0CBFF3B685E209847D3
:1036E0003B683B209847642303FB1A939BB2A34893
:1036F000053380FB0320DB17C3EBA000C0B21BF037
:10370000B7FF00201BF0B4FFDFF8949299F8063061
:10371000002B40F0DA83D8F80030990640F1B381ED
:10372000DFF8809299F800309A0700F17C83DFF887
:1037300078824FF0000BDA463B685E2098473B6882
:103740000120984750461BF093FF58461BF090FF0E
:103750003B685E2098473B680920984700201BF093
:1037600087FF00201BF084FFB8F8123098F814B0DF
:10377000B3F5967F0AD994F82C2102F00F02072A9C
:1037800004D842F20F7B9B4528BF9B463B68DFF87D
:10379000E4A15E2098473B68052098479AF80830D6
:1037A000002B00F0E784ABF1200307EE903A9FED89
:1037B000747AF8EEE77AF6EE006A67EE877ABEEE84
:1037C000007AF5EEC07AF1EE10FA58BFB0EE667AE4
:1037D00077EE877AFDEEE77ACDED027ABDF908B093
:1037E0005FFA8BF01BF044FFCBF307201BF040FF88
:1037F00099F80020002390070893099300F1FD82B7
:1038000094F83031012B00F0F882BAF90030DFED86
:103810005D6A07EE103ABAF9023007EE903AB8EE58
:10382000C77AF8EEE77A27EE267A67EEA67ABDEE3B
:10383000C77AFDEEE77A0AA88DED0A7ACDED0B7A0C
:103840001BF038FF94F82C313A68FEF74FB9DFF8D7
:103850005C919FED4D8A4FF0240B5E2090475846B7
:103860003B689847494BF9EC016A9B8A07EE103A8E
:10387000F8EEE66AB8EEC77A0BF1010BC6EE877A6E
:103880005FFA8BFB67EE887AFDEEE77ACDED027A80
:10389000BDF908A05FFA8AF01BF0EAFECAF3072020
:1038A0001BF0E6FEBBF1270F01D03A68D5E794F88C
:1038B0002C31D8F800103A68FEF711B93868FAF7D9
:1038C000C7F900287FF496AC386884F84A9188F8E4
:1038D0000190FAF7BDF900287FF477AC91E4F9F78D
:1038E000F9FE2B4B1B68A0EB030A40F6B8339A4550
:1038F00000F2BE81DFF8B8B09BF804303A2B00F03C
:103900005B84002388F80030FEF790B9386884F8AB
:103910004AA184F84BA184F84C9188F801A0FAF7E9
:1039200097F900287FF451AC6BE494F8481194F8AF
:10393000493118484A1CFEF746B90BF1FF3B84F8A1
:1039400077B1FFF75FBB013F84F87671FFF7F9B8F5
:10395000013B84F87231FFF707B8013B84F86E3100
:10396000FEF7CABB013B84F86F31FEF7E5BC00BF30
:10397000412F00208C7D00201F85EB516766666615
:10398000E4380E3F0050C34700007A4438650020F9
:1039900024930020946500209A7D0020847D0020DF
:1039A0001C65002082650020286B002068650020CF
:1039B0000C930020C54B1B88D80515D4D90600F1FF
:1039C000B6829A0600F1BA84580600F1E684190717
:1039D00000F1E784DA0700F1248513F0020F0CBF31
:1039E0004FF004084FF00C08B94BBA4A1B78D27854
:1039F00003F001030AB143F00203532003931BF0C9
:103A000069FAB54A128802EB820202EB8202900048
:103A100080B21BF043FA00201BF040FAAF49B04AD5
:103A2000B1F800A03868CAEBCA1A4FEA4A0A82FB0A
:103A30000A3252444FEAEA7ACAEB622A5FFA8AFAF9
:103A40005146FAF709F999F80020039B386848EACB
:103A500003088AEA020A002189F800A0FAF7FCF8B4
:103A600041463868FAF7F8F899F80030386888EA7B
:103A70000303DBB2194689F80030FAF7EDF894F841
:103A800060A1FFF743BB19077FF5DCAE954B93E8C8
:103A900003000AAB83E8030018461BF00BFED1E6D7
:103AA0000024DFF86482A1464FF0500A02E0DBB246
:103AB00083F3118815F804B0601C594628441BF0A4
:103AC000C1F8002840F0F9800BF101031C44EFF32A
:103AD00011838AF312882A6E9442E8DB0022DBB25B
:103AE0002A6683F31188FEF7EEB94FF0000A5E20D4
:103AF000D3F8008084F82CA190473B68DFF80C9243
:103B00001720984750461BF0B3FD774BA3FB0823C3
:103B10009B0BA9FB03125209C2EB0212A3EB820317
:103B2000D8B21BF0A5FD3B685E2098473B68182083
:103B300098476E4BA3FB08239B09A9FB031252096C
:103B4000C2EB0212A3EB8203D8B21BF091FD5046E8
:103B50001BF08EFD3A68FDF7CEBF0A9EAE424FF0D5
:103B600000014FD941F2210015F8013B81EA0323FE
:103B70005A0013F4004F80EA020192B289B208BFE2
:103B800011464B0011F4004F80EA03029BB292B23F
:103B900008BF1A46530012F4004F80EA03019BB29B
:103BA00089B208BF19464B0011F4004F80EA0302A6
:103BB0009BB292B208BF1A46530012F4004F80EA3B
:103BC00003019BB289B208BF19464A0080EA02038A
:103BD00011F4004F99B293B218BF0B46590013F479
:103BE000004F80EA010289B292B208BF0A46530030
:103BF00080EA030112F4004F9BB289B208BF194654
:103C0000B542B1D14846F5F7EDFC39490A9D39482E
:103C10006D1A152DA8BF15252A4628F03BF8364AFF
:103C200094F8BC321570FFF75FBB2D22DA768EE474
:103C3000324B02991B780968C4F83811013B012BFB
:103C40003FF6A4AB1021022391701371FFF79EBBC6
:103C50001BF0F0FCFDF7BFBF224A02EB8302D76ADC
:103C6000FFF729BB1BF0D6FC01233B70FDF770BFAB
:103C7000234AB2F8623100210133A2F8623188F898
:103C80000010FDF7D3BFDFED1F7AB0EE677AFEF7C5
:103C900075BF8846894604918B4605918E460691EC
:103CA0000B46FEF75CBA386884F85091F9F7D0FFFC
:103CB00000287FF48AAAFFF7A4BA41463A201FF0F1
:103CC0000BFF40EA09095FFA89F9FDE680650020EB
:103CD000644A0020442F0020847D00203E2F0020D5
:103CE00003082080BCD0030873B2E745D34D6210AF
:103CF000E0210020344B0020494B0020412F0020C0
:103D0000D020002000000000D9F7020889888888A8
:103D1000C949CA4B0093A1F13F07C94BC94A099150
:103D200001F8404C0AA8C8490897F5F733FD089FE9
:103D30007B1C08933C70089B2922591C08911A701F
:103D4000089BEA22591C08911A70089BC822591C2A
:103D500008910AA81A7027F05FF800F101080AA973
:103D60004246089827F096FF089A02EB08030133B1
:103D7000089302F80840089B5A1C08921C70089B84
:103D80005A1C08921C70089B5A1C08921C70089BB5
:103D90005A1C08921C70089B5A1C08921C70089BA5
:103DA0005A1C08921C70089B5A1C08921C70089B95
:103DB0005A1C08921C70089B5A1C08921C70089B85
:103DC0005A1C08921C70089B5A1C08921C70089B75
:103DD0005A1C08921C70089B0122991812A808917D
:103DE0001A7050F8283DDB1B3B701BF0DBFC974B37
:103DF0002C70C3F8B062FDF72FBF98E80C000121CA
:103E000008A884F83011089209931BF053FC19E5B7
:103E1000C4F83C6187F80090FDF79ABE4FF00009A6
:103E20004846FFF7F9BBDFF83C823B68DFF838B261
:103E30005E2098473B6811209847B8F80E304FF441
:103E4000F36A0AFB03F38BFB032BDB17C3EB6B3B20
:103E50005FFA8BF01BF00CFCCBF307201BF008FC87
:103E60003B685E20984719203B689847B8F80E30A9
:103E7000774A0AFB03F382FB0301DB17C3EB6113F1
:103E800082FB0321DA17C2EB6112642101FB1233BA
:103E9000D8B21BF0EDFB00201BF0EAFB99F80030D4
:103EA000B8F808B09B077FF544AC5FFA8BFA4FEA8D
:103EB0001B2B41E44846FFF798BBF9F7B5FEFDF729
:103EC0005CBE4FF0010AFFF7E7B83B68DFF89CA142
:103ED000DFF89CB15E2098473B6828209847DAF8C5
:103EE00000308BFB032BDB17C3EBAB0B5FFA8BF0C4
:103EF0001BF0BEFBCBF307201BF0BAFB3B685E2038
:103F000098473B6804209847B9F80830002B40F0E8
:103F10001982DAF8083083F310095FFA89F01BF090
:103F2000A7FBC9F307201BF0A3FBFFF7F4BB4FF07F
:103F3000340859E5474AD278002A0CBF4FF00408EC
:103F40004FF00508FEF724BF9BF8003099FBF3F90A
:103F5000FFF7AEBB0123D8F800003B70F9F770FE05
:103F60000746D8F80000F9F76BFE7B067DF4F0AD4C
:103F70008A2800F041828E287DF4EAAD9AF800305C
:103F8000002B7DF401AE3448344B03602D2384F8BC
:103F900040310268FDF7E0BD0127FEF7E7B9DFF821
:103FA000D4909FED2F8AB9F90230234A0B9207EE85
:103FB000903AF8EEE77A0DF1480867EE887AA2F1B8
:103FC0004003FDEEE77AA2F13D0148F8201D02F81A
:103FD000400C0822CDED027A5A701E229A70BDF86C
:103FE00008104046F5F7D8FAB9F9003007EE903AD4
:103FF000F8EEE77A404667EE887AFDEEE77ACDED97
:10400000027ABDF80810F5F7C7FAB9F9043007EEDF
:10401000903AF8EEE77A404667EE887AFDEEE77A66
:10402000CDED027ABDF80810F5F7B6FA40461BF060
:10403000B9FBFDF7B5BE00BFE86500200B98002076
:1040400058010408600104086C010408D020002015
:104050001F85EB51442F00209C6500209C2F0020E1
:1040600058A08B41286B002089B5F81458630020B4
:104070006766666630650020CC4ACD4B12680B93AC
:104080000021A3F1400903F8401C2123D10089F845
:10409000023040F17481C7494FF00308C64B1B88BA
:1040A0005A0500F15881D80700F1B78103F00203E7
:1040B000C24A002B1CBF4FF003081146DFF82CA3A7
:1040C0004246504627F0E6FD08EB0A0312A80133EA
:1040D000AAF1020140F8203D00225B1A08F80A20EC
:1040E00089F801301BF05EFBFDF760BEB04AB44BAF
:1040F0000B920DF14808A2F13D0048F8200D1988F7
:10410000DFF8C892A2F1400300204FF00A0E02F837
:10411000400C082283F801E040469A70F5F73CFA1B
:10412000D9F80030A749DA1781FB0313C2EBA303C8
:1041300099B24046F5F730FA17F0D6F8D9F808905A
:104140000A9B4FEA1942591C0A911A700A9B4FEABE
:104150001922591C0A911A700A9B5A1C0A9283F858
:1041600000900A9B5A1C0A92187040461BF01AFBDA
:10417000FDF719BE5FFA8BF01BF07AFA4FEA1B20AD
:104180001BF076FAFFF734BB8D4B8F4A1B88927970
:1041900003EB830303EB83034FEA83081FFA88F8DA
:1041A000002A00F04281894B1B680FFA83FA17F04E
:1041B0009BF840B2FDF7DBBE9BF80210584621F099
:1041C00099FA00287FF49DAB7D4A814F7F4B12887E
:1041D000FA61804C1A688049FA627F4A03919B68B1
:1041E000B4F86211F863C7F86CA01068FB64F96555
:1041F000F7F70AFF824600287DF413AD764B494657
:104200001868F9F711FD94F864319BF803200492C3
:10421000642B4FF0040287F8742040F0098194F871
:104220006531DFF8CCB1072B08BF84F865A194F89D
:104230006531079307EB0319D9F804100691084676
:1042400026F0EAFDD9F8083005935FFA80F91846A0
:1042500026F0E2FD5FFA80FA079B069909EB0A0255
:1042600008320AEBC9008BF8072023F00F0203F095
:104270000F038BF80A208BF80D304A468BF80E009E
:104280000BF10F0027F006FD0BF1060309F1090001
:1042900018445246059927F0FDFC9BF8073003F1BE
:1042A0000109D3B1013B5FFA83FC0CF1080CDFF884
:1042B00044E1DC440BF10700002310F8012B5A40C5
:1042C0009300D10883EA420301F0180153404EFAEB
:1042D00001F253408445DBB2EFD1404A049809F81B
:1042E000023027F0B3FC94F865310022013384F8E2
:1042F000653184F864219BF802305BB1039B1BF8A5
:1043000005101868F9F7A8FC01359BF80230EDB2EA
:10431000AB42F3D894F864310322013384F864315A
:1043200087F8742088F80020039BFFF716B9984699
:10433000994604939B460593FDF711BF4FF024085F
:10434000FFF752BB16F0D0FF1BF092F900201BF0D4
:104350008FF9FFF7E0B94FF003082149AEE63B685B
:104360005E2098473B68392098475FFA89F01BF038
:104370007FF94FEA19201BF07BF9FFF7C5B9194BFC
:104380000C4A1B68184903F48003002B16BF114622
:104390004FF004084FF0030880E64FF01008FFF7D5
:1043A00023BB4FF02008FFF71FBB00BF3095002054
:1043B000E8650020440104088065002054010408D9
:1043C000847D0020676666661C65002058630020B7
:1043D00020000020D0200020744D0020466B0020DB
:1043E00048010408C07A00203C010408AB650020A5
:1043F000406B00200007090E634B1B6899067DF592
:10440000A7AB9AF80030002B7DF4BEAB5F48604B41
:1044100003602D2384F84031BBE55E494FF004086A
:104420004CE64FF00808FFF7DFBA4FF0FF33BCE669
:1044300097F87590DFF870B119F00F0F04BF09F10C
:1044400001095FFA89F9B9F1070F28BF4FF0010997
:104450004FEA091A07EB0A035FFA8AFC187C4E4BF5
:104460001A180023117A8BF80A300BF10D0307EBB1
:104470000A024CEA000001291870D26803F1010E0B
:104480000CD90239C9B2881C1844734603F8012BB1
:1044900083424FEA1222F9D101318E44BA4422F00C
:1044A000600309F101099AF811205FFA89F91343B1
:1044B000B9F1080F8EF800300EF101034FD04FEA2A
:1044C000091A07EB0A01354A087C334901449A1A54
:1044D000097A02EB010E0CF1100CBEF1130F5FFA1A
:1044E0008CFCC4DDD2B2931DDBB243F040018BF8EB
:1044F000071003F1010CDFF8B4E0CBB105325FFA2D
:1045000082FA0AF1080ADA440EF10100002310F8D9
:10451000011B59408B0083EA4103CA084B402049E4
:1045200002F0180241FA02F253408245DBB2EED1AA
:1045300004980CF80E3087F8759027F087FBDAE6C0
:104540009846994604939B4605939E46FDF707BE01
:10455000144B8046B3F900A06420FDF708BD0F4A54
:104560009A1ABFE79846FDF7FABD98469946FDF7B7
:10457000F6BD984699460493FDF7F1BD98469946D5
:1045800004939B46FDF7EBBD2C6500209C65002045
:10459000C82F00204C010408BCD003084D6B00203C
:1045A0000007090E58630020406B0020466B002076
:1045B0002DE9F04F2DED0C8BDFF8F4B097B0DBF860
:1045C0000420079058469047002800F08C82BBF8E2
:1045D000A87000218BF85110002F6DD1BBF93A0063
:1045E000DBF82450DBF82810BBF93860DBF82040FA
:1045F000BBF93C20DFF8BCA0401B521ACBF83000BE
:104600009BF85210CBF83420341B0BF12C00CBF864
:104610002C4013F069F8DAF80020910042F117807D
:10462000DBED0C5A1F4CDBED0B7A1F4994ED406A11
:10463000D4ED416A94ED427AD4F80C2109681B4B01
:104640000593B8EEE58ADBED0D5AF8EEE77AF8EE61
:10465000E58A013277EE867A38EE268A78EE878A06
:104660008A42C4ED407A84ED418AC4ED428AC4F89E
:104670000C2101F06A8393F800E0BEF1140F03F0FF
:104680001A800023D4F814510693062D01F2BB843E
:10469000DFE815F0FE16EB16A6158216260CC017DD
:1046A000081600BF94230020B44500208C7C002015
:1046B000D4720020C07A0020D84BD9481A680893D9
:1046C0004FF47A76B6FBF2F2C2EB421602EB8602A8
:1046D000D600D44BDFF8A48344780593B6B2B74232
:1046E0001D78B8F9060003F04081DBF87C30BBF997
:1046F0003810DBF8602003F1010E07EE901A0A442F
:10470000BEF1010FCBF87CE0CBF86020F8EEE77A41
:1047100003F03881DBED1B5ADBED1D6A07EE10EA72
:1047200037EEE56AB8EEC75A012F86EE057A37EE06
:10473000257A77EEC77A8BED1C7AE7EE866A8BEDE9
:104740001B7AF0EE667ACBED1E6ACBED1D6A03F0A4
:104750003385DBF89030BBF93A10DBF8642003F1C5
:10476000010E07EE901A0A44BEF1010FCBF890E05B
:10477000CBF86420F8EEE77A03F01F81DBED205AD6
:10478000DBED226A07EE10EA37EEE56AB8EEC75AAB
:10479000012F86EE057A37EE257A77EEC77A8BED14
:1047A000217AE7EE866A8BED207AF0EE667ACBED21
:1047B000236ACBED226A03F03685DBF8A430BBF91F
:1047C0003C10DBF8682003F1010E07EE901A0A4452
:1047D000BEF1010FCBF8A4E0CBF86820F8EEE77A41
:1047E00003F00681DBED255ADBED276A07EE10EAC0
:1047F00037EEE56AB8EEC75A012F86EE057A37EE36
:10480000257A77EEC77A8BED267AE6EE276A8BED6E
:10481000257AF0EE667ACBED286ACBED276A03F0B5
:10482000F484814CA8F80600BBF8A820059B013A47
:104830001D78ABF8A82008990022072D4A608A60ED
:10484000CA6040F05781F8F745FF059BDFF82C82DE
:104850001D78079BC01A94F82831A8F80000099326
:10486000002B40F04D816E4A5279002A01F09A8166
:104870006E4A1278013AD2B2072D84F8282102F04C
:10488000598200230B936A4BD4F83421D3F800A04B
:10489000624B0893079B9FED676AD4ED4C9A66497B
:1048A000DFF8DC81D1ED006AC4F834319A1A07EEE2
:1048B000902AF8EE677AB7EE007AC6EE278A08F1FA
:1048C0001C0300250A93DFF8BC915C4B5C4F0693F8
:1048D0002E4677EE69BA94ED4BCA9FED5A9ADFEDFA
:1048E0005AAA9FED5ABA9FED5AAA6BEEA6BAF4EEF9
:1048F000C7BAF1EE10FA88BFF0EE47BA554B98ED03
:10490000008A2B44D3ED007AF5EE407AF1EE10FAEE
:1049100017D0514B2B4493ED007A78EE476AB0EEF6
:10492000E66AF4EEC67AF1EE10FA08D5F5EEC06A42
:10493000F1EE10FACCBF37EE878A37EE678A83ED47
:10494000008A464B1A8893073FD0022E3DD0444B35
:104950009AF82E1033F9163007EE103A0A9B07EE3C
:10496000901A2B44F8EEE76AB8EEC77AD3ED007AD6
:104970004B42A6EEA77A700007EE903AF8EEE77A7F
:10498000B4EEE77AF1EE10FA0AD407EE901AF8EED8
:10499000677AF4EEC77AF1EE10FA88BFF0EE477A44
:1049A000304B31490344085EB3F90C30C31A07EEAB
:1049B000103AB8EEC77AD007E7EE497A41F188801D
:1049C0002A4B93ED008A27EE888A089B94F86C2185
:1049D0002B4493ED01DA78EE4DCA002A00F0F18005
:1049E000234BD4F8702107991B688A1A9A4240F326
:1049F000E8809AF84830022B02F00382022E04F07D
:104A000068851C4B1B68990700F192801A4B87ED53
:104A100000BA1B689342C0F2C48035E0B07A00202F
:104A2000C07200208C7C0020942300207095002010
:104A30008465002000247449B42C00207C490020A7
:104A400088490020CDCCCC3DAE47813F000000001E
:104A50000000C842A82C0020D82400208065002037
:104A6000E42400207C95002030650020902C00205C
:104A7000BC2C00202C650020B82C0020907C00204D
:104A8000CC24002094490020F7EE007AF4EEE79A57
:104A9000F1EE10FA40F1958008991F4BD1ED017AA3
:104AA00093ED007AF0EEE77AF4EEC77AF1EE10FAC1
:104AB00040F18780D1ED027AF0EEE77AB4EEE77A42
:104AC000F1EE10FA7DDDD1ED037AF0EEE77AB4EE87
:104AD000E77AF1EE10FA74DD104B1B689B0760D586
:104AE0000F49104B44E0104B104C1D780593072DD7
:104AF0003FF4A9AE94F828310993002B3FF4B3AEEC
:104B0000013B84F82831012D01F0CF8217B0BDECB4
:104B10000C8BBDE8F08F00BFC42C00202C6500205A
:104B2000306500207C9500208C7C002094230020A0
:104B3000D24BD349DFF8C4E331F916C09EED008AA9
:104B4000DFF8BCE387ED00BA03EB460028EE098AE4
:104B5000B0F90C00A0EB0C0007EE900AF8EEE77A33
:104B6000DEF8000027EE888A904278EE4DCA8BDA94
:104B7000B3F90C20B1F900E0C248AEEB020E0068B8
:104B80008EEAEE72A2EBEE7282421ADAB3F90E30BE
:104B9000B1F90220D21A82EAE273A3EBE2739842DF
:104BA0000FDDB94B1A88002384F86C31002A43F0DA
:104BB000F486B64AB64B1178186881F00101F9F70E
:104BC00089FAB44B2B4493ED000A069B2CEE000AA5
:104BD000022E20EE2C0AA3EC010A069304F0A48412
:104BE000AD4BD7ED006A93ED007AAC4BD3ED007A74
:104BF000AB4B93ED006AAB4B67EE277A2B4427EE65
:104C0000AB7AD3ED007A67EE277AF0EE665AECEED7
:104C1000A75AB1EE467AB4EEE57AF1EE10FA08DC66
:104C2000B4EEE56AF1EE10FA8CBFB0EE657AB0EE44
:104C3000467A94ED4C6AF7EE007AB4EEE76AF1EE4C
:104C400010FAACBF0123002343B1F0EEE66AF0EEA8
:104C5000C77AF4EEE67AF1EE10FA01D587ED007A24
:104C6000022E04F0E283904A904B52F826001B6813
:104C7000B0EE4D0A98478E4A8E4B52F826001B68BC
:104C800098479AF8373023B18B4B1B88002B00F0E4
:104C90008C87B0EE4B8A894B38EE400A2B4493ED5B
:104CA000008A83ED000A9AF8483030EE480A20EE78
:104CB000288A002B33D0824B1B7813F0010300F0BD
:104CC000CC86F7EE007AF4EEE79AF1EE10FA94F85B
:104CD0006C31C1F25D85002B01F00C80D4F870318D
:104CE000079AD31A774A12689A4218DD764BD3EDA9
:104CF000007AF0EEECCAF4EEE7CAF1EE10FA42F1F7
:104D00009180614B1A88002384F86C31002A00F0EE
:104D1000B0866E494A6912B10A6813604B746C4BD5
:104D200094F87C212B4493ED000A2CEE000A20EE2F
:104D3000088A89ED008A32B9069B87ED00BA03ED37
:104D400001BA89ED00BA0136032E08F1040809F111
:104D5000040907F1040705F104057FF4CFAD059BB5
:104D60001A78072A01F02A85012A01F0D08700234A
:104D7000069394F88421002A41F0A481DFF884A1ED
:104D8000544BDAF800201968D60491F82C0000F191
:104D90002787DFF87491504AB9F81A3092ED006A0B
:104DA0004E4A4F4DD2ED005AD5ED036A4D4A84ED7F
:104DB000656A07EE103A4C4B92ED005AD3ED007A3B
:104DC000D3ED013AD3ED024A84ED636AB8EEC77AB7
:104DD00035EEC64A012236EEC77A84ED624AC4ED4A
:104DE000665A84F89C21C7EE055A0A8D534206EE96
:104DF000103A3E4BDFED3E6A93ED005A3D4B93ED8A
:104E0000004AB7EE007AF4EEC75A35EE045AF1EED6
:104E100010FA88BFF0EE475A35EE275AB8EEC66A48
:104E2000F4EEE65AF1EE10FA07EE902AB4EEC65A06
:104E3000B8BFF0EE665AF1EE10FAC4ED695AB8EE5A
:104E4000677A01F12C83B4EEC75AF1EE10FA88BFED
:104E5000B0EE475A254BDFED286AD3ED017A254B9A
:104E600093ED014A77EE847A25EE265A77EEA37AFF
:104E7000B4EEE76AF1EE10FA51DC47E07C950020D1
:104E800030650020C02C0020EC5D0020EE5D00208D
:104E9000F05D0020642C00200828002098000020ED
:104EA000D82C0020702C0020102800200C28002076
:104EB000642800206028002080650020082500204C
:104EC000644A0020BC2C0020C82C0020F45D002087
:104ED0007C2C002084650020CC9300204C95002081
:104EE0009C7D0020702D0020884900207C490020F6
:104EF00000000000944900206F12833A902C00209B
:104F0000B82C0020C07A00209C710020B4EEE77A13
:104F1000F1EE10FA8CBFB0EE676AB0EE476AEC4B68
:104F20004A8DD3ED027A9FEDEB7A534204EE103AAC
:104F300074EEA77AB8EEC44A26EE076AF4EEC47A95
:104F4000F1EE10FA0AD407EE102AB8EE474AB4EE92
:104F5000E74AF1EE10FA88BFB0EE674ADE4ADFEDAD
:104F6000DD7A527824EE274A0AB9B1EE444A002885
:104F700041F06486B7EE003AD84E3278002A02F04B
:104F8000DB87D749DFEDD77AD1ED024AD1ED016A4F
:104F900091ED037A66EE244AE5EE264AE4EE074AEE
:104FA00063EE244AF4EEE74AF1EE10FAB4BFF0EEF5
:104FB000673AF0EE643A98BFF0EE647A012ACDEDDC
:104FC0000E4A02F0DE8791ED067AD1ED052AD1ED89
:104FD000076A26EE077AA5EE227AA4EE267A23EE59
:104FE000077AB4EEE77AF1EE10FAB4EEE37A8CBF0A
:104FF000F0EE676AF0EE476AF1EE10FA88BFF0EE65
:10500000676AB4BFF0EE637AF0EE477A022A8DED5C
:105010000F7A00F0DE8091ED0A7AD1ED092AD1ED08
:105020000B3A26EE077AA5EE227AA4EE237A23EE37
:10503000077AB4EEE67AF1EE10FAB4EEE77A8CBFB6
:10504000F0EE663AF0EE473AF1EE10FA98BFF0EE65
:10505000636AA8BFF0EE477A032A8DED107A00F05C
:10506000B88091ED0E7AD1ED0D2AD1ED0F3A26EEF2
:10507000077AA5EE227AA4EE237A23EE077AB4EE1D
:10508000E67AF1EE10FAB4EEE77A8CBFF0EE663A0B
:10509000F0EE473AF1EE10FA98BFF0EE636AA8BF5F
:1050A000F0EE477A042A8DED117A00F09280D1ED6E
:1050B000123AD1ED112A91ED137A66EE233AE5EE1C
:1050C000223AE4EE073A63EE233AF4EEE63AF1EEE2
:1050D00010FAF4EEE73A8CBFB0EE667AB0EE637A7F
:1050E000F1EE10FA98BFF0EE476AA8BFF0EE637ACF
:1050F000052ACDED123A6CD0D1ED163AD1ED152A34
:1051000091ED177A66EE233AE5EE223AE4EE073A9D
:1051100063EE233AF4EEE63AF1EE10FAF4EEE73AF3
:105120008CBFB0EE667AB0EE637AF1EE10FA98BFFB
:10513000F0EE476AA8BFF0EE637A062ACDED133A87
:1051400047D0D1ED1A3AD1ED192A91ED1B7A66EECE
:10515000233AE5EE223AE4EE073A63EE233AF4EE20
:10516000E63AF1EE10FAF4EEE73A8CBFB0EE667A6A
:10517000B0EE637AF1EE10FA98BFF0EE476AA8BF7E
:10518000F0EE637A072ACDED143A22D091ED1E7A23
:10519000D1ED1D2AD1ED1F3A26EE077AA5EE227A2F
:1051A000A3EE847A27EE037AB4EEE67AF1EE10FAF3
:1051B000B4EEE77A8CBFB0EE666AB0EE476AF1EE05
:1051C00010FA8DED157A98BFF0EE466AA8BFF0EEA2
:1051D000477A77EEE67AF7EE006AF4EEE67AF1EED9
:1051E00010FAC4ED4C7A43F32E8786EEA77A022A92
:1051F000DDED0F7A67EE244A67EE877ACDED0E4A31
:10520000CDED0F7A2DD0DDED107A67EE877A032A87
:10521000CDED107A25D0DDED117A67EE877A042A7C
:10522000CDED117A1DD0DDED127A67EE877A052A71
:10523000CDED127A15D0DDED137A67EE877A062A66
:10524000CDED137A0DD0DDED147A67EE877A072A5B
:10525000CDED147A05D0DDED157A27EE877A8DED48
:10526000157A2149096811F080530A9301F04782A9
:10527000F6EE005AC4ED695A002A02F0F88594F956
:105280009C311A4994ED666AC87894ED655ADAF84B
:105290000010DFF868E0164FDEED004AB7F906E0CF
:1052A000B9F81A700B9707EE103A124BD4ED626AF8
:1052B0001D78114BD4ED637A1B780893BDEEC66A56
:1052C00001F4805316EE10CABDEEC56A0D9317E0C7
:1052D0007C4900206F12833AD84900205C9100205D
:1052E000E02C00200000000030950020442F00201A
:1052F00080910020644A0020AC670020DC2C002054
:1053000001F4800301F01007B8EEC77A0C9305F0A2
:10531000010816EE101A002840F02887002F41F0EF
:105320005C83D04D9DED0E5A95ED006ACE4825EE7A
:10533000866AA5EE076AB0EE675AA6EE265ABDEE5B
:10534000C56A16EE10EA16EE107AE645A8BF674663
:105350007145C8BF0F4606EE107AB8EEC66A012A3C
:1053600080ED006A00F0DC8095ED046A9DED0F5A37
:1053700025EE866AA5EE076AB0EE675AA6EE265AB3
:10538000BDEEC56A16EE10EA16EE107AE645A8BF25
:1053900067467145C8BF0F4606EE107AB8EEC66A7A
:1053A000022A80ED016A00F0BB8095ED086A9DED50
:1053B000105A25EE866AA5EE076AB0EE675AA6EE89
:1053C000265ABDEEC56A16EE10EA16EE107AE645CC
:1053D000A8BF67467145C8BF0F4606EE107AB8EE03
:1053E000C66A032A80ED026A00F09A8095ED0C6A85
:1053F0009DED115A25EE866AA5EE076AB0EE675A52
:10540000A6EE265ABDEEC56A16EE10EA16EE107A22
:10541000E645A8BF67467145C8BF0F4606EE107A3D
:10542000B8EEC66A042A80ED036A79D095ED106A59
:105430009DED125A25EE866AA5EE076AB0EE675A10
:10544000A6EE265ABDEEC56A16EE10EA16EE107AE2
:10545000E645A8BF67467145C8BF0F4606EE107AFD
:10546000B8EEC66A052A80ED046A59D095ED146A33
:105470009DED135A25EE866AA5EE076AB0EE675ACF
:10548000A6EE265ABDEEC56A16EE10EA16EE107AA2
:10549000E645A8BF67467145C8BF0F4606EE107ABD
:1054A000B8EEC66A062A80ED056A39D095ED186A0D
:1054B0009DED145A25EE866AA5EE076AB0EE675A8E
:1054C000A6EE265ABDEEC56A16EE10EA16EE107A62
:1054D000E645A8BF67467145C8BF0F4606EE107A7D
:1054E000B8EEC66A072A80ED066A19D095ED1C6AE7
:1054F0009DED155A65EE865AE7EE055AE6EEA57A59
:10550000FDEEE77A17EE905AAC45A8BFAC46A9422B
:10551000D8BF614607EE901AF8EEE77AC0ED077A39
:10552000B8F1000F00F03087504A1268002A40F0AE
:1055300038874F4A127892B1307868B14A4FDFF815
:1055400054810025E8B2D8F80030B7EC010A98473A
:10555000307801358542F5DB464A12689047059B55
:105560001A78072A01F0198100230693DAF800203F
:10557000510501F10480404B1E68320700F1A487F9
:105580003E4B1B78BBB13E4AB9F81A30B2F906203F
:105590009A4210DC3B4B1B78012B01F0D083192B76
:1055A00001F0CD830E2B06D0082B04D0364D0023FE
:1055B000AB60C4F8403194F8AE5125B1334B1B8831
:1055C000980741F07C8394F8B471002F40F0E28793
:1055D00099F81E30002B00F04584022B01F0638304
:1055E000032B41F05C8399F82030C3EB431203EBAB
:1055F0008202D20092B299F81F300233DBB2002F40
:1056000000F07685002A00F0738521490968B2FB15
:10561000F1F20FFA82F8A4F8E481002B03F0C781BD
:1056200007EE908AF8EEE77AF7EE006A86EEA77A40
:10563000154D012BD4ED7E6AD5ED007A77EEE67A32
:1056400067EE877AC4ED7A7A3CD0D5ED017AD4ED55
:105650007F6A77EEE67A022B67EE877AC4ED7B7A73
:1056600030D019E0E02C0020B0490020A0970020A5
:10567000D46A0020A86700202C650020D71C0020D9
:1056800080910020D84900209C7D0020806500206A
:10569000D4490020A0670020D5ED027AD4ED806ABD
:1056A00077EEE67A032B67EE877AC4ED7C7A09D031
:1056B000D5ED037AD4ED816A77EEE67A67EE877AE4
:1056C000C4ED7D7A059A1278092A03F0D782B8F1E1
:1056D000000F40F3CE839BB394ED7E7AD4ED7A7ABB
:1056E00077EE877A012BC4ED7E7AC5ED007A21D062
:1056F00094ED7F7AD4ED7B7A77EE877A022BC4ED36
:105700007F7AC5ED017A15D094ED807AD4ED7C7A5C
:1057100077EE877A032BC4ED807AC5ED027A09D043
:10572000D4ED817A94ED7D7A77EE877AC4ED817A33
:10573000C5ED037A013B022BB8BF0223DBB209930C
:10574000002F099E18BF0226CF4BDFEDD06A1A68E2
:10575000059B91781878137807EE903AF8EEE77A7F
:10576000B0EE007A67EEA67AF4EEC77AF1EE10FAA0
:1057700040F38086DFEDC66A37EEC77AB0EE676A1F
:10578000A7EE266AF0EE466A95ED007A9FEDC16AB3
:1057900027EE066AF0EEC65A84ED556AC4ED585AF3
:1057A00099B107EE101AB8EEC75A9FEDB87A66EEB7
:1057B000064A25EE075AB7EE007A37EE457A64EED0
:1057C000A54AA4EE857A26EE076A9FEDB37A53794F
:1057D00026EE877A27EE067ACBB1DFEDAC6A9FED35
:1057E000AF6A65EEA65A06EE903AF8EEE66A65EE06
:1057F000A65AF4EEC65AF1EE10FA01F3F781B7EEAD
:10580000006A76EE655AC6EE256A27EE267A0C28DF
:105810009FEDA38ADFEDA36A00F09F87B4EEC87AFC
:10582000F1EE10FA98BFB0EE478AB4EEE68AF1EED8
:1058300010FAB8BFB0EE668A84ED4E8A002E00F0F2
:10584000DC80B0EE007AF4EEC77AF1EE10FA05DDF6
:1058500037EEC77ADFED8E6AE7EE267A95ED017AAC
:10586000DFED8C6A27EE267AF0EEC75A84ED567A81
:10587000C4ED595A99B106EE901A9FED846AF8EE7C
:10588000E66A27EE075A66EE866AB7EE006A36EEDB
:10589000666A25EE255AA5EE266A27EE067ADFED22
:1058A0007E6A937967EEA67A67EE877AABB107EEE8
:1058B000103AB8EEC77A9FED756ADFED786A27EE89
:1058C000257A27EE067AB4EEE67AF1EE10FA41F385
:1058D0009181DFED756A67EEA67A0C2800F01E87CD
:1058E000DFED6F6A9FED6F7AF4EEE67AF1EE10FA73
:1058F00088BFF0EE667AF4EEC77AF1EE10FAB8BF20
:10590000F0EE477A012EC4ED4F7A76DD5378DFED65
:105910005F6A07EE903AF8EEE77AB0EE007A67EE4B
:10592000A67A537AF4EEC77AF1EE10FA05DD37EE77
:10593000C77ADFED576AE7EE267A95ED027ADFED5A
:10594000556A27EE267AF0EEC75A84ED577AC4EDF1
:105950005A5A9BB106EE903A9FED4C6AF8EEE66A11
:1059600027EE075A66EE866AB7EE006A36EE666A7A
:1059700025EE255AA5EE266A27EE067ADFED466A61
:10598000D37967EEA67A67EE877AFBB107EE103A15
:10599000B8EEC77A9FED3D6ADFED406A27EE257AC3
:1059A00027EE067AB4EEE67AF1EE10FA01F33081D2
:1059B000B5EEC07AF1EE10FA02F17484B7EE006A27
:1059C00036EE477AC6EE076A67EEA67A0C2800F034
:1059D0009D86DFED336A9FED337AF4EEE67AF1EEE1
:1059E00010FA88BFF0EE667AF4EEC77AF1EE10FA9C
:1059F000B8BFF0EE477AC4ED507A092800F07186FE
:105A000099F82150002D40F02686284B1E6800236F
:105A100084F8B431B50609D5254B1B8803F0300353
:105A200023B1244B1B78D80702F1AC81224B1B78A1
:105A300023B9224DAB78002B41F05781059B1D788F
:105A4000072D7FF460A8F7F745FE059A1C4B1578E3
:105A5000069A801AD880FFF756B894F86C21002A6D
:105A60003FF45DA9174A84F86C311288002A7FF44C
:105A700050A9154A154B1178186881F00101F8F703
:105A800029FBFFF74CB900BF886500200AD7233CEB
:105A9000D7A368416F12033B00004843A4707D3FC9
:105AA00000C0F94400C0F9C40000C8422C650020C1
:105AB0008065002082650020D9420020046100201A
:105AC000907C0020EC5D0020EE5D0020F05D002069
:105AD00094ED587AB1F90000D4ED596AB1F902E0B9
:105AE000E54AF4EEC76A80EAE0738EEAEE71A3EB52
:105AF000E073F1EE10FAA1EBEE71B4BFB0EE476ABD
:105B0000B0EE666A8B42B8BF0B4607EE103A1378C8
:105B1000B8EEC77A27EE097A002B40F0BC80D74B4D
:105B2000D3ED005AF4EEEA5AF1EE10FA41F1C280D8
:105B3000B7EE005A75EE654ADFEDD16A9FEDD15A96
:105B4000D14B36EEC77A24EE855AD3ED006AE5EEE6
:105B5000075A65EEA65AF5EEC05AF1EE10FA40F279
:105B6000CA85CAEE256AB7EE007AF0EE475AE6EE2D
:105B7000665AF0EE656AF4EEC76AF1EE10FA88BF75
:105B8000F0EE476AF5EEC06AF1EE10FAB8BFF0EE3B
:105B90004B6ABE4B93ED007A67EE877AA7EEA68A32
:105BA000FEF713BF0122FEF767BEB94BB94A2B447B
:105BB00093ED007AD2ED007AB74B67EE277AF7EED5
:105BC000006AF4EEE67AF1EE10FA93ED007A88BFFF
:105BD000F0EE667A67EE877A27EE888AFFF75BB881
:105BE000AE4BDFF8F4921A78D5075CBFB9F81820ED
:105BF000A4F89021AA4AAB4D1288D5ED037A07EE9E
:105C0000102AB8EEC77AF4EEC77AF1EE10FA42F233
:105C10008980A54D2B8807EE103AB8EEC77AF4EECE
:105C2000C77AF1EE10FAC1F29680A04AA04D92ED2B
:105C3000006AD5ED006A94F99C21C4ED656A76EEA0
:105C4000665A012AC4ED636AC4ED625A84ED666A3D
:105C500001F08586079BC4F8A031002537EEC77A8E
:105C6000FCEEE77A934E84ED697A17EE902AA4F859
:105C70009021012296ED005A84F89C218E4A95428B
:105C800042F23D808D4BD3ED007AD3ED013AD3ED56
:105C9000024AFFF7A8B87C4B93ED005AB5EEC05A04
:105CA000F1EE10FA40F32785854BD3ED006AF5EE4F
:105CB000C06AF1EE10FA40F31E8536EEC77A66EE42
:105CC0004A5A87EE266AC5EE856AB7EE007AB4EEC8
:105CD000C76AF1EE10FA88BFB0EE476AB5EEC06A47
:105CE000F1EE10FA76EE876AB8BFB0EE4B6A66EE58
:105CF000266A40E7734AD2ED007AB0EEC87AB4EE75
:105D0000E77AF1EE10FA7FF70AA86F4AD2ED007A2F
:105D1000B0EEEC7AB4EEE77AF1EE10FA7EF7FFAF70
:105D20006A4AD8ED007A92ED007AF0EEE77AF4EE66
:105D3000C77AF1EE10FA7EF5F2AF01220799C4F8A6
:105D4000701184F86C21FEF7CDBF07EE102A197888
:105D5000DFF88881C4F80C71B8EEC77AF7EE006AF4
:105D6000132986EE879AB8F90400B4F810619BED08
:105D7000070A01F03185564A564992ED001AD2EDD4
:105D8000053A92ED122A92ED173AD2ED091AD2EDA8
:105D90000E4A92ED016A92ED064A92ED0A7AD2ED30
:105DA0000F5AD2ED132AD2ED186A92ED045AD2EDB1
:105DB000030A67EE897A69EE288A29EE088AE1EEFD
:105DC000273A01EB86070025A2EE283AC4F80051D5
:105DD000C4F80451E1EE884AA6EE274AE7EE085AD5
:105DE00092ED167A92ED0D6A92ED021AD2ED0C1A2E
:105DF000C7ED003AE2EEA86A25EE635A27EE437A31
:105E000092ED0B2AD2ED152AC7ED204AA0EEE34A07
:105E100026EE646AD2ED143A82ED054AA1EE275AC5
:105E2000F0EE477AE1EEE45AA2EE086AE2EEC36AC7
:105E3000E3EEA87A82ED065AC2ED0E5A82ED0F6AA1
:105E400087ED403AC2ED176AC2ED187AC4F80851DE
:105E5000721C02F01F02A4F81021A8F80400059B90
:105E6000FEF709BCA4F8E4319846002F3FF4D2AD08
:105E70000C4D022668E400BF9C2C0020A42C0020BE
:105E800000003443610BB63B982C0020942C00207A
:105E9000F42400208C2C0020882C0020644A002050
:105EA000742D00209C7D0020762D00204C95002034
:105EB000602D00207C2D00208FD003008849002019
:105EC000A02C0020CC2C0020C82C0020D02C00209E
:105ED00044480020D84500209C710020907C002080
:105EE0008B4A1178D4F818718A4B9FED8B7AFE009B
:105EF0009A1982ED007A002979D08848B0EE476A75
:105F0000F0EE476A0022F0EC017A013267EEA77AE0
:105F100005EE902AB4EEE77AF1EE10FAF8EEE55AC3
:105F2000B8BFB0EE677A914276EEA76AA7EEA56A8F
:105F3000E9D1F5EEC06A9A19F1EE10FA82ED007A15
:105F400055DDC6EE265A764A76490988F7EE007A7C
:105F500075EEE75AD2ED007A65EEA77AFDEEE77AA4
:105F600017EE902A812A42F3B0818A42A8BF0A46DE
:105F700007EE902AF8EEE77A6B4AF01902EB8002FE
:105F800092ED057AD2ED003A92ED066A92ED014A61
:105F9000D2ED046AD2ED034A92ED025AA3EEA77A3B
:105FA000A4EE276A66EEC76AA7EE646ABDEEC77AFA
:105FB000E5EE276A17EE100A812882ED056AC2ED28
:105FC000066A42F37F818142A8BF014607EE901A1C
:105FD000F8EEE77AFCEEE77ACDED087ABDF82020FE
:105FE00099198A801FB9BEF1130F03F01E80BEF10C
:105FF000150F41F047811E44DFF84C81B28828F824
:106000001720D4F81451494A013582FB0532511941
:10601000EA17C2EBA102C2EBC202AD1AC4F81451D6
:106020004348D4F81C11079B424D02682D78C4F8F0
:106030001C31591A0A440260002D40F0B68107EE67
:10604000901A3D4EDFF818913C4FB8EEE78A06F201
:10605000447506F5F668F6EC017A9BED070ADBF865
:106060006C37F8EEE77A284627EE800A9847A5F1C4
:10607000E000DBF88C369847A5F17000DBF8FC36C1
:106080009847D6F85006DBF8AC309847D7ED007A41
:10609000A9EC010AE0EE087A2435A845E7EC017A7C
:1060A000D9D1059B1D78FEF722BD254B254A1968DD
:1060B0001288254BC96919805A8017B0BDEC0C8B2A
:1060C000BDE8F08F214B224E1A7812F0010F327882
:1060D00040F0B283002A00F0AB8592001D491E48B3
:1060E000DFF880A0DFF8809025F0D4FDFFF71CBA20
:1060F000B4F8E48108F1FF380FFA88F8B8F1000F1E
:10610000A4F8E4817FF7B1AE144DFFF7E4BA00BF05
:10611000BA450020B0480020000000009423002071
:10612000BC450020B8450020D84700209324499260
:10613000CC270020AC45002000730020D027002091
:1061400078660020943F0020907C0020644A002064
:106150005C9100206C420020B04900209C7D002012
:10616000B47A0020C07A00209C710020002F00F03B
:106170004D87B8F1000F42F03384089BCA4D002BC5
:1061800042F0BD8295ED006A9DED0E5AC74825EE9E
:10619000866AFDEEE44AA5EE076AB0EE675AA6EEFF
:1061A000265A14EE901ABDEEC56A16EE10EA16EEE7
:1061B000107AE645A8BF67467145C8BF0F4606EE90
:1061C000107AB8EEC66A012A80ED006A00F0DF801E
:1061D00095ED046A9DED0F5A25EE866AA5EE076AD5
:1061E000B0EE675AA6EE265ABDEEC56A16EE10EA64
:1061F00016EE107AE645A8BF67468E45B8BF0F4633
:1062000006EE107AB8EEC66A022A80ED016A00F046
:10621000BE8095ED086A9DED105A25EE866AA5EEC2
:10622000076AB0EE675AA6EE265ABDEEC56A16EEAC
:1062300010EA16EE107AE645A8BF67468E45B8BF4D
:106240000F4606EE107AB8EEC66A032A80ED026A9F
:1062500000F09D8095ED0C6A9DED115A25EE866A41
:10626000A5EE076AB0EE675AA6EE265ABDEEC56ADD
:1062700016EE10EA16EE107AE645A8BF67468E4580
:10628000B8BF0F4606EE107AB8EEC66A042A80ED53
:10629000036A7CD095ED106A9DED125A25EE866A50
:1062A000A5EE076AB0EE675AA6EE265ABDEEC56A9D
:1062B00016EE10EA16EE107AE645A8BF67468E4540
:1062C000B8BF0F4606EE107AB8EEC66A052A80ED12
:1062D000046A5CD095ED146A9DED135A25EE866A2A
:1062E000A5EE076AB0EE675AA6EE265ABDEEC56A5D
:1062F00016EE10EA16EE107AE645A8BF67468E4500
:10630000B8BF0F4606EE107AB8EEC66A062A80EDD0
:10631000056A3CD095ED186A9DED145A25EE866A03
:10632000A5EE076AB0EE675AA6EE265ABDEEC56A1C
:1063300016EE10EA16EE107AE645A8BF67468E45BF
:10634000B8BF0F4606EE107AB8EEC66A072A80ED8F
:10635000066A1CD095ED1C6A9DED155A65EE865AAD
:10636000E7EE055AE6EEA57AFDEEE77A17EE905ACB
:10637000AC45A8BFAC46A942D8BF614607EE901A0B
:10638000F8EEE77AC0ED077A002A3FF4CDA8920034
:106390004749464825F07EFC464A1268002A3FF4E9
:1063A000C8A821F0F1FDFFF7C4B807EE901A424DDE
:1063B000424BDFF80C81DFF80C910694F8EEE78A87
:1063C00005F2D4660027CDF824801C46059BDBED42
:1063D000077A1B78172B51D095ED007AB8EEC78A53
:1063E000082B28EE278A07D1B0EE480A089325F03B
:1063F00091FD089BA8F80000DAF8002092000BD568
:10640000002F03F04B80B0EE480ADBF86C3706F142
:1064100070009847B0EE408AB0EE480ADBF88C3640
:10642000A6F170009847DBF8FC3630469847059B8C
:106430001B78032BB0EE408A2CD0D5F85406DBF83D
:10644000AC30B0EE480A9847D9ED007AA4EC010AC6
:10645000E0EE287A0137032F06F1240608F102083E
:1064600005F10405E9EC017AB0D1059B069C1D7885
:10647000FEF73DBBF0EE676AFFF786B995ED007A4F
:106480000BEB4702B8EEC78A128FA8F8002028EE5F
:10649000278AB1E725F03EFDA8F80000CDE7B0EE71
:1064A000465AFEF7D7BC00BFE02C0020B0490020C0
:1064B0006C420020A097002000730020B47A0020D6
:1064C000907C0020D0270020C74DD5ED027AB2EE97
:1064D0000E7AF0EEE76AF4EEC76AF1EE10FA41D5F3
:1064E000C24B1B885B073DD5C14BC24AB3F9043090
:1064F000C14982FB03020988DB17C3EBA2035B1AC5
:106500009BB219B211F1B30FBCBF03F5B47319B24A
:10651000B329C4BFA1F5B47319B2B84BB84A1B79FB
:106520001278002B4FF6FF7318BF012317077FF572
:1065300027A8B44A126811FB03F3117EB24A9BB23A
:1065400011FB03F382FB03121A44DB17C3EB221384
:1065500007EE103AB8EEC77A77EEC77AC5ED027A41
:10656000FFF70EB8A24BA34AB3F90430A24982FB4D
:106570000302DB17C3EBA2030B80FFF701B8DBF8C4
:106580000830002B3EF4F7AFA049A1F14C0098472A
:10659000FEF7F1BF9E4A9F4BD2F8EC201B6844F6F1
:1065A00020618A42A8BF0A46B2F57A7FB8BF4FF48D
:1065B0007A7292B213F0100FA4F8B621DAF8003014
:1065C00000F0C483DB0441F176868E4BD3F800E003
:1065D000BEF832004008844D8F49D4F8B831D5ED6B
:1065E000037AA1FB02129109642292FBF1F2142AB0
:1065F000BDEEE77A04EB4305A8BF142201339A42AB
:10660000C4F8B83117EE10CADCBF0023C4F8B831A3
:1066100004EB4303A5F8BCC1B3F9BC3107EE103A53
:10662000B8EEC77A77EEC77AFDEEE77ACDED087A55
:10663000BDF9202082EAE273A3EBE273834201F307
:10664000C987764A4FF07E531360FEF7C1BF744B83
:106650000593744CE4E41E216E48F3F799FC00287E
:106660003FF4D3A9614B1B885E063FF5CEA994F891
:106670000832AB4242F01E83684BD4ED837AD3EDEF
:10668000016A94ED505ADFED685A9FED686A27EE73
:10669000C57A68EE277AA8EE267AE5EE267AB4EE79
:1066A000E57AF1EE10FA88BFB0EE657AB4EEC67AFC
:1066B000F1EE10FAF4EEE57AB8BFB0EE467AF1EEFC
:1066C00010FA88BFF0EE657AF4EEC67AF1EE10FAB1
:1066D000B8BFF0EE467A84ED4E7AC4ED507AFFF7FB
:1066E00094B9FDEEC87A524A17EE903AA2F80480A7
:1066F000D380FFF785B9DFED4F6AFFF74ABADAF8C2
:10670000001048023EF5B4ADFEF7B6BDBDEEE77A27
:10671000474B17EE102A9A80FFF75BB99FED427A3C
:10672000DFED426A4249F4EEC77AF1EE10FA98BF03
:10673000B0EE677AFDEEE77AB4EEE67AF1EE10FAA3
:1067400017EE903AB8BFB0EE667A012E84ED4F7A1C
:106750004B803FF7DBA8FFF753B9B4EEC87AF1EEF0
:1067600010FA98BFB0EE478ABDEEC77AB4EEE68A5B
:106770002F4FF1EE10FA17EE103AB8BFB0EE668A5E
:1067800084ED4E8A3B80002E7FF45BA8FFF738B97A
:10679000002B3EF4C4AAFEF7A1BAF6F79BFF059BB7
:1067A00023491A78069B072AA0EB030088807EF411
:1067B000DBAEF6F78FFF0690FEF7D8BEF6F78AFF3E
:1067C000059BDFF86C801A780B9B012AA0EB030075
:1067D000A8F8020000F09D82072A7EF4C8AAF6F706
:1067E00079FF0690FEF7C5BA9C7D002080650020E9
:1067F0003065002067666666483E0020749500207C
:1068000082650020846500208988888820730020A4
:106810007811002030950020D34D621098000020A0
:106820008C7C00209423002000C0F94400C0F9C4EF
:10683000907C002000000000002A00F0F981D4EDD7
:10684000593A94ED584AD4ED637AF34994ED627A5B
:1068500091ED005AD4ED565A94ED556AEF4DF0483B
:10686000F4EEC43AF3EE046AF1EE10FA77EEA64ABB
:1068700000F1E78295ED026A26EE656AB0EE674A9E
:10688000A6EE074AB4EEE44A34EE666AF1EE10FA78
:1068900048BFB0EE456A012A80ED006A00F0C88169
:1068A00095ED066A26EE656AB0EE674AA6EE074ADF
:1068B000B4EEE44A34EE666AF1EE10FA48BFB0EE88
:1068C000456A022A80ED016A00F0B28195ED0A6AFC
:1068D00026EE656AB0EE674AA6EE074AB4EEE44AD1
:1068E00034EE666AF1EE10FA48BFB0EE456A032A4C
:1068F00080ED026A00F09C8195ED0E6A26EE656AD5
:10690000B0EE674AA6EE074AB4EEE44A34EE666A91
:10691000F1EE10FA48BFB0EE456A042A80ED036A32
:1069200000F0868195ED126A26EE656AB0EE674A40
:10693000A6EE074AB4EEE44A34EE666AF1EE10FAC7
:1069400048BFB0EE456A052A80ED046A00F0708108
:1069500095ED166A26EE656AB0EE674AA6EE074A1E
:10696000B4EEE44A74EE666AF1EE10FA48BFF0EE57
:10697000456A062AC0ED056A00F05A81D5ED1A6A0B
:1069800066EEE56AB0EE674AA6EE874AB3EE046AA1
:10699000B4EEE44A74EE466AF1EE10FA48BFF0EE47
:1069A000456A072AC0ED066A00F04281D5ED1E6AED
:1069B000DFF874A2DFF8749266EEE55AE5EE877AA6
:1069C000F4EEE47A77EEC67AF1EE10FA48BFF0EE14
:1069D000457AC0ED077AFEF7A7BDB8F1000F41F088
:1069E000E2828E4D9DED0E5A95ED006A8C4825EEA3
:1069F000866AA5EE076AB0EE675AA6EE265ABDEE85
:106A0000C56A16EE10EA16EE107AE645A8BF67468C
:106A10007145C8BF0F4606EE107AB8EEC66A012A65
:106A200080ED006A3FF4B3AC95ED046A9DED0F5A1A
:106A300025EE866AA5EE076AB0EE675AA6EE265ADC
:106A4000BDEEC56A16EE10EA16EE107AE645A8BF4E
:106A500067467145C8BF0F4606EE107AB8EEC66AA3
:106A6000022A80ED016A3FF492AC95ED086A9DED33
:106A7000105A25EE866AA5EE076AB0EE675AA6EEB2
:106A8000265ABDEEC56A16EE10EA16EE107AE645F5
:106A9000A8BF67467145C8BF0F4606EE107AB8EE2C
:106AA000C66A032A80ED026A3FF471AC95ED0C6A68
:106AB0009DED115A25EE866AA5EE076AB0EE675A7B
:106AC000A6EE265ABDEEC56A16EE10EA16EE107A4C
:106AD000E645A8BF67467145C8BF0F4606EE107A67
:106AE000B8EEC66A042A80ED036A3FF450AC95ED17
:106AF000106A9DED125A25EE866AA5EE076AB0EE81
:106B0000675AA6EE265ABDEEC56A16EE10EA16EED4
:106B1000107AE645A8BF67467145C8BF0F4606EE26
:106B2000107AB8EEC66A052A80ED046A3FF42FACED
:106B300095ED146A9DED135A25EE866AA5EE076A57
:106B4000B0EE675AA6EE265ABDEEC56A16EE10EAFA
:106B500016EE107AE645A8BF67467145C8BF0F46D6
:106B600006EE107AB8EEC66A062A80ED056A3FF492
:106B70000EAC95ED186A9DED145A25EE866AA5EEC9
:106B8000076AB0EE675AA6EE265ABDEEC56A16EE43
:106B900010EA16EE107AE645A8BF67467145C8BFF1
:106BA0000F4606EE107AB8EEC66A072A80ED066A2E
:106BB0003FF4EDAB95ED1C6A9DED155A65EE865AD6
:106BC000E7EE055AE6EEA57AFDEEE77A17EE905A63
:106BD000AC45A8BFAC46A942C8BF8C4607EE90CAD8
:106BE000F8EEE77AC0ED077AFFF7CEBBDFED0D6A6E
:106BF000FEF70BBEB5EEC07AF1EE10FA01F13C8360
:106C0000B7EE006A36EE477AC6EE076AFEF763BE55
:106C1000DFED046AFEF7D8BEDC2C0020E02C00205B
:106C2000B04900200000C842C07A00209C710020BA
:106C3000DFF8CCA3DFF8CC93FEF776BCDA494A79CB
:106C4000002A3EF497A9D94A1278002A3EF492A964
:106C50000B78D749DFEDD74A07EE903A0B88B8EEAC
:106C6000677A07EE902A06EE903AF8EEE77AF8EEA9
:106C7000666A67EE277AB7EE007A87EEA63AB4EE38
:106C8000E43AF1EE10FA88BFB0EE643AB4EEC73AD7
:106C9000F1EE10FAB8BFB0EE473AFEF76DB9C64B49
:106CA0005A88FEF7A8BCB4F8B62102F57A7292B2FF
:106CB000FEF7A1BCC14BD3ED005AFEF74CBFC04B51
:106CC0009FEDC07AD3ED087AF4EEC77AF1EE10FAB0
:106CD00000F226859FEDBC7ABC4DD5ED037A77EEA8
:106CE000877AC5ED037AFEF76EBCB94E3278013A69
:106CF0000A2A72D8DFE812F0E107F807A907880727
:106D0000700756074107E4051C075D00DA06DFF847
:106D1000F882F6F7DFFCAF49D4F8802109680690C5
:106D2000821A511AC4F88001A8F80420A8F80610A5
:106D3000FEF71FB8F6F7CEFC0B90FDF7A4BDA64BEF
:106D40009B7B002B3EF432ACFEF735BCD9003FF5FF
:106D500039ACFEF73DBCB4F89051954240F22B851A
:106D600094F8A851002D41F0BD809C4A9C4E92EDB4
:106D7000007AD6ED007A94F99C21C4ED657A77EE1D
:106D8000676A012AC4ED637AC4ED626A84ED667AAB
:106D900002F06281079BC4F8A031924A9FED8A7A83
:106DA00092ED005A84ED697A012284F89C21FEF765
:106DB00065BF8D4B1B78002B02F054811A200AF01E
:106DC00049FC002842F04E81884B1B78002B42F092
:106DD0004981092333701FF06DFE2B79012B00F0E0
:106DE0008585022B7EF42AAE3378012B7EF426AE05
:106DF0007E4B1B78002B7EF421AE1FF0DDFAFEF7F0
:106E00001DBE7B4B1B88002B40F03886794A7A4B9D
:106E100011781868F7F75EF9D4F87021079B9A1A71
:106E2000FDF7ECBD754BD8ED007A93ED007AF0EEEE
:106E3000E77AF4EEC77AF1EE10FA7DF770AFFDF75E
:106E400060BFD5ED015A65EEC65AB0EE674AA5EEB1
:106E5000874AB4EEE44A74EE665AF1EE10FA48BF7F
:106E6000F0EE455A012AC0ED005A3FF4E1AED5EDEF
:106E7000055A65EEC65AB0EE674AA5EE874AB4EEEB
:106E8000E44A74EE665AF1EE10FA48BFF0EE455A45
:106E9000022AC0ED015A3FF4CBAED5ED095A65EE9A
:106EA000C65AB0EE674AA5EE874AB4EEE44A74EEDD
:106EB000665AF1EE10FA48BFF0EE455A032AC0EDCB
:106EC000025A3FF4B5AED5ED0D5A65EEC65AB0EE96
:106ED000674AA5EE874AB4EEE44A74EE665AF1EECC
:106EE00010FA48BFF0EE455A042AC0ED035A3FF4A9
:106EF0009FAED5ED115A65EEC65AB0EE674AA5EEC3
:106F0000874AB4EEE44A74EE665AF1EE10FA48BFCE
:106F1000F0EE455A052AC0ED045A3FF489AED5ED8E
:106F2000155A65EEC65AB0EE674AA5EE874AB4EE2A
:106F3000E44A74EE666AF1EE10FA48BFF0EE456A74
:106F4000062AC0ED056A3FF473AED5ED196A66EE08
:106F5000C66AB0EE674AA6EE874AF3EE045AB4EE6C
:106F6000E44A74EE656AF1EE10FA48BFF0EE456A45
:106F7000072AC0ED066A3FF45BAED5ED1D6ADFF867
:106F800080A0DFF8809026EEC66AE6EE077AF4EE7F
:106F9000E47A77EEE57AF1EE10FAB8BFF0EE457AD2
:106FA000C0ED077AFEF7C0BA1C6500209A7D00206C
:106FB000847D0020713DAA3F38980020982C002045
:106FC000A42700208FC2753C000000009C7D00209B
:106FD00002610020D4490020F07100204C9500206F
:106FE000602D00207C2D0020DA4900209C93002099
:106FF000EC5D0020EE5D0020F05D0020D02C002034
:10700000C07A00209C710020907C0020089BD94D04
:10701000002B41F0688195ED006A9DED0E5AD6482F
:1070200025EE866AFDEEE44AA5EE076AB0EE675AE1
:10703000A6EE265A14EE901ABDEEC56A16EE10EAB8
:1070400016EE107AE645A8BF67467145C8BF0F46E1
:1070500006EE107AB8EEC66A012A80ED006A3EF4A8
:107060005FAA95ED046A9DED0F5A25EE866AA5EE9E
:10707000076AB0EE675AA6EE265ABDEEC56A16EE4E
:1070800010EA16EE107AE645A8BF67468E45B8BFEF
:107090000F4606EE107AB8EEC66A022A80ED016A43
:1070A0003EF43EAA95ED086A9DED105A25EE866ADB
:1070B000A5EE076AB0EE675AA6EE265ABDEEC56A7F
:1070C00016EE10EA16EE107AE645A8BF67468E4522
:1070D000B8BF0F4606EE107AB8EEC66A032A80EDF6
:1070E000026A3EF41DAA95ED0C6A9DED115A25EE3B
:1070F000866AA5EE076AB0EE675AA6EE265ABDEE7E
:10710000C56A16EE10EA16EE107AE645A8BF674685
:107110008E45B8BF0F4606EE107AB8EEC66A042A4E
:1071200080ED036A3EF4FCA995ED106A9DED125ABC
:1071300025EE866AA5EE076AB0EE675AA6EE265AD5
:10714000BDEEC56A16EE10EA16EE107AE645A8BF47
:1071500067468E45B8BF0F4606EE107AB8EEC66A8F
:10716000052A80ED046A3EF4DBA995ED146A9DEDD5
:10717000135A25EE866AA5EE076AB0EE675AA6EEA8
:10718000265ABDEEC56A16EE10EA16EE107AE645EE
:10719000A8BF67468E45B8BF0F4606EE107AB8EE18
:1071A000C66A062A80ED056A3EF4BAA995ED186A0A
:1071B0009DED145A25EE866AA5EE076AB0EE675A71
:1071C000A6EE265ABDEEC56A16EE10EA16EE107A45
:1071D000E645A8BF67468E45B8BF0F46FEF77EB9A5
:1071E000664ED4ED017A94ED006A3188726977EECB
:1071F000A77AF0EE006AB0EE677AA6EE267A4E1E07
:1072000004EBC601D6EE267A08391032F6EE003AC3
:1072100027EE237A67EEA37A84ED207AC4ED217AF3
:10722000574C274604F1800091ED027A91ED036AF4
:10723000D7ED036AD7ED027A52ED014A12ED025AF8
:1072400037EE674A76EEC65A77EE277AE4EE845A2E
:10725000013EA1F10801E5EE047A07F1080702F109
:10726000080236EE267A00F10800E4EE877AE5EEB1
:10727000475A67EEA37A25EEA37AC0ED007A80ED37
:10728000017AD1D1BEF1140F7EF4BDAEF6F722FA29
:10729000069BDFF80081C01AA8F80200D4F8145148
:1072A000FEF7B1BED4F818C1B4F81031C3F1200212
:1072B0005FFA82F9334A03EB4C1702EB87075FEA68
:1072C000990201F0D486013216012F482F4907EBAD
:1072D000060807F1100212ED024A12ED035A12EDF0
:1072E000016A12ED047A50ED024A50ED035A50ED56
:1072F000016A50ED047A64EE244A65EE255A66EE82
:10730000266A67EE277A1032904541ED024A41ED38
:10731000035A41ED016A41ED047A00F1100001F1D8
:107320001001D8D11A48A6F110010F4400EB010852
:10733000214419F0030209D0B7EC017AF8EC017A84
:1073400067EE277A013AE1EC017AF5D1002B41F0A2
:107350005F81BEF1140F7EF456AEF6F7BBF9069BC3
:10736000DFF83080D4F81451C01AA8F80200FEF7F4
:107370004ABE00BFE02C0020B0490020C0450020DC
:1073800094230020D845002068470020A423002033
:1073900058470020907C0020D04E31785FEA910C55
:1073A00001F05887CE4F0CF101094FEA491907EB5C
:1073B000090807F12002A7F1700012ED076A52EDEB
:1073C000056A12ED037A52ED017A52ED025A12ED7E
:1073D000084A52ED064A12ED045A26EE066A66EE97
:1073E000A66A27EE077A67EEA77AA4EE046A20322F
:1073F0009045E4EEA46A00F11000A5EE057AE5EEF2
:10740000A57AF1EEC65AB1EEE66AF1EEC76AB1EEC0
:10741000E77A40ED085A00ED076A40ED066A00ED94
:10742000057ACAD1A9F120023A4404EB0C1711F0F5
:10743000030018BF08320FD052ED017A12ED027A24
:1074400067EEA77A0138E7EE077A02F10802B1EE9B
:10745000E77AA7EC017AEFD1BEF1140F01F028868C
:107460000135C4F81451FEF73DBD9E4E9E48B268EA
:10747000B18923F071FC059B93F800E0BEF1140F75
:1074800001F00986D4F814510135C4F81451A8E666
:10749000944E318873684FEA51094FEA89005FEAD8
:1074A000D10C04EB000204EB810500F0A18000F197
:1074B00010010CF1010C8D4F02EB0C1C2944103211
:1074C00003F1100E05F1100050ED032A50ED043ABF
:1074D00017ED043A17ED032A50ED026A10ED016A28
:1074E00017ED021A57ED010A11ED044A11ED035A86
:1074F00052ED044A52ED035A12ED027A52ED017A2E
:1075000051ED021A11ED010A73EE238A32EE228A3E
:1075100047ED048A07ED038A71EE268A30EE868AEB
:1075200047ED028A07ED018A74EE848A35EE858A7A
:1075300042ED048A02ED038A77EE218A37EE808AD3
:1075400042ED028A02ED018A73EE633A75EE655AE6
:107550001EED035A32EE623A74EE644A25EE638AF7
:107560001EED044A23EE052A64EE652AA3EE048A82
:107570001032944524EE843AA3EE842A07F11007D2
:107580000EF1100EA5EE853A00F1100001F1100188
:10759000E4EE852A00ED078A00ED082A01ED073A9E
:1075A00041ED082A5EED055A1EED065A71EE666A37
:1075B00030EEC66A31EEC77A70EE677A26EE253A6B
:1075C00065EEE63A25EE674A67EE054AE6EE053ACD
:1075D000A6EE853AA7EE254AE7EEA54A00ED063A63
:1075E00040ED053A01ED064A41ED054A7FF46CAFE6
:1075F0001FFA89F91A4649463B4815F007FD72689B
:107600004946284615F002FD059B1A78142A7FF496
:1076100045AE3BE6D4F8185135493648364BEA00BA
:10762000114415448A88196800EE102A643AC82A61
:10763000A8BFC822782AB8BF782207EE902AB8EEF1
:10764000C07AF8EEE77A00EB850577EE670A77EE09
:10765000876A67EE877A20EEA67AB8EE400AC7EE10
:10766000870A2846D5F81490D5F81880EF692E6A55
:1076700019F0B8FE059BC5F8149093F800E0C5F822
